:020000040800F2
:20000000F0FF0120CDB70608E1F40008E1CF040845B8060845B8060845B806080000000084
:20002000000000000000000000000000DDF40008D9F4000800000000D5F40008F506050839
:2000400045B8060845B8060845B8060845B8060845B8060845B80608AD17050875170508F4
:200060003D17050805170508CD160508A971060899710608897106087971060865710608E2
:20008000517106083D71060845B80608000000000000000000000000000000009516050811
:2000A000FDD404084DD50408EDD4040875D504083DD504082DD504081DD504086DAE0608BF
:2000C00075AE060861AE060869AE060845B8060845B80608C9080508110805080000000093
:2000E0005D16050845B80608990D010800000000000000000000000000000000297106081E
:2001000000000000954D06080DD5040845B8060800000000000000000000000000000000F6
:200120001571060801710608ED700608D9700608C5700608000000000000000000000000A6
:2001400000000000000000000000000075EE0008B17006089D700608897006085907050876
:2001600055AE06085DAE060800000000000000000000000000000000000000000000000055
:200180000000000045B80608000000000000000045B8060845B806086CB306000100000018
:2001A0000E02010002000000D07400203475002000000000D8F30708307500201402010049
:2001C00005000000F03900203C75002000000000DAF307083875002013020100040000003D
:2001E000D82B00204875002000000000E0F3070844750020031101000A0000001874002079
:200200005075002000000000E51901084C7500200D1001004C000000B06F00206075002073
:2002200000000000ED4C04085C7500200902010001000000186F0020B0750020000000008F
:20024000E4F30708AC750020FD01010024000000D06E0020B875002000000000EBDF0408D3
:20026000B4750020FB01010001000000E0690020E0750020000000005D590508DC75002025
:20028000FC01010009000000AC680020E87500200000000065590508E4750020F701010069
:2002A00006000000A0680020F875002000000000E6F30708F4750020F90101000400000013
:2002C0009C6800200476002000000000B9E0040800760020160215003F0000008C2D0020E0
:2002E0000C760020000000007D590508087600203400010010000000CC670020507600205D
:20030000000000002D9C02084C7600201102010008000000A46700206476002000000000E7
:20032000ECF307086076002012120100040000009C6700207076002000000000F4F3070891
:200340006C76002018300100380000006467002078760020000000000D6405087476002099
:20036000000201000B000000E8630020B476002000000000A1590508B0760020FF2101004C
:200380000500000094630020C4760020000000004D590508C0760020081203000F000000B2
:2003A000A0630020D076002000000000D5590508CC760020FA01010003000000005D00209B
:2003C000E476002000000000BD590508E07600202A020100080000000C520020EC760020D5
:2003E00000000000F8F30708E8760020205201000800000068500020F876002000000000A4
:20040000519C0208F47600200610010024000000A82C002004770020000000003D5A0508ED
:20042000007700200C02010004000000F84800202C77002000000000C55905082877002005
:20044000FE01010014000000203B00203477002000000000115905083077002026100100CD
:200460000E00000018E6002008E6002000000000C11E010804E600200B3001001A000000FA
:20048000B0DC00205CE600200000000000F4070858E600201F50010024000000DCDB002082
:2004A0007CE60020000000001CF4070878E60020050201000400000098DE0020A4E60020D1
:2004C0000000000040F40708A0E60020010201000B000000A0EC002028F60020000000003A
:2004E0009159050824F60020020201000300000098EC002038F600200000000000000000D1
:2005000034F600201B0201001000000084EC002040F6002000000000A95905083CF600201C
:200520001B2001000C000000B4E9002054F60020000000006983010850F6002021020100CD
:20054000F0000000E8E7002064F6002000000000719B010860F6002037100100300000003F
:200560003CEF002058F700200000000044F4070854F70020161001000600000040EC002096
:200580008CF700200000000074F4070888F700202F1001002200000000F6002098F700207B
:2005A000000000007AF4070894F7002023220100100000007CEB0020C0F70020000000005F
:2005C0009CF40708BCF700201E0001000900000068EB0020D4F7002000000000ACF4070874
:2005E000D0F70020052001000C00000014EC0020E4F7002000000000B8F40708E0F7002015
:20060000123001001000000050EB0020F4F7002000000000C4F40708F0F70020FD0701004E
:200620007C000000ACE6002008F8002000000000ED7C010804F80020F59101006C000000EB
:200640006CE7002088F80020000000001591010884F8002023200100100000009EEE00203C
:20066000F8F8002000000000250D0208F4F80020F62101000C00000014160120AC170120CF
:2006800000000000D4F40708A81701201C0202001C000000A4150120001801200000000054
:2006A000AD5E0508FC1701202830010016000000C01501202018012000000000F51A020817
:2006C0001C18012014000100050000009C1501203C18012000000000E0F407083818012010
:2006E000012001000C000000F40E01204818012000000000E6F40708441801200C40060070
:20070000E4000000140D0120581801200000000065E30308541801200A9001002400000083
:20072000D00C01204019012000000000DD0C02083C1901200E300300BC0100000C0B0120A3
:200740006819012000000000699C02086419012013100100040000002C130120281B01205E
:2007600000000000F4F40708241B01200101010004000000500A0120301B01200000000034
:20078000000000002C1B01200001010004000000480A0120381B012000000000F8F4070809
:2007A000341B01200201010003000000440A0120401B012000000000A5E303083C1B0120CC
:2007C000220201001C01000014110120481B012000000000B5600508441B01201500100046
:2007E00070000000E42701209029012000000000000000008C2901200300010001000000A8
:20080000DC270120042A01200000000000000000002A01202A00080060000000182201202D
:200820000C2A012000000000059C0208082A01202C00040010000000802A0120702A01209D
:2008400000000000ED9502086C2A0120292014007800000054250120942A01200000000007
:2008600000000000902A01201A0001000E000000AC240120102B012000000000FCF4070828
:200880000C2B01202B0012002400000088240120242B012000000000C1950208202B012096
:2008A0001902010010000000782401204C2B01200000000081590508482B012025201E00D9
:2008C0002C010000D02F0120A43301200000000000000000A0330120031201003D0000008C
:2008E00068320120D4340120000000000AF50708D0340120F831010006000000702C0120F4
:20090000183501200000000048F50708143501201010010002000000742F01202435012052
:20092000000000004EF50708203501201900010005000000EC2B01202C3501200000000016
:2009400050F5070828350120020001000C000000343E01204C3E0120000000000000000078
:20096000483E012029020100400000005C3701205C3E01200000000056F50708583E0120E4
:200980002C02010004000000043E0120A03E01200000000096F507089C3E01200A02010020
:2009A00014000000A83C0120C83E01200000000031E30308C43E01201A0201003C0000005C
:2009C000E84301203049012000000000F95D05082C490120382001000300000094410120E6
:2009E00070490120000000009AF507086C4901200400080080000000F04A0120704B0120E6
:200A00000000000000000000F04B01202802040004000000B0490120F84B012000000000CA
:200A2000395A0508F44B01202702040004000000AC490120004C0120000000002D5A05086E
:200A4000FC4B01201F020800100000009C490120084C01200000000029590508044C01207A
:200A60001D02020006000000B0540120DC5401200000000000000000D85401200612030071
:200A800012000000C05401206865012000000000795F050864650120270001000400000026
:200AA000004E012080650120000000009EF507087C6501200B2201003D00000034880120D5
:200AC000BC8E012000000000A4F50708B88E01200D12010014000000988D0120008F012072
:200AE00000000000E4F50708FC8E01201E02010006000000188C0120188F012000000000AF
:200B0000F8F50708148F0120100201000100000074A0012070A0012000000000FEF5070899
:200B20006CA001200403090412010002EF0201408304563200020102030100001201000200
:200B400002020040830440570002010203010000FFFFFFFF0000000000000000010000002D
:200B60000000000000000000EC39002000000000010000000000000000000000000000002F
:200B8000000000000000000000000000000000000000000000000000000000000000000055
:200BA000000000000060024010600240000000000000000000000000000B000000000000D6
:200BC00000000000000000000060024028600240010000000000000000000000060C000096
:200BE00000000000000000000000000000600240406002400200000000000000000000006F
:200C0000100D00000000000000000000000000000060024058600240030000000000000018
:200C200000000000160E0000000000000000000000000000006002407060024004000000D8
:200C40000000000000000000200F0000000000000000000000000000006002408860024099
:200C6000050000000000000000000000261000000000000000000000000000000060024097
:200C8000A060024006000000000000000000000030110000000000000000000000000000CB
:200CA00000600240B8600240070000000000000000000000362F00000000000000000000CC
:200CC000000000000064024010640240000000000000000000000000003800000000000080
:200CE000000000000000000000640240286402400100000000000000000000000639000040
:200D0000000000000000000000000000006402404064024002000000000000000000000045
:200D2000103A000000000000000000000000000000640240586402400300000000000000C2
:200D400000000000163B000000000000000000000000000000640240706402400400000082
:200D60000000000000000000203C0000000000000000000000000000006402408864024043
:200D800005000000000000000000000026440000000000000000000000000000006402403E
:200DA000A06402400600000000000000000000003045000000000000000000000000000072
:200DC00000640240B86402400700000000000000000000003646000000000000000000008C
:200DE000000000007D000000098500080585000801850008F5840008F1840008FD84000839
:200E0000F984000800000000A591000885A90008D58F0008E1AA0008759200088D850008B1
:200E20006585000849850008FDA2000875880008658A000861900008DD90000899940008A4
:200E4000798500085185000841850008010000000000803F813E010885430108FD3E010843
:200E6000E9120108CD140108F912010815130108C1120108B1120108000000000000000097
:200E800009022000010104C03209040000020806500507058102400000070501024000009F
:200EA00009026400030100C03209040000010300000009211101000122360007058303098C
:200EC000000A080B0102020201000904010001020201000524001001052401000204240249
:200EE000020524060102070582030800FF09040200020A000000070501024000000705812F
:200F00000240000009024300020100C03209040000010202010005240010010524010001D4
:200F2000042402020524060001070582030800FF09040100020A0000000705010240000054
:200F40000705810240000000FF000000140000FF0000000000000000AA550701000001AAFE
:200F600055050100002D202D2D202D2D2D2D202D2D2D2D00000000000000000000000000C7
:200F800000000000080000008CDE0608FF1FFF1F05010905A101A10005010930093109328A
:200FA000093309350934093609371581257F750895088102050919012908150025019508F3
:200FC00075018102C0C0000009022200010100E03209040000010301020009211101000106
:200FE0002236000705830309000A000000000000010203040102030406070809AA550B01B7
:201000000000AA5505010000AA550902000000AA5503009F01000000C0120000FFFFFFFF51
:2010200050E600200000000028E6002000000000010000000100000000000100E0017EFFCB
:20104000FFFFFFFFFF000000FFFFFFFF08FF0101FF01000001000000110202080000000072
:201060000000000038E50608000000000000000000000000DCFC060800000000000000005F
:201080000000000094FD060800000000000000000000000040FD0608000000000000000066
:2010A000850D0208EA0F012001010000F922020800000000000000005CFE06085926020862
:2010C000000000000000000014FE06082D202D2D202D2D2D2D202D2D2D00000000000000CE
:2010E000000000000000000000000000FFFFFFFFBD12020800000000000000006CFC0608A5
:2011000001000000FA00000001000000010000000101000000010101000000005A0E012044
:201120000000F40101000000580E01200000F40101000000560E01200000F40101000000C1
:20114000540E01200000F40101000000520E01200000F40101000000500E01200000F4012B
:20116000010000004E0E01200000F40101000000BD0A0208810A02080000000000E70608A0
:201180003E0E0120053201004C0E01206400F401010000004A0E01206400C409010000002A
:2011A0003C0E0120E803D007010000003A0E0120E803D00701000000380E0120E803D007AC
:2011C00001000000360E01201E00B80B01000000440E012005000F0001000000460E0120CA
:2011E00003000A0001000000340E01201E00F40101000000480E0120020000008CE7060870
:20120000320E01201400640001000000400E01203200E80301000000300E01200000C80040
:2012200001000000110D012000C80100100D0120005001000F0D0120005A01000D0D012043
:2012400002000000F4E606081C6A0708246A0708E80F01200100C40900000000E60F012076
:201260000100C40900000000E40F01200100C40900000000E20F01200100C40900000000DE
:20128000DE0F01200100C40900000000E00F01200100C40900000000DC0F01200100C409BA
:2012A00000000000DA0F01200100C409000000006F0A012000C801006E0A012000C8010091
:2012C0006C0A01200000FFFF0A0000006A0A01200100C80001000000680A012032003075A6
:2012E00032000000660A01207EFF140005000000640A012005002C0105000000630A012041
:20130000055A0500600A012000FF0100620A012002000000BC0800205E0A012003000000DF
:2013200044E006085F0A012000FF0100610A012002000000BC0800205D0A012003000000F4
:2013400044E00608BC090120FF7F0100B809012000000000FFFFFFFF01000000B409012039
:2013600000000000FFFFFFFF01000000B009012000000000FFFFFFFF01000000110A020874
:20138000A109020800000000DCE70608040F0120EE02CA0801000000020F012000C80100D6
:2013A00064000000010F012002C8010064000000000F01200200000098E70608560A012029
:2013C0000000803E05000000540A012080C1803E050000004E0A01200083007D0500000049
:2013E0004C0A012080C1803E05000000470A012000FF0100400A01206400F401010000003B
:201400003E0A01206400F401010000003C0A01206400F401010000003A0A012004000000DF
:20142000E8E80608390A012002000000FCE80608FB0A01200D00000008E90608F80A012021
:2014400000640100F60A0120320010270A000000F40A01200D00000008E90608F30A01204A
:201460000D00000008E90608F20A012002000000A4E70608000000000000000000000000A8
:2014800040E90608090F01204600000078E90608070F01200300000094EA0608080F012029
:2014A00004000000B0E70608FD0A012003000000A4EA0608FC0A012003000000A4EA0608F6
:2014C000FE0C0120000A0100FC0C01200000E80301000000FA0C01200000E80301000000AE
:2014E000F80C0120000A0100F60C01200000E80301000000F40C01200000E80301000000A0
:20150000C80C0120C800E80301000000CE0C01203C00FA0001000000CC0C01200100E8030B
:2015200001000000CA0C0120000501000C0D012002000000C4E706080A0D01200000F4018B
:2015400001000000080D01200000F40101000000060D01200000F40101000000040D012002
:201560000000F40101000000020D01200000E80301000000000D01200000E803010000003F
:201580001E0E0120006401000A0000001D0E0120006401000A0000000B0E0120196401001C
:2015A0000A0E012002000000D0E70608080E0120E803D0070A000000060E0120006401008E
:2015C0000A000000FB0D012000640100FA0D012000640100020E0120006401000A00000046
:2015E000010E0120006401000A000000000E0120006401000A000000050E012000FF01007A
:201600000A000000040E012000FF01000A000000030E012000FF01000A000000FF0D01201A
:2016200001FF01000A000000FE0D012001FF01000A000000FD0D012001FF01000A00000032
:20164000060B01200000F40101000000040B01200000E80301000000020B01200000E8032D
:2016600001000000000B01200000E80301000000FE0A01200000E803010000003B100120D0
:20168000009601003210012000C80100311001200064010030100120006401002F1001209A
:2016A000006401002E100120006401002D100120FF0801002C100120016401009108020835
:2016C0005508020800000000B4EA06083510012001320100341001200100000024EB0608DA
:2016E00033100120040000002CEB06082B100120009601002A100120006401002810012051
:201700001400E8030100000026100120000030750A0000002410012000C801002310012051
:2017200000C801002210012000C8010038100120003201003A10012000140100391001203E
:20174000004B0100371001200400000040EB060836100120006401000A0000002A0E012069
:201760000AC805000A000000290E01200100000050EB06082C0E01200AC805000A000000AA
:201780002B0E01200100000050EB0608210E012000C805000A000000280E012000C805005A
:2017A0000A000000220E012000C805000A000000230E012000C805000A000000260E012079
:2017C00000C805000A000000270E012000C805000A000000250E012000C805000A000000DA
:2017E000240E012000C805000A000000200E01200200000058EB06084A1001200000D007CB
:20180000010000004410012000C801004310012000C801004210012000C801004810012097
:201820000000D007010000004110012000C801004010012000C801003F10012000C8010022
:20184000461001200000D007010000003E10012000C801003D10012000C801003C1001205D
:2018600000C80100587B07080000000000008C170120647B0708070800000000D00E0020FE
:201880006C7B0708070800000000C80E0020747B0708070800000000C00E00207C7B07084C
:2018A000080800000000B40E002068650708070800000000AC0E002070650708070800007E
:2018C0000000A40E0020786507080708000000009C0E002024660708080800000000900E2A
:2018E0000020847B0708071000000000880E00208C7B0708071000000000800E0020947B03
:201900000708071000000000780E00209C7B07080810000000006C0E002084690708010026
:20192000000000000000000000000000100000000000000000000000250602080906020849
:201940009912020864EB0608EF0A0120005A0100EE0A012000C80100EC0A0120E803D00745
:20196000010000000000000000000000C50D020800EC06085C0A01200300000054EC0608B8
:201980005B0A0120000301005A0A01200003010045050208F90402080000000064EC06087B
:2019A000B9040208710402080000000000ED0608910502087D1202080000000080ED060832
:2019C000580A012001030100DD010208BD01020800000000F4F00608990B02086D0B0208AD
:2019E0000000000074F10608E10302088903020800000000E4F10608350602085D2E020833
:201A0000000000009CF2060805180208C50B02080000000044F3060885060208000000004F
:201A200000000000E0F3060869070208090702080000000044F4060811080208CD070208EA
:201A400000000000FCF40608E1740208CD0802080000000088F506082E0E0120010601005A
:201A6000CD0602089906020800000000A0F60608FD730208451402080000000010F706084A
:201A8000FD08020865150208000000008CF80608257502082515020800000000D80E002033
:201AA0002D0E012001030100D9050208A90502080000000098F906081D120208000000004D
:201AC00000000000FCF9060839040208651202080000000098FA060800000000000000009B
:201AE0000000000034FB060879090208B116020800000000B4FB060800000000000000008F
:201B000000000000DCFD060870DC00209CFF2C0100000000C4120120E0150C17000000009B
:201B2000C61201200200000014010708340A012088136F1701000000360A012088136F1783
:201B4000000000004C74002000000000000000004A740020000000000000000048740020EB
:201B60000000000000000000467400200000000000000000447400200000000000000000B3
:201B80004274002000000000000000008C0600200000000000000000BD09012003000000D3
:201BA000F8FE06082C0A012088136F17010000008EDE002088136F1700000000C902020826
:201BC000000000000000000008FF0608A50F0120010000005CFF060890DE00200100000022
:201BE00068FF060886DE00200200000070FF06080000000000000000000000007CFF0608E4
:201C0000B10202080000000000000000180007080000000000000000000000006C00070865
:201C2000000000000000000000000000DC000708380A012002000000140107088ADE0020A8
:201C4000E0150C1700000000D81D01202C1E012001F11F3FD601FF0048A70020FFFFFFFFBA
:201C60000000803F00000000000000000000000000000000000000000000000000000000A5
:201C800000000000000000000000803F0000000000000000000000000000803F00000000C6
:201CA00000000000000000000000803F000000000000000000000000010000000000FA4327
:201CC0000000FA430000803FFFFFFFFFFF000000B5AE04080000000000000000000000009E
:201CE00000000000B43E01200800000000000000A43E012008000000354D04080000000030
:201D000000000000000000006DDE040800000000000000000000000001000000A00F0000BC
:201D2000B80B000002FFFF01685E0C0002000000D93D0108DD130108713D0108000000003C
:201D4000AD12010859460108C13C01080D39010800000000000000006D1201081985000890
:201D60000D850008618F00087D8F0008458F0008298F00080D8F0008913D0108B9130108D1
:201D8000C53C0108000000008512010811390108953C01086D3801080000000000000000BE
:201DA00079120108949C0708C4660708000000002DE40308A086010004000000949C070891
:201DC0009C9C0708000000004D890408E8030000040000003070070800000000000000003C
:201DE000F93A03087D000000FF000000346E07080000000000000000A9BF03087D00000088
:201E0000FF000000607307080000000000000000055C03087D000000FF000000C8700708B2
:201E20000000000000000000E9AE0408E803000003000000A49C07080000000000000000C2
:201E4000B13E0308102700000300000008E107080000000031940208B5B804085F76000039
:201E600005000000BCE407080000000000000000E9DB04081027000002000000B09C07084A
:201E80000000000000000000C14C0408E803000005000000BC9C07080000000000000000D2
:201EA00005EC0308204E000003000000CC9C07080000000000000000EDE90308204E0000EF
:201EC00003000000DC9C0708000000000000000089B40408400D030003000000908D0708B0
:201EE000000000000000000031AC04081027000002000000F066070800000000000000005B
:201F0000E9E601081027000003000000EC9C070800000000000000002D840408A086010034
:201F200002000000DC6E070800000000000000002987040850C3000002000000846C070876
:201F40000000000000000000757F0408A861000002000000AC8D070800000000000000002E
:201F6000854D0408A00F000002000000F49C0708000000000000000021D001081027000002
:201F8000020000007C7D070800000000A17C010875C301088545010002000000446C070844
:201FA00000000000000000001D1A01081027000002000000D866070800000000000000005B
:201FC0005137020850C3000002000000009D0708000000000000000019260108400D030016
:201FE00001000000089D070800000000000000007D4C0408400D030002000000109D070849
:020000040800F2
:202000000000000000000000CDF6010850C30000030000001C9D0708000000000000000016
:20202000C505040840420F0001000000289D070800000000000000005D4D040850C300009B
:2020400001000000349D07080000000000000000756901081027000002000000FFFF000081
:20206000FFFFFFFFE4E00708000008020503030000000000F0E00708010008020504030086
:2020800000000000FCE0070800000802050303000000000004E10708010008020504030035
:2020A00000000000E08C07080200FE010110030000000000786D0708030014020003000080
:2020C000000000000CE1070804001F02020008000000000014E1070805001F0202010800A0
:2020E000000000001A030000000000000000000000000000000000000000000000000000C3
:202100000403090412010002000000408304205700020102030101005D6A0508316A0508D2
:20212000D5690508E55A0508F169050895690508E15A050840190020516B0508716105082D
:20214000416B0508C55A0508FD6A0508B56A0508B55A05081C19002069640508CD5A05087B
:20216000C95A0508C15A0508B9640508BD5A0508B95A050858550708F545010899130108E5
:20218000D544010800000000000000006D3C01087D3B0108000000000000000000000000AA
:2021A000611201086D5B0508615B0508A96B0508C56B0508195B05088D6B0508716B050838
:2021C000020000000000000018190020D45401200200000001000000D55C050814190020D5
:2021E000000000000100000001000000115D050834180020000000000000000000000000F6
:202200000000000000000000000000000000000001000000000000000000000000000000BD
:2022200000000000010000000000000000000000000000000000000001000000000000009C
:20224000D8000000000000000500000006000000FFFFFFFF03000000000000000500000097
:20226000050000001F0000001C0000001F0000001E0000001F0000001E0000001F00000085
:202280001F0000001E0000001F0000001E0000001F0000000068214C010000007C550708EF
:2022A0000600000005000000008002021F00000053544D202020202050726F64757420201E
:2022C0002020202020202020302E3031008002021F00000053544D202020202050726F6473
:2022E000757420202020202020202020302E30310B0101010100000050C300000101FF01D2
:2023000025000000AC59070800000000000000000000000001000000000000000000000083
:2023200000000000000000000100000000000000F40100002AFF0000A400000000000000DA
:2023400000000000000004010000020001000002100000000700000000000000000000005C
:202360000102030406070809C70000000500000006FF0000EC19002000000000000000003F
:2023800000000000000000000000000000000000000000000000000000000000000000003D
:2023A00000000000000000000000000000000000000000000000000000000000000000001D
:2023C000000000000000000000000000000000000000000000000000FFFFFFFFFFFFFFFF05
:2023E000FFFFFFFFFFFFFFFFFFFFFFFFFFFFFFFFFFFFFFFFFFFFFFFFFFFFFFFFFFFFFFFFFD
:20240000FFFFFFFFFFFFFFFFFFFFFFFFFFFFFFFFFFFFFFFFFFFFFFFFFFFFFFFFFFFFFFFFDC
:20242000FFFFFFFFFFFFFFFFFFFFFFFFFFFFFFFFFFFFFFFFFFFFFFFFFFFFFFFFFFFFFFFFBC
:20244000FFFFFFFFFFFFFFFFFFFFFFFFFFFFFFFFFFFFFFFFFFFFFFFFFFFFFFFFFFFFFFFF9C
:202800000828000800400008232042657461666C69676874202F2053544D33324634313157
:202820002028533431312920342E312E31204E6F762031352032303139202F2031323A3526
:20284000353A3137202831653565336433363929204D5350204150493A20312E34320A2371
:2028600020636F6E6669673A206D616E7566616374757265725F69643A20424546482C2074
:20288000626F6172645F6E616D653A2042455441465056463431312C2076657273696F6EA0
:2028A0003A2065646364323434622C20646174653A20323032322D30362D32395430323A0D
:2028C00032343A34365A0A0A626F6172645F6E616D652042455441465056463431310A6DFD
:2028E000616E7566616374757265725F696420424546480A0A23207265736F7572636573A5
:202900000A7265736F75726365204245455045522031204230320A7265736F7572636520CB
:202920004D4F544F522031204230340A7265736F75726365204D4F544F52203220423035B3
:202940000A7265736F75726365204D4F544F522033204230360A7265736F75726365204D5A
:202960004F544F522034204230370A7265736F757263652050504D2031204130330A726581
:20298000736F75726365204C45445F53545249502031204130380A7265736F757263652014
:2029A00053455249414C5F54582031204130390A7265736F757263652053455249414C5F80
:2029C00054582032204130320A7265736F757263652053455249414C5F54582031312042F5
:2029E00030330A7265736F757263652053455249414C5F5458203132204231300A7265737D
:202A00006F757263652053455249414C5F52582031204131300A7265736F757263652053B7
:202A2000455249414C5F52582032204130330A7265736F757263652053455249414C5F5207
:202A400058203131204230330A7265736F757263652053455249414C5F5258203132204297
:202A600031300A7265736F75726365204932435F53434C2031204230380A7265736F75729F
:202A80006365204932435F5344412031204230390A7265736F75726365204C454420312065
:202AA0004331330A7265736F75726365204C45442032204331340A7265736F75726365205C
:202AC0005350495F53434B2031204130350A7265736F75726365205350495F53434B2032A3
:202AE000204231330A7265736F75726365205350495F4D49534F2031204130360A7265738F
:202B00006F75726365205350495F4D49534F2032204231340A7265736F75726365205350A6
:202B2000495F4D4F53492031204130370A7265736F75726365205350495F4D4F5349203235
:202B4000204231350A7265736F75726365204144435F424154542031204230300A72657362
:202B60006F75726365204144435F435552522031204230310A7265736F7572636520464C7C
:202B80004153485F43532031204130300A7265736F75726365204F53445F43532031204232
:202BA00031320A7265736F75726365204759524F5F455854492031204130310A7265736F70
:202BC00075726365204759524F5F43532031204130340A7265736F75726365205553425FFF
:202BE0004445544543542031204331350A0A232074696D65720A74696D657220413033207B
:202C00004146330A232070696E204130333A2054494D39204348322028414633290A746936
:202C20006D657220423034204146320A232070696E204230343A2054494D332043483120E4
:202C400028414632290A74696D657220423035204146320A232070696E204230353A205496
:202C6000494D33204348322028414632290A74696D657220423036204146320A2320706992
:202C80006E204230363A2054494D34204348312028414632290A74696D657220423037206C
:202CA0004146320A232070696E204230373A2054494D34204348322028414632290A746998
:202CC0006D657220423033204146310A232070696E204230333A2054494D32204348322047
:202CE00028414631290A74696D657220423130204146310A232070696E204231303A205400
:202D0000494D32204348332028414631290A74696D657220413030204146320A23207069F9
:202D20006E204130303A2054494D35204348312028414632290A74696D65722041303220D7
:202D40004146320A232070696E204130323A2054494D35204348332028414632290A7469FB
:202D60006D657220413038204146310A232070696E204130383A2054494D312043483120A0
:202D800028414631290A0A2320646D610A646D6120414443203120310A2320414443203175
:202DA0003A20444D41322053747265616D2034204368616E6E656C20300A646D6120706977
:202DC0006E2042303420300A232070696E204230343A20444D41312053747265616D2034D8
:202DE000204368616E6E656C20350A646D612070696E2042303520300A232070696E2042F5
:202E000030353A20444D41312053747265616D2035204368616E6E656C20350A646D612085
:202E200070696E2042303620300A232070696E204230363A20444D41312053747265616DEE
:202E40002030204368616E6E656C20320A646D612070696E2042303720300A232070696EA7
:202E6000204230373A20444D41312053747265616D2033204368616E6E656C20320A646D47
:202E8000612070696E2042303320300A232070696E204230333A20444D41312053747265E1
:202EA000616D2036204368616E6E656C20330A646D612070696E2042313020300A2320704F
:202EC000696E204231303A20444D41312053747265616D2031204368616E6E656C20330AE8
:202EE000646D612070696E2041303020300A232070696E204130303A20444D41312053748F
:202F00007265616D2032204368616E6E656C20360A646D612070696E2041303220300A23A8
:202F20002070696E204130323A20444D41312053747265616D2030204368616E6E656C2035
:202F4000360A646D612070696E2041303820300A232070696E204130383A20444D413220A4
:202F600053747265616D2036204368616E6E656C20300A0A2320666561747572650A66654E
:202F800061747572652052585F53455249414C0A6665617475726520534F465453455249A2
:202FA000414C0A666561747572652054454C454D455452590A66656174757265204F5344B7
:202FC0000A66656174757265204149524D4F44450A6665617475726520414E54495F4752A0
:202FE00041564954590A0A232073657269616C0A73657269616C2030203634203131353220
:2030000030302035373630302030203131353230300A0A23206D61737465720A736574203C
:203020006261726F5F62757374797065203D204932430A736574206261726F5F6932635F70
:20304000646576696365203D20310A736574206261726F5F6861726477617265203D204EC0
:203060004F4E450A7365742073657269616C72785F70726F7669646572203D20534255530A
:203080000A73657420626C61636B626F785F646576696365203D20535049464C4153480AC4
:2030A000736574206473686F745F69646C655F76616C7565203D203435300A736574206419
:2030C00073686F745F6275727374203D204155544F0A736574206473686F745F6269746255
:2030E000616E67203D204F46460A736574206D6F746F725F70776D5F70726F746F636F6C17
:20310000203D204453484F543630300A7365742063757272656E745F6D65746572203D20A8
:203120004144430A73657420626174746572795F6D65746572203D204144430A736574201F
:203140006D61675F6861726477617265203D204E4F4E450A736574206265657065725F692F
:203160006E76657273696F6E203D204F4E0A736574206265657065725F6F64203D204F4694
:20318000460A7365742073797374656D5F6873655F6D687A203D20380A736574206D617810
:2031A000373435365F7370695F627573203D20320A73657420666C6173685F7370695F6246
:2031C0007573203D20320A736574206779726F5F315F62757374797065203D205350490AB3
:2031E000736574206779726F5F315F737069627573203D20310A736574206779726F5F31A8
:203200005F73656E736F725F616C69676E203D2043573138300A736574206779726F5F31D4
:203220005F616C69676E5F796177203D20313830300A00FFFFFFFFFFFFFFFFFFFFFFFFFF31
:20324000FFFFFFFFFFFFFFFFFFFFFFFFFFFFFFFFFFFFFFFFFFFFFFFFFFFFFFFFFFFFFFFF8E
:20326000FFFFFFFFFFFFFFFFFFFFFFFFFFFFFFFFFFFFFFFFFFFFFFFFFFFFFFFFFFFFFFFF6E
:20328000FFFFFFFFFFFFFFFFFFFFFFFFFFFFFFFFFFFFFFFFFFFFFFFFFFFFFFFFFFFFFFFF4E
:2032A000FFFFFFFFFFFFFFFFFFFFFFFFFFFFFFFFFFFFFFFFFFFFFFFFFFFFFFFFFFFFFFFF2E
:020000040800F2
:20400000AEBE08000E02000000000B0014020000000000FF000A00130200000000013F108D
:2040200000030101000000000000000000000052000D0001000100000014050405000000F8
:204040000040000000000504050000000000000000010504050000000000000000050504F5
:204060000500000000000000001E05040500000000000000001F050405000000006400522C
:2040800000070009020000002A00FD01000019120000000000000000232A1A130000000041
:2040A00000000000232A0000000000000000000000000700FB010000130F00FC0100000091
:2040C00000000000000000000C00F70100002201000000000A00F90100003D3E00004500F5
:2040E000160200001303FF2401002501002601002701002301002A0100100200120200186C
:2041000001000000000000000000000000000000000000000000000000000000000000009E
:20412000000000160034000000DC0532000000000000000000000001040E001102000000FC
:20414000000000010101010A0012020100FFFFFFFF3E0018000300000103020405060702C9
:20416000000000000001006400DC051A046C070019750343080E000001000000001E1E1E23
:204180000101000000000000000000000000001100000200000000000000FF00000000000B
:2041A0000B00FF0102000000000000150008020100151617FFFF2D2E2FFFFF000000FFFF0C
:2041C0000900FA0100001002000E002A020000960058022C0103000E0020020500036432A1
:2041E00000F40196002A0006000100E0010700000200242526270000000000000000010280
:204200000304050607C2012E04D007E8030E000A000C020000012C02001A00FE010000015F
:2042200020000001210000010000000000000001FFFF0014002600010001000001000115E9
:20424000005802D903000020000B000300AE014A015E012C0164010100000001000A019A68
:2042600001001E0A0000022A001F00050000000000000100010005000001020300000000B8
:2042800000000000000000000000000000008017000A000502000000000000110001020062
:2042A00000000000000200000000000009000202000000000016001B02000006000000E8CE
:2042C000030000000000000000000012001B000200001800020301F40132000164F60021EB
:2042E0000200000000000000000000000000000000000000000000000000000000000000BC
:2043000000000000000000000000000000000000000000000000000000000000000000009D
:2043200000000000000000000000000000000000000000000000000000000000000000007D
:2043400000000000000000000000000000000000000000000000000000000000000000005D
:20436000000000000000000000FFFF000000FF1E0000FF3C0000FF5A0000FF780000FF9682
:204380000000FFB40000FFD20000FFF00000FF0E0100FF2C0100FF4A0100FF000000000027
:2043A000000000010B020D0A03050B030D0A030A0B040D0A03080B040D0A03070B030D0A18
:2043C00003000000000000060A0100000203060000000336003700010020003200C800D063
:2043E0000796001400320028004C0440060005500014000F00080064000100010005000A27
:20440000000000F40196000F000C0016000100C4090000190028002F0001000000000000A1
:20442000000000000000000000000000000000000000000000000000000000000016002343
:20444000020200000000000000000000000000FF0000000F001E0000000005010000000026
:204460000000120005000200020100000000000000000000160012000300000000010001F3
:20448000055334313100000802008200FD070000EA00EA00CD004E00CE00EA00EA00EA0023
:2044A000EA00EA00EA00EA00EA00EA00EA00EA00EA00EA00EA00EA00EA004939EA00EA00C4
:2044C000EA00EA00EA00EA00EA00EA00EA00EA00EA00EA00EA00EA00EA00EA00EA00EA003C
:2044E000EA00EA00EA00EA00EA00EA00EA00EA00EA00EA00EA00EA00EA00EA00EA00EA001C
:20450000EA002300EA00EA00CD00EA007200F5010900980864001401000A010A0000FF1F46
:204520000000142800002C3700008000FFFFFFFF4600010200000000000000000000000017
:2045400000000000000000000000000000000000000000000000000000000000000000005B
:2045600000000000000000005000C4FF00FFFFFFFF0100000005180B0C00000000001600E1
:20458000230002000A0000000000000000000000000000001200F6010200000000000100E0
:2045A00000000202000022001C02000000020114000011030000000008070102000000007A
:2045C00000010000000000001C002800030000010200000000000000000000000000000090
:2045E000000000000B00140000000300002300120001000200E80364000F0A00010A001ED0
:2046000000EA000C000400320003070707000000434343410046050064CE07CE07CE07011D
:2046200000000000000000000000000000320003070707000000434343410046050064CEA9
:2046400007CE07CE0701000000000000000000000000003200030707070000004343434154
:204660000046050064CE07CE07CE07010000000000000000000000000032000307070700C1
:204680000000434343410046050064CE07CE07CE07010000000000000000000000000032AF
:2046A0000003070707000000434343410046050064CE07CE07CE07010000000000000000A9
:2046C0000000000000320003070707000000434343410046050064CE07CE07CE0701000057
:2046E00000000000000000000000002A000A00090030000000FA00F401000000000000005E
:20470000000000020000029E077D00FA00F401000105016400C2010E00030064004B000096
:204720000000002D50280078002F542E007D002D500000780032324B000000280000000062
:20474000000055F401900101374B000000FA00AC0D00000000320090015E01F40100000A27
:2047600064C8009001960000050F00010F0114004B3200005A140B00004B009600001400C2
:20478000280100C8001E220025146400000000000000000000000032323296000019070FF0
:2047A0005A050000026464646464646401646464004B00000000002D50280078002F542E96
:2047C000007D002D500000780032324B0000002800000000000055F401900101374B000032
:2047E00000FA00AC0D00000000320090015E01F40100000A64C8009001960000050F00017D
:204800000F0114004B3200005A140B00004B009600001400280100C8001E220025146400BB
:20482000000000000000000000000032323296000019070F5A050000026464646464646400
:2048400001646464004B00000000002D50280078002F542E007D002D500000780032324BF1
:204860000000002800000000000055F401900101374B000000FA00AC0D000000003200903D
:20488000015E01F40100000A64C8009001960000050F00010F0114004B3200005A140B0037
:2048A000004B009600001400280100C8001E22002514640000000000000000000000003203
:2048C000323296000019070F5A05000002646464646464640164640A00130001004804441B
:2048E000100A0001010000000000000A0000010000900100000900020100006E0A01220158
:20490000220200000000000000000000000000000000000000000000000000000000000073
:20492000000000000000000000000000000000000000000000000000000000000000000077
:20494000000000000000000000000000000000000000000000000000000000000000000057
:20496000000000000000000000000000000000000000000000000000000000000000000037
:2049800000000000000042414E44312020200042414E44322020200042414E443320202022
:2049A0000042414E44342020200042414E44352020200042414E44362020200042414E44E4
:2049C000372020200042414E443820202000313233343536373831003200330034003500F0
:2049E000360037003800000000000000000000000000000000000000000000000000000012
:204A00004C5630004C5631004C5632004C5633004C5634004C5635004C5636004C563700EA
:204A20007600150000000000000000000000000000000000000000000000000000000000EB
:204A4000000000000000000000000000000000000000000000000000000000000000000056
:204A6000000000000000000000000000000000000000000000000000000000000000000036
:204A8000000000000000000000000000000000000000000000000700030000000066002A7C
:204AA00000000000000000E803D007DC0564FF00000000E803D007DC0564FF00000000E802
:204AC00003D007DC0564FF00000000E803D007DC0564FF00000000E803D007DC0564FF00AC
:204AE000000000E803D007DC0564FF00000000E803D007DC0564FF00000000E803D007DC0C
:204B00000564FF16002C000000E803D007E803D007E803D007E803D0077E0029000200003A
:204B2000000000000000000000000000000000000000000000000000000000000000000075
:204B4000000000000000000000000000000000000000000000000000000000000000000055
:204B6000000000000000000000000000000000000000000000000000000000000000000035
:204B8000000000000000000000000000000000000000000000000014001A0000007E05EA7A
:204BA00005B4053200E803D00700002A002B000000001E001E001E0005011E011E011E0131
:204BC0001E011E011E011E011E011E011E011E011E011E011E160019020000000000000050
:204BE00000000000000000000000003201250002000000000000000000000000000000005B
:204C0000000000000000000000000000000000000000000000000000000000000000000094
:204C2000000000000000000000000000000000000000000000000000000000000000000074
:204C4000000000000000000000000000000000000000000000000000000000000000000054
:204C6000000000000000000000000000000000000000000000000000000000000000000034
:204C8000000000000000000000000000000000000000000000000000000000000000000014
:204CA0000000000000000000000000000000000000000000000000000000000000000000F4
:204CC0000000000000000000000000000000000000000000000000000000000000000000D4
:204CE0000000000000000000000000000000000000000000000000000000000000000000B4
:204D000000000000000000000000000000000000000000000000000000000000004300034D
:204D2000020100000000000000000000000000000000000000000000000000000000000070
:204D4000000000000000000000000000000000000000000000000000000000000000000152
:204D60000C00F80103000201F401140008001000010000050B0019000000000028010012A2
:204D80000002000000000000000000000000000000460029020000000000000000000000A0
:204DA0000000000000000000000000000000000000000000000000000000000000000000F3
:204DC00000000000000000000000000000000000000000000000000A002C02000001000199
:204DE000001A000A02000000004A01B400D6010000C2010E0196004400000042001A0200AD
:204E0000000000000000000000000000000000000000000000000000000000000000000092
:204E2000004245464800424554414650564634313100000000000000000000010009003837
:204E4000000200000A078600040000000000000000000000000000000000000000000000B5
:204E6000000000000000000000000000000000000000000000000000000000000000000032
:204E8000000000000000000000000000000000000000000000000000000000000000000012
:204EA0000000000000000000000000000000000000000000000000000000000000000000F2
:204EC0000000000000000000000000000A0028020000000000000A0027020000000000006B
:204EE00016001F020000FFFFFFFFFFFFFFFFFFFFFFFFFFFFFFFF0C001D0200000000000060
:204F000000001800060201002829000020030000000020030000000020030A002700000085
:204F20002003000043000B02020000000000000000000000000000000000000000000000FC
:204F4000000000000000000000000000000000000000000000000000000000000000000051
:204F6000000000010000001A000D0201000000000000000000000000000000000000000006
:204F8000000C001E020000000000000000070010020000000000F437FFFFFFFFFFFFFFFFA9
:204FA000FFFFFFFFFFFFFFFFFFFFFFFFFFFFFFFFFFFFFFFFFFFFFFFFFFFFFFFFFFFFFFFF11
:204FC000FFFFFFFFFFFFFFFFFFFFFFFFFFFFFFFFFFFFFFFFFFFFFFFFFFFFFFFFFFFFFFFFF1
:204FE000FFFFFFFFFFFFFFFFFFFFFFFFFFFFFFFFFFFFFFFFFFFFFFFFFFFFFFFFFFFFFFFFD1
:20500000FFFFFFFFFFFFFFFFFFFFFFFFFFFFFFFFFFFFFFFFFFFFFFFFFFFFFFFFFFFFFFFFB0
:020000040800F2
:020000040800F2
:20800000134B0268196821EA02011960596821EA0201596019680A431A609968026821EA4A
:2080200002019960D96821EA0201D9604179102907D001F1804303F59E3319680A431A602C
:208040007047996811439960D9680A43DA607047003C0140024B9A6D136A002BFCD170479F
:20806000501A0020F0B401292D4C2E4D4FF0000694BF00230123EE62C4F81861C4F81C6117
:20808000C4F82831D4F82871D4F8F43047EA4207C4F82871EE63EC6B002A38D144F495748B
:2080A000EC631C6824F001041C601C68E407FCD4490289085960D8601968EAB921F04001D6
:2080C000196019498B421DD018494FF47410C860196841F01E011960596941F08001596143
:2080E000196841F00101196022B90E4AD36A43F00803D362F0BC704741F0400119600A49CF
:208100008B42E1D14FF0746041F8500CE0E744F01A04EC63EC6A44F00804EC62C1E700BF85
:20812000501A0020002C014058640240006402401248002302461178032902F1060218D047
:208140000133062BF7D10E4AD2F85031052B0FD0591C03EB4303C2F8501100EB4303032028
:2081600040F2EB3140F2FF32187059809A807047704703EB430300EB4303F0E77C1B002072
:20818000501A002030B5134A134B8DB0082102F1580082F8F0100693694400230DF1070517
:2081A0000124CDE9073302938DF8143009938DF828300B93CDE9035449F07CFDFFF74AFF37
:2081C0009DF80700A0F1FF00B0FA80F040090DB030BD00BF501A0020DD810008826D136A4B
:2081E0005B681B78FF2B08D090F8F030013BDBB280F8F0301BB10120704700207047126A27
:20820000526802201370704770B4C3080D4CE25C00F00706B24004EBD004D2B20020C6F1B5
:2082200008038B4228BF0B46C3F108052A419840C91A40EA02004FF0000614F8012FEED1DB
:2082400070BC7047901A0020084AD2E9553199420AD0D118013391F85C110170C3F30A03E2
:20826000C2F854310120704700207047501A0020064BD3F86009D3F85C29D3F85C3982428D
:2082800098BF03F50063181A704700BF501A0020012380F85130704707B501A8FFF7D4FFF8
:2082A0000028FAD09DF8040003B05DF804FB044BD3E95503984288BF03F50063181A704764
:2082C000501A002001207047024BC3F86429C3F868197047501A0020024BC3F86C29C3F8D2
:2082E00070197047501A00207047704730B4134DD5E955239A4286BF03F50064A21A9A1ADF
:208300000A44B2F5006F13D8A9B101444A1E013810F8014FE918824203F1010381F85C41A3
:20832000C3F30A03F4D1C5F85831002030BC7047022030BC70470846F8E700BF501A002071
:2083400041B370B5144C0144D4F860394E1E451E1A4604E0012048F02DF9D4F86029D4F847
:208360005C19531CC3F30A038B42F3D0D4F85C19B1F5006FEED094F874190029EAD115F8A8
:20838000011FC4F860392244B54282F87819DFD1002070BD00207047501A002010B5094C88
:2083A000D4F88030084611465BB1D4F88030052B07D1002AD4F8843003DDFFF7C1FFD4F800
:2083C000843010BD482B002010B590F85010002380F8503081B10B4CD4F8802072B1D4F8DD
:2083E0008020052A0CD13C30D4F88430FFF7A8FFD4F88430012010BD0120FCE71046FAE79F
:208400001846F8E7482B0020002280F85120DBE790F85020531C0244DBB280F8503082F813
:208420003C1090F851200AB1132B00D9CCE77047212838B50C4605D022282FD0202813D0EA
:20844000002038BD0029FBD0072AF9D11A4BD3F8880093F88C1093F88D2093F88E30206038
:2084600021716271A371EBE70029E9D0072AE7D1124AD2F868391BB1D2F8640909689847CC
:208480000D4B256820796179A279C3F8885083F88C0083F88D1083F88E20D1E70029CFD00E
:2084A000022ACDD1054AD2F87039002BC8D00988D2F86C099847C3E7482B0020501A0020F7
:2084C000024B0020C3F88000704700BF482B0020054B064A00200521C2F88010C3F8700987
:2084E000C3F86809704700BF501A0020482B0020704700BF704700BF704700BF704700BFE5
:20850000704700BF704700BF704700BF042301480B8070479801002010B4074A074B92F89D
:208520009000122403F114020C8001280CBF184610465DF8044B7047482B00209C0100208C
:2085400000487047781A002000487047781A0020034B93F82400032894BF00200120704746
:20856000501A0020034B93F82400032894BF002001207047501A0020034B93F8240000383F
:2085800018BF0120704700BF501A0020034B93F82400003818BF0120704700BF501A0020B6
:2085A000A0B182680D4B12B107229A7070471978DA6003294FF004000CBF80214FF48071A1
:2085C000C3E901111A611A7598707047034B41F2E47101225A545A70704700BFF8BD002058
:2085E0000378022B10D0006908B9012070470C4B1B78032B0EBF0B4B80B24FF6F7739842FB
:2086000094BF0020012070470549436841F650028A58B3EB422F2CBF01200020704700BFFA
:20862000F8BD0020F7FFFF0F0378022B14D030B4104A4368006941F6480402F5C251155988
:20864000096841F63C042B4012595B0A023801FB0030104430BC7047064B426841F6340133
:2086600041F630005958185800EB410000EB5220704700BFF8BD002030B593B040F0400204
:208680000B0E0D0C04468DF80810080A8DF80420952101AA8DF805308DF8065000230625C2
:2086A0008DF807008DF809100DF1030001210392134A0493CDE90733CDE90D33CDE909013E
:2086C0008DF818308DF82C300F938DF84030119305950C92FFF756FD00B974B9094B0822CC
:2086E00003F1580003A983F8F02049F0E3FAFFF7B1FC9DF8030013B030BDFF2013B030BD27
:2087000009870008501A0020836D1B6A5B681B78FF2B0AD190F8F030002B03F1FF3380F8F6
:20872000F03014BF0120022070470020704700BF30B5104A104B8DB0014682F8F01002F12B
:208740005800069302A900230DF107050124CDE9073302938DF8143009938DF828300B93C6
:20876000CDE9035449F0A6FAFFF774FC9DF807000DB030BD501A00200987000870B51C4DB7
:2087800090B00024FD220DF1030305F15800012601A98DF803200693CDE90144CDE90A44F3
:2087A000CDE90C442C628DF81040059407948DF824408DF838400F940396089649F07AFAAF
:2087C000FFF748FC3046FFF7B3FFFF2809D0094BD3F884306B612046092385F8243010B07F
:2087E00070BD0423022085F8243010B070BD00BF501A0020482B002070B5064690B0082090
:208800000D46FFF795FFFF2821D0FE2802D0022010B070BD002402230E48089301A9CDE9C2
:208820000265CDE90544CDE90A44CDE90C4401948DF8104007948DF824408DF838400F943A
:2088400049F038FAFFF706FC204610B070BD012010B070BDA81A002008B5FFF7FBFB0A209F
:2088600047F08AFD024B186EBDE8084048F088BE501A002070B50379254C002B14BF01223F
:2088800000228AB084F8502003D184F824300AB070BD054690F9001004F1580049F080FB20
:2088A000AD784DBB01261B482566C4F8EC4084F8646049F0ABFB03464FF47A70A4F85C30D1
:2088C00047F078FE206E48F05BFE28226846002165F0FDF80A2310480293694649F0EAF984
:2088E000FFF7B8FB0D4B84F82460D3F884306361002323760AB070BD284648F057FB05464E
:2089000008B11E23C3800921284647F005F9C9E7501A0020801A0600A81A0020482B0020FE
:208920002DE9F84F494B98420ED003F56853083398424ED0464B0020C3E94000A3F8FC0074
:20894000A3F80801BDE8F88F414C424FDFF810810223C4F8943004F198060025FB6AAB4212
:20896000294605F1010503D0D4F8180153F08EFD94F81C31D4F8182186F82430326230464C
:20898000414653F097FFD4F894309D4206F13006E4DB002384F80A31D4E92803D4F89410EA
:2089A000B4F89C20B4F8A850C4F8283112FB01F203FB01F3A4F8FC20B4F89E10264AA4F886
:2089C0000851C4E94003A4F8FE10C4F8F8200120B8E71F4C1F4F0223C4F8943004F1980500
:2089E0004FF0000B4FF4806A4FF040094FF40068FA6A01265A455946B34403D0D4F8180155
:208A000053F044FDD4F8181194F81C21296285F824204FF400314FF00062C5E90212A5F854
:208A200004A0A5F81090A5F80680AE74FFF780FB28466E7653F08AFED4F89420074B45F873
:208A4000303B9345D4DB84F80A61A5E71971EF00482B0020980100209CDB060870DB06080E
:208A60001940EF002DE9F843194C94F82460042E0546894690461F4608D0082E02D0002061
:208A8000BDE8F883FFF77AFE0228F8D1206E48F071FDA37E9BB969021120FFF7EDFDA0B9D7
:208AA0000C4BC4F80090D3F8842065600523C4E90387626184F824300120BDE8F88329463D
:208AC0001120FFF7D9FD0028EAD0FFF7C5FED6E7501A0020482B00202DE9F04FCF4ED04D95
:208AE00086468C4617460FCE05F596742DED068B0FC40FCE0FC496E8070089B095F862318E
:208B0000039784E80700CDE904EC042B00F24881DFE813F0B401460141010500C4019FED5A
:208B2000C18ADFEDC18AC149C5F84811C049C14BC14AC5F844110399002918BF134638EE66
:208B4000887AF5EE006AC6EE879ABC4EC5F85031A6F1120B06F1C0080027DFEDB97A9FED84
:208B6000B99A28EE278AB0EE67AA059BBB4200F00C811BF8013BEA1892F86741002C00F073
:208B80001481002202E0152A00F00F8102EB42014FEA420918F80100A04202F10102F2D11D
:208BA000294491F84512002900F066812046029344F03CFF029B82465046029344F056FFE5
:208BC0000178002940F0F180029BA9440133DBB2032289F8853289F88422BAF1000F00F0D9
:208BE000E4804FEA141909F1FF39B9F1040F04F00F0000F20881944C04EB4901B1F884C038
:208C00004CFA00F111F0010100F0FD80012101FA00F0013800EA0C00A144029362F05EFC4B
:208C200099F890C0DFF838E2029B60440EEBC00C03228CF807308CF806205EF83000C6F88E
:208C400014C000F13F4303F57E0304EB9324012194F898309AF8082003F01F045B09032BD6
:208C600001FA04F100F00381042B00F0FB80022B00F0CF80BCF804300693B3FA83F3C3F132
:208C80001F03C3F3CC0100EB810103F007030C6A9B004FF00F0C0CFA03FC24EA0C040C62C9
:208CA0000C6A02FA03F323430B62022306A907930BF0E2FF039B002B00F08380B5F8603135
:208CC000D5F8301507EE903AF8EEE77AFCEEE77A17EE900AB1FBF0F202F57F42FF32120CFD
:208CE000B1FBF2F295F86211B2FBF0F0042983B27ED007EE902AF8EE676A66EE887A29EED4
:208D0000677A95F8630104990091A8EEA67A019051463046C6ED027A86ED037A36F0FEFFBD
:208D2000002F72DD7368D5F8882193426FD0012F6BD0D5F8A021934269D0022F65D0D5F816
:208D4000B821934263D0032F5FD0D5F8D02193425DD0042F59D0D5F8E821934257D0052FAF
:208D600053D0D5F80022934251D0062F4DD0D5F81822D31A18BF012301370122082F337471
:208D8000727406F118067FF4F0AE304809B0BDEC068BBDE8F08F9FED2E8AF0EE488AC2E69C
:208DA0009FED2C8AF0EE488ABDE62B4A224BC5F848210020C5F8503109B0BDEC068BBDE820
:208DC000F08FB0EE690A63F0EFFAFCEEC07A4FF6FF7317EE902AD5F83015B1FBF2F21A442D
:208DE000120CB1FBF2F295F862110429184680D107EE900A07EE102AF8EE677AF8EE476ACD
:208E000067EE8A7A7BE7716154E70123B4E70023B2E7124B5C6C214359642BE7C8DB060806
:208E2000482B0020ACC5A737ACC5A736C1E9030881E00408B5E0030875E00408CC2C0020C7
:208E40006F12833A00007A4470DB0608742C0020282930386F12033905E20308003802401B
:208E6000F82D00200F4B1C6B2143196302E70D4B1C6C21431964FDE68A469DE69FED0A8AEC
:208E80000A4A0B4BC5F84821C5F8443100220123CDE90332F0EE488A064B50E69FED068A4C
:208EA000EEE700BF003802406F12833AC1E9030881E0040875E0040800000000F8B5104ED8
:208EC000D6F83045054600680F4664080BF0D8FDB4FBF7F1B1F5803F03D3012CFAD96408CD
:208EE000F6E72246284689B244F03EFC054BC6F8983D28460449BDE8F840002244F042BB48
:208F0000482B0020B1270208E038002010B5044C04480A4621460AF02DFC204610BD00BF77
:208F2000E8380020D05D070810B5044C04480A4621460AF01FFC204610BD00BFE838002056
:208F4000E05D070810B5044C04480A4621460AF011FC204610BD00BFE8380020EC5D07081C
:208F600010B5044C04480A4621460AF003FC204610BD00BFE8380020F85D070810B5044C35
:208F800004480A4621460AF0F5FB204610BD00BFE8380020045E070810B50C4C94F8F22086
:208FA0000023236212B10A4AC2F8A03E5BF052FF20B10423022084F8243010BD044BD3F8ED
:208FC00084306361092384F8243010BD501A0020482B002070B50D4D95F82430042B04465A
:208FE0000E460AD0082B06D1EB6983420CD0FFF7D3FF022801D0012070BD0823C5E907460D
:2090000085F82430022070BD022070BD501A002010B50AF083FB0F4C48B194F82430032BB8
:2090200011D8237E0133DBB2072B237603D9002384F8243010BD084A0123D2F884206261D7
:2090400084F8243010BD054848F0E0FFA4F85C00E7E700BF501A0020482B0020801A0600CD
:2090600070B51D4C94F82430042B06460D4608D0082B20D1E36983422BD0FFF77FFB022812
:2090800019D1206E48F076FA00213720FFF7F4FA29461720FFF7F0FAA8B9A37E6BB97102B5
:2090A0001920FFF7E9FA70B90823C4E9076584F82430022070BD012070BD31461920FFF71E
:2090C000DBFA0028F0D0FFF7C7FBFFF7A1FF032070BD022070BD00BF501A00202DE9F04156
:2090E0002B4C0546884617461E4694F82400042834D0082806D1E369AB4206D0FFF73EFBFA
:209100000228F2D00120BDE8F0814FF0FC0CA26D2048117B204B80F8A4CEC3F8588051B1F8
:20912000526942B194F8E020002A0CBF4FF480724FF4007201E04FF480721A6617491848C0
:2091400048F0B8FD01220623C4E90085C4E90376227284F824300020BDE8F081206E48F01E
:2091600009FAA37E5BB969021820FFF785FA40B994F82430082BC8D04FF0FE0CC7E7294695
:20918000F2E7FFF769FBFFF743FF0320BBE700BF501A0020482B002098010020C801002021
:2091A000A81A002070B50379204C002B14BF0123002384F8503003D1002384F8243070BD8B
:2091C0001B4D002195F9AB2E032047F0ADFD0028F2D04668304647F095FD84F8F10000282F
:2091E000EAD095F8A93E003B18BF0123304684F8F2305CF089FD0AF091FA28B9237E84F8A2
:2092000024000133237670BD5BF00EFF30B1237E00220133237684F8242070BDD5F88430F9
:2092200063610123207684F8243070BD501A0020482B002010B55BF0F7FE48B10B4C237EA0
:209240000133DBB2072B237603D9002384F8243010BD0AF063FA0028F7D0054A0123D2F863
:209260008420626184F8243010BD00BF501A0020482B00202DE9F041844C94F85050002D9E
:2092800000F0F28094F82420814E0227531E082B3FD8DFE803F035379C3E694F153E0500D9
:2092A0005BF0D8FD002840F0E6806369D6F88420FA3393422AD2FFF7BDFF94F82420E5E746
:2092C0005BF0C8FD0028F0D0236A0022012B227640F2D580E16994F8F200013B0131C4E9B9
:2092E000071310B16A4BC3F8A02E082284F82420A2F10805B5FA85F56D092846BDE8F081A8
:2093000084F824705BF0A6FD002844D194F82420531EDBB2022B0AD85D4B6169D3F8843044
:209320005B1AC82BE4D9FFF785FF94F82420042ADED1E2E7D4F82431002BD9D1544BE66835
:20934000D3F884306361072284F82420002ECFD0D4E9002123690120B047D7E76369D6F83A
:20936000841064338B42C3D2D4F82081B8F1000FF4D15BF06FFD00289FD0E66884F81880C6
:20938000042384F82430002E73D0D4E9002123694046B047BAE75BF003FA0028B6D196F858
:2093A000AD3E002BA3F10203B3FA83F314BF022201225B096276A3765BF0F2F900287FF49B
:2093C0007AAF344A0323926CA26284F824305BF0E7F900289AD12E4B206293F8DC6EB3F8B5
:2093E000DE0ED3F8E0EED3F8E0CED3F8E07ED3F8E02E84F82E6093F8E41EA08593F8E56ED3
:2094000084F8322093F8E50ED3F8E82E6263B3F8EE8EB3F8EE2E84F83310B3F8EE1EC2F341
:209420000B1343EA182303F00F0301F00F024FEA1E6E4FEA1C4C3F0A360900F00F0003F5BA
:20944000FA63042184F8390084F82FE084F830C084F8317084F83860638784F83C2084F86F
:2094600024102846BDE8F08184F824502846BDE8F081054641E7042384F824303DE7FAD167
:20948000FFF78AFD94F82420531E42E7501A0020482B0020F83900202DE9F04FC64C94F884
:2094A000506095B0002E00F0818194F82420C34F04F1580804F14009531E082B00F2968076
:2094C000DFE813F034005A00200194008300A500190094000900FEF755FE002840F01A8265
:2094E0006369D7F88420FA3393427CD2FFF790FD94F82420E0E7FEF745FE0028F0D0236A16
:209500000022012B227640F21B82E269013B511CC4E90713082284F82420A2F10806B6FAA0
:2095200086F67609304615B0BDE8F08F206E48F021F800210846FFF79FF80546FFF78CF930
:20954000012D50D1206E4FF0000A84F819A048F011F840F2AB110820FFF78EF8052800F0C0
:209560007A81012800F04281FFF776F9627E002AD1D0022384F82430206E47F0FBFF637E6F
:20958000022B0CBF4FF08045002500213720FFF773F829462920FFF76FF80546FFF75CF926
:2095A0000DBB637E022B00F06981A576206E47F0E1FF00210920FFF75FF8002873D0FFF743
:2095C0004BF994F82420531E10E020684FF40071FFF712F9012800F02681022800F02A8154
:2095E000002800F03A8194F82420531EDBB2022B0AD8724B6169D3F884305B1AC82B8CD9E8
:20960000FFF706FD94F82420042A86D18AE7A26D117B136A002900F0D5805269002A00F030
:20962000D18094F8E020002A00F0CC80B3FA83F35B09002BD7D004A900250DF10F03022288
:209640000591404605A94FF0010ACDE90B3A0792CDE90955CDE90E55CDE91055ADF8105015
:2096600006958DF820508DF834508DF84850139548F020FBFEF7EEFC9DF80F3003F01F0371
:20968000052B00F05081FFF7C3FCD4F80CB0BBF1000F00F0DD802A46236961685046D8471A
:2096A00094F8242008E710214846FFF7A5F88246002884D101217F20FEF7A6FD0128054687
:2096C0007FF47DAF50460221FEF79EFD002800F0038101287FF473AF16213A20FEF794FD31
:2096E00001308002A062FFF7B7F8206E47F042FF00210A20FEF7C0FF002840F0E680032327
:2097000084F82430102105A8FFF776F800287FF46AAF9DF821309DF822109DF81C209DF870
:2097200015009DF816501B01DBB243EA111303F5FA636387DDF81D3001F00F0184F83C10F5
:209740001BBA110902F00F0245EA002084F8381084F839209DF814109DF817206363069B43
:209760002363A08584F82E1084F82F20FFF774F8A37E6BB9206E47F0FDFE4FF4007110206E
:20978000FEF77AFF0546FFF767F8002D7FF4AEAE0B4848F03BFC00220423A4F85C00304646
:2097A000226284F8243015B0BDE8F08F304684F8246015B0BDE8F08F501A0020482B0020F0
:2097C00040787D012268217A4FF4807302EB01214046002248F03AFE237A0133DBB22372DE
:2097E000A3F10203B3FA83F35B0922E7042304AA05A9404607930692CDE909AACDE90BAA31
:20980000CDF814A08DF820A08DF834A0CDF838A048F050FAFEF71EFC9DF81330AB2B04BF92
:2098200002236376A0E66369D7F8842064339342BFF4D9AEFFF710F8FFF7EAFBE5683DB1AB
:209840000022104623696168A84794F8242033E694F8242030E6657686E60190FEF7FCFFB5
:20986000E56801982076042384F82430002D3FF459AED4E900212369A847B4E6206E47F056
:2098800079FE29463A20FEF7F7FE04AA8246042305A9404606920793CDE90955CDE90B5571
:2098A00005958DF820508DF834500E9548F002FAFEF7D0FBBAF1000F07D1FEF7CDFF049B87
:2098C0001BBAC3F38073A37670E6FEF7C5FFFFF79FFB94F82420EFE504212C20FEF794FCB8
:2098E000032182464E20FEF78FFC0C2183463620FEF78AFC0BF1020B421C02FA0BF205FA68
:209900000AF5A2FB0501420A42EAC152A262FEF7A3FFEAE60190FEF79FFF0198042306467F
:2099200084F82430FEE50E4BE568D3F884306361072284F82420002D3FF4EFAD504698E791
:2099400008D0042384F82430FEF786FF94F82420531E4BE6FEF712FF02287FF444AE2EE6A3
:20996000482B00202DE9F84FBA4C94F8081F0546C1F34001D4F8100F47F008FE94F8081F23
:20998000D4F80C0FC94301F0010147F0FFFD002D00F0CD806E1EB04FB04D5FFA86FB4FF0A3
:2099A0001008D4F8100F47F0D5FDD4F80C0F47F0D1FDB4F8183F002B40F0438194F81A1FC8
:2099C000D4F81C0F47F0E2FD4FF0FA094FF47A704FF0010C7B68C3F30803002B40F0088137
:2099E000EFF31183002B40F00381D4F88420A968D4F884309A42F8D1D4F8403F9942F4D87A
:209A0000D4F83C6F00FB06F35B1AB3FBF6F300FB02327B68C3F30803002B40F0A880EFF397
:209A20001183002B40F0A380D4F88430D5F808A0D4F884108B42F7D1D4F8401F8A45F3D865
:209A4000D4F83C6F00FB06F1A1EB0A01B1FBF6F100FB03139B1AB3F57A7FDAD3B9F10109AB
:209A6000B8D1D4F8100F47F075FDD4F80C0F47F071FDB4F8183F002B40F0D78094F81A1FC3
:209A8000D4F81C0F81F0010147F080FD4FF0FA0C4FF47A704FF0010E7B68C3F30803002B19
:209AA00040F08680EFF31183002B40F08180D4F88420A968D4F884309A42F8D1D4F8403FAD
:209AC0009942F4D8D4F83C9F00FB09F35B1AB3FBF9F300FB02327B68C3F308034BBBEFF377
:209AE000118333BBD4F88430D5F808A0D4F884108B42F7D1D4F8401F8A45F3D8D4F83C9F8E
:209B000000FB09F1A1EB0A01B1FBF9F100FB03139B1AB3F57A7FDED3BCF1010CBCD10BF1C8
:209B2000FF365FFA86FBBBF1FF0F7FF43AAFBDE8F88FEFF3118988F31288AE682B68DB03BC
:209B400044BFC4F838EFAE68D4F88430D4F8381F5FFA89F989F31188D4F83C9F0B4400FB85
:209B600009F1891BB1FBF9F100FB0313D0E7EFF3118E88F31288D5F808A02B68D90344BF6C
:209B8000C4F838CFD5F808A0D4F88430D4F8381F5FFA8EFE8EF31188D4F83C6F0B4400FB2A
:209BA00006F1A1EB0A01B1FBF6F100FB031351E7EFF3118188F31288D5F808902B68DA03DD
:209BC00044BFC4F838EFD5F80890D4F88430D4F8382FC9B281F31188D4F83C1F1A4400FB7F
:209BE00001F3A3EB0903B3FBF1F300FB023272E7EFF3118188F31288AE682B68DB0344BFAA
:209C0000C4F838CFAE68D4F88430D4F8382FC9B281F31188D4F83C1F1A4400FB01F39B1B06
:209C2000B3FBF1F300FB0232F3E6D4F8343F002B3FF42CAFD4F8203FC3F8009084F8319F50
:209C400024E7D4F8343F002B3FF4BEAE46F072FDBAE600BF482B002000ED00E010E000E0BC
:209C60002DE9F84FB74CB84F94F8081FD4F8100FB64DC1F3400147F089FC94F8081FD4F8AC
:209C80000C0FC94301F0010147F080FC4FF0050B4FF01008D4F8100F47F05CFCD4F80C0FF0
:209CA00047F058FCB4F8183F002B40F0438194F81A1FD4F81C0F47F069FC32264FF47A701A
:209CC0004FF0010C7B68C3F30803002B40F00781EFF31183002B40F00281D4F88420A968DC
:209CE000D4F884309A42F8D1D4F8403F9942F4D8D4F83CEF00FB0EF35B1AB3FBFEF300FB4B
:209D000002327B68C3F30803002B40F0A780EFF31183002B40F0A280D4F88430D5F808A001
:209D2000D4F884108B42F7D1D4F8401F8A45F3D8D4F83CEF00FB0EF1A1EB0A01B1FBFEF146
:209D400000FB03139B1AB3F57A7FDAD3013EB9D1D4F8100F47F0FEFBD4F80C0F47F0FAFBF8
:209D6000B4F8183F002B40F0DA8094F81A1FD4F81C0F81F0010147F009FC4FF0320C4FF400
:209D80007A7001267B68C3F30803002B40F08780EFF31183002B40F08280D4F88420A96858
:209DA000D4F884309A42F8D1D4F8403F9942F4D8D4F83C9F00FB09F35B1AB3FBF9F300FBE4
:209DC00002327B68C3F308033BBBEFF3118323BBD4F88430D5F808A0D4F884108B42F7D177
:209DE000D4F8401F8A45F3D8D4F83C9F00FB09F1A1EB0A01B1FBF9F100FB03139B1AB3F567
:209E00007A7FDED3BCF1010CBCD10BF1FF3616F0FF0B7FF43FAFBDE8F88FEFF3118988F38C
:209E20001288D5F808A02B68DB0344BFC4F8386FD5F808A0D4F88430D4F8381F5FFA89F949
:209E400089F31188D4F83C9F0B4400FB09F1A1EB0A01B1FBF9F100FB0313CFE7EFF3118E8D
:209E600088F31288D5F808A02B68D90344BFC4F838CFD5F808A0D4F88430D4F8381F5FFAB2
:209E80008EFE8EF31188D4F83CEF0B4400FB0EF1A1EB0A01B1FBFEF100FB031352E7EFF37E
:209EA000118188F31288D5F808902B68DA0344BFC4F8386FD5F80890D4F88430D4F8382FA8
:209EC000C9B281F31188D4F83C1F1A4400FB01F3A3EB0903B3FBF1F300FB023271E7EFF3F1
:209EE000118188F31288D5F808E02B68DB0344BFC4F838CFD5F808E0D4F88430D4F8382F67
:209F0000C9B281F31188D4F83C1F1A4400FB01F3A3EB0E03B3FBF1F300FB0232F1E6D4F842
:209F2000343F002B3FF429AFD4F8203F1E6084F8316F22E7D4F8343F002B3FF4BEAE46F06B
:209F4000F9FBBAE6482B002000ED00E010E000E00E4B30B4DB68427801780D4CDB43C3F35D
:209F60000223C3F10403DBB202FA03F360181B0101F01F050122490903F0F003AA4080F81C
:209F8000003344F8212030BC704700BF00ED00E000E100E000F01F0240090123032803FA7B
:209FA00002F304D004280CD0022805D07047074A116C0B4313647047044A516C0B435364C0
:209FC0007047024A116B0B43136370470038024000285FD00368374A2DE9F04103F13F440C
:209FE00004F57E0402EB9422012492F8982002F01F055209032A04FA05F456D0042A4FD0D4
:020000040800F2
:20A00000022A48D08588B5FA85F0C0F11F00C0F3CC0603EB860600F0070082000F24306AB6
:20A02000944020EA04003062306A01FA02F20243002132624FF0010E0A464FF0030C022714
:20A040000EFA02F838EA050002F101021CD118680CFA01F420EA04001860186807FA01F67B
:20A0600006431E609E6826EA04069E6098689860586820EA0800586058685860D86820EAB7
:20A080000400D860D868D860102A01F10201D7D1BDE8F0817047084A556C2C435464B1E796
:20A0A000054A156B2C431463ACE7034A156C2C431464A7E770DB0608003802402DE9F043F9
:20A0C00085B00D461746044647F0BEFA002859DB3B4EDFF8F88008EB000206EB800006F6CC
:20A0E000847392F8A090C0F8443F002C60D0A2884FF00043B2FA82F2D34005D0314A116870
:20A1000021EA0301116053612946204645F004FD256805F13F4505F57E05AD0A204647F028
:20A1200093FA00F0FC0303F1804303F59C3300F003009A6880000F21814022EA01029A60B6
:20A140009A68EDB205FA00F0104398602CB1A0884FF00044B0FA80F0C44008EB87074E446B
:20A16000D7F8B0308DF80D300021012302A88DF80E3002948DF80C10FDF742FF96F8883FFB
:20A18000F02B02D805B0BDE8F0830F4B13F809308DF80430F02103224FF4807301A886F813
:20A1A000881F8DF80520ADF80630FFF7D1FEE9E72946204645F0B0FC4FF0FF35AEE700BF61
:20A1C000482B0020003C01406C5E070870DB0608002869D0F0B58388B3FA83F3202B85B089
:20A1E0000446C3F11F024AD0304E314D16444FF0004005EB820230FA03F396F8A060C2F875
:20A20000441F05D02B4A116821EA0301116053612046002145F080FCA3882268B3FA83F4D3
:20A22000C4F11F0303F0FC0101F1804101F59C3103F0030398000F2702F13F438A688740EC
:20A2400022EA070203F57E038A60C3F38723834088684FF000420343354422FA04F48B6034
:20A260004FF40062012302A88DF80E300294ADF80C20FDF7C5FE95F8883FF02B01D805B08D
:20A28000F0BD0D4B9B5D8DF80430F02103224FF4807301A885F8881F8DF80520ADF806304A
:20A2A000FFF756FE05B0F0BD704700BF70DB0608482B0020003C01406C5E070810B4B8B10D
:20A2C0000D4CD4F8903F102B05D15DF8044B0521002045F009BF03EB4302224482F8951FCB
:20A2E00001210B4482F8940F82F8961FC4F8903F5DF8044B704700BF482B00208078202130
:20A30000DCE700BF2DE9F04FDFF8ACA32DED028B9AF8D81F002297B0CAF8C82FCAF8CC2F31
:20A32000CAF8D02FCAF8D42FCAF8C42F19B19AF8D92F8AF8C42F9AF8DA2F1AB19AF8DB2F07
:20A340008AF8D32F9AF8DE2F1AB19AF8DF2F8AF8CE2F9AF8DC2F1AB19AF8DD2F8AF8C92F70
:20A360009AF8E03F05935A1ED3B257B203937B1C00F0AA80C54AC64E52F83790029602EB8E
:20A38000C70200231279019308EE102A1D463446984626783946304648F0FAFC83463046C7
:20A3A000BBF1000F1ED046F001FEEA1D1321D2B220B14FF0000E827180F807E045F0ACFBB4
:20A3C000207848F00FFD4FF0070308F1010223714FF0010384F802806070CDF804B05FFAE5
:20A3E00082F8E3700135042D04F10504D1D118EE100A029ECDF81080FFF7CCFDA549A64AD7
:20A400004868024042F440324A600FB9019B5BB9A24C4820FFF7BEFD2046022160F03CFD67
:20A42000A26842F00102A2609A489C4A4168BAF8E24F41F400014160516821F48051516060
:20A44000916B21F4401141F480119163D16841F46001D160956B85F44011C1F3015101EB24
:20A4600081011F2000FA01FC25EA0C0C112505FA01F141EA0C019163D16841F0E061D160CE
:20A48000956BC5F30151C1F10401C9B201EB810188404FF0120C25EA00000CFA01F108439B
:20A4A0009063E4B1BAF8E41FCAF8EC4FA1B1BAF8E62FCAF8F01F62B1019B7948521A90FB11
:20A4C000F2F2CAF8F42F6BB917B0BDEC028BBDE8F08F744A1288EFE7734A1188E7E7734A5F
:20A4E0001488DFE74846049960F0D6FC684B012003F114080723F278441CE4B252B375784D
:20A500003279A5F10A0101EB410105EB450C092D03FA01FE03FA0CFB02FA01F140F2A0800A
:20A52000D9F80C2022EA0E0E41EA0E01C9F80C10421E02EB82021F21062801FA02FC05FAA8
:20A5400002F273D8D9F8341021EA0C010A432046C9F834200536B045CDD1D9F80820039964
:20A5600042F40072C9F80820D9F8082042F48072C9F80820D9F80820574442F00102C9F8B6
:20A58000082097F9E82F022046F0CEFB044600289AD04668304646F0B5FB454A431E2421B0
:20A5A00001FB032393F89C50002D8DD1059983F89D10062283F89C20002885D0304646F029
:20A5C000A1FB5BF0CDFA60680AF0B4F907A80AF073F9049EA26837480792012E8CBF4FF4C8
:20A5E000806300230D9309F14C034FF48072CDE90A56089309904FF4003360680C9507A95E
:20A600004FF400674FF40056CDE91023CDE90E760AF064F96268136843F001031360D9F8BD
:20A62000083043F08043C9F808304DE7C11FA0F10D0201EB81014FF01F0E02EB82020C28C0
:20A640000EFA01FC0EFA02F005FA01F113D8D9F8302022EA0C0211432046C9F8301079E7C9
:20A66000D9F8101002FA0CF221EA0B0B42EA0B02C9F810205CE7D9F82C1005FA02F221EA56
:20A6800000010A432046C9F82C2063E72CDC06080C3B002000230140E030FCFF0020014062
:20A6A000803801002E7AFF1F2C7AFF1F2A7AFF1F98010020403B0020482B00202DE9F84F51
:20A6C0002E4F00EB800407EBC40454F8F46C2EB1054614F8DF0C00F0FF0820B14FF00008F8
:20A6E0004046BDE8F88F89469A46934645F036FF4FEA49010123C9B204F8DE1C04F8DDBC09
:20A7000004F8DB3C04F8DA8C04F8DC3C04F8DF3C04F8E08CB28844F8D8AC9105814644F89E
:20A72000D4AC1DD43388DA0510D442F20F7405E045F014FFA0EB0903A34215DC33889B057E
:20A74000F6D433889BB243F480733380B3889BB243F440734FF00108B3804046BDE8F88FAB
:20A7600098464046BDE8F88F37F8803C01339BB2284627F8803C5FF0C7FEB1E7403C00204C
:20A7800070B5464E16F87E4C04EB440306EBC303650013F87C3C032B6ED8DFE803F0592963
:20A7A0001E02254406EBC50555F8780C002870D116F81C3C9C425FD0013404F003029342A5
:20A7C00006F87E2C58D002EB420406EBC404022344F8780C04F87C3C70BD2B1906EBC303FC
:20A7E00053F8782C72B1013A43F8782C002070BD2B1906EBC30353F8782C002AF3D10222E4
:20A8000003F87C2C254406EBC50515F8703C013BDBB205F8703C8BBB214B16F81C6CD3F833
:20A82000C01255F8740C621C02F003024B1E0324B242034405F87C4CB3FBF1F045F8780C24
:20A840001AD0994218D8013845F8780C012070BD47F0C6FF80B1124B2C44D3F8C02206EB63
:20A86000C404012102F51C5304F87C1C0F33B3FBF2F344F8783C70BD012070BD084BD3F896
:20A88000C022012002F2E733B3FBF2F345F8783C70BD013845F8780C002070BD403C002013
:20A8A000980100202DE9F84F3249DFF8D4B091F8AD1E01240229074619461046CBF82041E2
:20A8C0004FF000022C4C1D4618BF7F02FDF7CAFB2A4B63626B02A362E36A40F2FF5943F095
:20A8E00093034FF400704FF48A62E3620121C4F83890A0601020E2605AF09EF8012D40F243
:20A9000051434E46C4F83890CA4640F252488EBF4FF0120998464FF011090A25C4F838A00E
:20A920000121A7604846C4F80C805AF085F803464FF0000C40F2774201213720A6632BB96C
:20A9400000231846CBF81C31BDE8F88FA663C4F808C0E2605AF070F8013DA6630028EFD08B
:20A9600015F0FF05DAD10346CBF82051CBF81C31BDE8F88F482B0020002C014000E1F5058F
:20A98000501A00202DE9F843DFF8748098F82450042D0446894617461E4608D0082D02D023
:20A9A0000020BDE8F883FEF7F7FA0228F8D101234A4620460021FFF775FF68B1FEF73AFC95
:20A9C000D8F80C40002CEBD00022D8F81030D8F804101046A047E3E7084BC8F80090D3F8E9
:20A9E0008420C8F804400523C8E90376C8F8142088F824300120BDE8F88300BF482B002002
:20AA0000501A00202DE9F84F3149DFF8CC9091F8AD1E1E4602292F4B07464FF0010418BFDD
:20AA20004702012E40F25948C3F8244198BF4FF48B683B469346474640F2FF55B0468CBF70
:20AA40004FF0190A4FF0180A0A241E4640F2FF53C9F838300121C9F808605046C9F80C70D6
:20AA600059F0EAFF03464FF0000C40F2774201213720C9F83850ABB9584641460122FDF7C3
:20AA8000F1FA4646144A154B536276029662D36A43F09103D3620F4B00210846C3F81C1172
:20AAA000BDE8F88FC9F83850C9F808C0C9F80C2059F0C2FF013CC9F838500028DCD014F043
:20AAC000FF04C3D1034BC3F82441BDE8F88F00BF482B0020501A0020002C014000E1F50521
:20AAE0002DE9F047364C82B005460E461746984694F8240004280CD0082806D1E369AB4283
:20AB000007D0FEF749FA0228F2D0012002B0BDE8F087DFF8B4A02660DAF8A09E6560C9F309
:20AB20004F210F294FEA592222D8236A0193FBB194F8F200E0B1B9F5005F13D02148314613
:20AB40004FF40072484462F061FF09F50072C2F34F211029CAF8A02E4FEA522202D0019B89
:20AB6000012B20D192B2013A164EAD1A0B4600E0012332462846062601250021E760C4F85D
:20AB80001080257284F82460FFF73CFF0028BDD0FEF750FBE66886B12846236961680022FE
:20ABA000B0470320B2E7E269013B01320421C4E9072384F824100220A8E70320A6E700BF5C
:20ABC000501A002048770020482B0020F0B53B4C54F8185C2B78022B95B018D0012B02D092
:20ABE000002015B0F0BD95F904506B1CF8D0022DF6DC0091134614F8141C024628465FF066
:20AC000025FE0028ECD028465FF0D0FEE9E72B6A002BE5D10DF10F0C8DF80F000026012068
:20AC20000027CDE90833CDE90A12CDE90E6705938DF81C300D9310931293CDF810C0069083
:20AC40008DF830008DF84400EFF31180102383F3128854F8183C1B6A13B3069B04AE32460A
:20AC60001BB1D3691432002BFBD12B6A13B3996839B993420AD0196829B15B68996800294A
:20AC8000F7D01433F3E70E4AC3E90026C0B280F3118854F8182C136A002BFCD10120A0E777
:20ACA00004ABC0B22B6280F31188A4F118005CF035FBEEE7024A1A60FFDE00BF403C0020DE
:20ACC000283C002003681A78012A01D00020704793F90430044A03EB830302EBC30313F8E0
:20ACE000DF0CC0B2704700BF403C002070B503681D78022D13D0012D01D0002070BD044618
:20AD000093F904000A4B421C83F8B450F5D00228F3DC0A46B4332179BDE87040CEE41B6A56
:20AD2000002BEAD1012247F0F1FA012070BD00BF403C002010B50C4C54F8183C1B78022BC2
:20AD400010D154F8100C46F01BFC54F8100C08B12123C380012144F0DFFE044847F056F9B0
:20AD600024F8140C10BD00BF403C00208096980030B583B00D46012301460DF1070204469A
:20AD8000074847F033FC9DF8072035EA020304D003482A43214647F0BFFC03B030BD00BFDA
:20ADA000283C002038B505460A460C460648294647F0ACFA45F08001034847F051F9231ADC
:20ADC0005842584138BD00BF283C002013B53A4C0023D4F8C4208DF80730137803F0FD01AF
:20ADE000012905D194F8C81011B90C2184F8C810022B1ED0032B2ED001220B212F4857F050
:20AE00000FFE042045F0D6FB2C4801230DF10702002157F027FE002839D09DF80730482B5F
:20AE200035D1274BC4F8B830264BC4F8BC3002B010BDD4F8CC0046F0A3FBD4F8CC0008B1A1
:20AE40003523C380012144F067FE1F4847F0DEF8A4F8C800D0E7D4F87435506846F2A811EF
:20AE60001961002380F888301222372157F0ACFDD4F8C4300D225868242157F0A5FDD4F8E0
:20AE8000C430302258686A2157F09EFDB4E7D4F8C4301A78022A03D0032A07D00020C6E782
:20AEA000D4F8CC0046F0E6FE0020C0E758681022372157F089FDF1E7403C0020043D00202D
:20AEC000C32A0608452B0608809698002DE9F04FB54CB64E95B0002305464FF4F0728B46C8
:20AEE00004F6F800202184F8F43884F8F538019562F0EDFD202104F6D8204FF4F07262F0D2
:20AF0000E6FDDFF8C0C2AA4932274FF0100E4FF47A704FF00108DCF80430C3F30803002BE3
:20AF200040F0BC80EFF31183002B40F0B780D6F884208D68D6F884309A42F8D1D6F8403FC2
:20AF40009D42F4D8D6F83C9F00FB09F35B1BB3FBF9F300FB0232DCF80430C3F30803002B73
:20AF60007BD1EFF31183002B77D1D6F88430D1F808A0D6F88450AB42F7D1D6F8405FAA45F6
:20AF8000F3D8D6F83C9F00FB09F5A5EB0A05B5FBF9F500FB03539B1AB3F57A7FDBD3013F72
:20AFA000B9D194F8B92C002A52D094F8BA3C013B022B4DD803EB830004EBC0017D4D91F8C6
:20AFC000547D05EBC0004FF0010C022FC4F8BC0C84F844CD00F0C182DBB204EB0313D3F8D2
:20AFE000CC3DC1F8583D9BB302234FF4807081F8543DA5F188034C3DA1F8600DC1F86C3D38
:20B00000C1F8705D1509013D042D02F00F0200F28782694F07EB4503B3F8840040FA02F3CF
:20B02000DB0740F17D82012303FA02F2013A10403D4460F053FA95F89020604B104403EB16
:20B04000C000C4F8C40C8379002B47D0412B45D06FF0010015B0BDE8F08FEFF311898EF39F
:20B060001288D1F808A00B68DD0344BFC6F8388FD1F808A0D6F88430D6F8385F5FFA89F9B7
:20B0800089F31188D6F83C9F2B4400FB09F5A5EB0A05B5FBF9F500FB03537CE7EFF3118521
:20B0A0008EF31288D1F808900B68DB0344BFC6F8388FD1F80890D6F88430D6F8382FEDB284
:20B0C00085F31188D6F83C5F1A4400FB05F3A3EB0903B3FBF5F300FB02323CE72323C3809A
:20B0E000092144F019FDD4F8C43C13B11A689B881383D6F83025324BB3EB920F80F033820D
:20B10000B3EBD20F80F03182B3EB121F80F03182B3EB521F80F03182B3EB921F80F03182F7
:20B12000B3EBD21F80F03182B3EB122F80F02F824FF4807000230122FF210DF10F088DF82A
:20B140000F10CDE90483CDE90833CDE90A33D4F8BC1CA4F8C00C0D9306928DF81C208DF825
:20B160003020EFF31180102383F31288D4F8BC3C1B6A002B00F0D881069B04AD2A461BB17E
:20B18000D3691432002BFBD10B6A002B00F01582996839B99A421AD01968A9B15B689968B7
:20B1A0000029F7D01433F3E7403C0020482B002010E000E09449002070DB0608F82D0020E4
:20B1C000404B4C0000ED00E0B74AC3E90025C0B280F31188D4F8BC1C0B6A002BFCD18C22BC
:20B1E0000120CDE908330DF10E0A05938DF81C300D93109312938DF80E2000230022CDE928
:20B200000E23CDF82880CDF810A006900B908DF830008DF84400EFF31180102383F31288B6
:20B22000D4F8BC3C1B6A002B00F08781069B2A461BB1D3691432002BFBD10B6A002B00F0BC
:20B24000BC81996839B993420AD0196829B15B6899680029F7D01433F3E7934AC3E9002531
:20B26000C0B280F31188D4F8BC2C136A002BFCD19DF80F301B2B40F09081D4F8C43C0122DD
:20B2800084F8F4280BB12322DA80DFF81C92402248460A2147F03AF88A21002301228DF83C
:20B2A0000E1000200021CDE90E01CDE90833D4F8BC1CCDF810A0CDF8288005938DF81C308A
:20B2C0000D931093129306920B928DF830208DF84420EFF31180102383F31288D4F8BC3C19
:20B2E0001B6A002B00F03181069B2A461BB1D3691432002BFBD10B6A002B00F05B81996839
:20B3000039B9934209D0196829B15B6899680029F7D01433F3E7C3E90095C0B280F311889E
:20B32000D4F8BC2C136A002BFCD19DF80F2094F8B81CC2F3801284F8FC2D002900F0D48067
:20B34000022900F0B980D6F830355849B1EB930F80F01F81B1EBD30F80F00981B1EB131F31
:20B3600080F00981B1EB531F80F00981B1EB931F80F00981B1EBD31F80F00D81B1EB132F19
:20B3800034BF4FF48076802694F8001EA4F8FE6D182914D1464F474800215B08B3FBF6F3C5
:20B3A000A7FB03730F465B0B66F30F076BF30F0163F31F4762F31F41C4F8081E47603A4861
:20B3C000A4F8C06C0222002146F0A0FFC82044F0D3FFD4F8BC0C4FF0800B002600270023CF
:20B3E0000122CDE90E67CDE908338DF80EB0CDF810A0CDF8288005938DF81C300D9310933D
:20B40000129306920B928DF830208DF84420EFF31182102383F31288D4F8BC3C1B6A002B68
:20B4200038D0069B002B3DD02B46D96914330029FBD1006A002800F0BA80816839B98342E0
:20B4400009D0016829B1406881680029F7D01430F3E7C0E90095D2B282F31188D4F8BC0CCD
:20B46000036A002BFCD19DF80F3013F00203B6D1019841788278007884F8100EC1F12001D3
:20B48000C2F11002184684F8111E84F8122E15B0BDE8F08F0562D2B282F3118802485BF0AB
:20B4A0003DFFDBE72B46C4E7FC480020809698005917B7D1484A0020D6F830354048B0EB60
:20B4C000930F72D2B0EBD30F51D2B0EB131F52D2B0EB531F53D2B0EB931F54D2B0EBD31FC3
:20B4E00034BF802640264FE7D6F830353549B1EB930F4ED2B1EBD30F39D2B1EB131F3AD2A5
:20B50000B1EB531F3BD2B1EB931F3CD2B1EBD31F41D2B1EB132F34BF4FF48076802633E749
:20B520000020C4F8C40CDBE504ADC0B20D6280F3118825485BF0F2FE4CE60D62C0B280F3D3
:20B54000118821485BF0EAFE8DE60D62C0B280F3118848465BF0E2FEE2E691F8613D634407
:20B5600081F8613D4EE50220E4E50420E2E504260AE70820DEE5082606E71020DAE5102665
:20B5800002E72020D6E52026FEE64020D2E58020D0E50226F8E64026F6E6D4F8C40C20210C
:20B5A00044F0BAFA4FF0FF3054E50E46ECE6C0F80090FFDEC3F80090FFDE034A1A60FFDEE5
:20B5C000002D3101404B4C00FC4800200146014846F046BD544A0020014488420ED010B499
:20B5E0000346074C074813F8012B04FB00F0994280EA0200F7D15DF8044B704701487047D0
:20B6000093010001C59D1C81094B93F86231042B08D9053B032B08D801231A4600B103701E
:20B620001046704700230122F8E700231A46F5E7482B0020F0B40D6800240CE0BCF1050FFC
:20B6400018D8A0F137030A2B14D104EB840415F8010B03EB4404A0F13003DEB2092EA0F133
:20B660006107A0F1410CF0D9052FE7D8A0F157030A2BEAD00D601460F0BC70479FED727A32
:20B6800007EE901A20EE070AF8EE677A27EE800AFDEEC07A17EE903A2033402B00F2C4809E
:20B6A000DFED6A7AB4EEE70AF1EE10FAF0EE407A0CDD9FED676ADFED676AB0EE677AB4EEC2
:20B6C000E67AF1EE10FA77EEC67AF6DC9FED627AF4EEC77AF1EE10FA0CD59FED5D6ADFED36
:20B6E0005F6AB0EE677AB4EEE67AF1EE10FA77EE867AF6D49FED5A7AF4EEC77AF1EE10FA7C
:20B7000000F38A809FED577AF4EEC77AF1EE10FA44BF9FED517A77EE677A27EEA76ADFED31
:20B72000525A9FED527ADFED526AA6EE257A67EE865AE6EE076AB6EE007AE5EEA67A27EEAA
:20B74000877ADFED476A70EE267ABDEEE76A16EE103A2033402B64D8B4EEE60AF1EE10FAAE
:20B760000CDDDFED3B5A9FED3B6AF0EE676AF4EEC66AF1EE10FA77EEE57AF6DCDFED366AA2
:20B78000F4EEE67AF1EE10FA0CD5DFED315A9FED336AF0EE676AF4EEC66AF1EE10FA77EE0E
:20B7A000A57AF6D4DFED2E6AF4EEE67AF1EE10FA3DDDDFED266A76EEE77A67EEA75A9FEDF4
:20B7C0002A5A9FED2A6ADFED2A6AA5EE856A27EEA55AE5EE866AB8EE006AE5EE267A67EE34
:20B7E000867AC7EE206AB7EE006A76EE865A76EE666A86EE257A80ED091A67EE277A66EE96
:20B80000876AC0ED017AC0ED037A80ED007A80ED027AC0ED046A70479FED0C7A77EE677AEB
:20B820007BE7DFED147ADCE79FED127A89E7DFED0D6AF4EEE67AF1EE10FA44BFDFED066A54
:20B8400076EEE77AB9E700BF27D4D236DB0F4940DB0FC940E4CB1641DB0F49C0E4CB16C1DC
:20B86000DB0FC93FDB0FC9BF92E741B99730083C15A82ABE00000000E14B2DE9F04103F5D6
:20B880006B63E04ED3ED000A96F83043F8EE600A2DED028BC6EDCB0A002C6FD1DFF8C4C398
:20B8A00096F84073C6F83C439CF80040002F39D0B6F836339FEDD46A9FEDD47A07EE903A84
:20B8C000F8EE677A20EE877AC6EE276AD04B0022012F1A6076EE876AC7EE267AC3ED017A91
:20B8E00020D0022F9A60C3ED037A1BD0032F1A61C3ED057A16D0042F9A61C3ED077A11D013
:20B90000052F1A62C3ED097A0CD0062F9A62C3ED0B7A07D0072F1A63C3ED0D7A02D09A6372
:20B92000C3ED0F7ABB4B9FEDBC6A93F882319FEDBB7A9FEDBB0ABB4A07EE903AF8EEE77ABB
:20B940009CF8583BC6EE276A1C4414FB07F4E4B207EE904A60EE870AF8EEE77AC2ED006A6D
:20B96000A7EEA00A60F02CFEBDEC028BFCEEC07A17EE903A86F89034BDE8F08196F831339B
:20B980009FEDA96AB6F832239FEDA82ADFEDA86ADFF8D0C296F84073C6F83CC307EE903AA3
:20B9A000FCEEE05AB6F834338CF8004007EE103A15EE903AF8EE655AF8EE677A86EE255A1F
:20B9C000CCF81430012386F8383306EE102AB8EEC77A27EE822AB8EE466A67EE266A22EE31
:20B9E000252A8CED025ACCED017A8CED036ACCED046A002F96D0DFED8F7A9FED8F4ADFED47
:20BA00008F5AC7EE871AC7EB0715A7EB07180CEBC5054FEAC8084FF0000EB1EE611A9FEDAB
:20BA2000886A08EB05009FED873ADFED873ADFED876A0346002207EE902AB8EEE77A27EE4F
:20BA4000027AFDEEC77A17EE901A2031402900F2D080B4EEC47AF1EE10FAF0EE477A0CDD42
:20BA6000DFED7B4A9FED7B5AF0EE672AF4EEC52AF1EE10FA77EEE47AF6DCF4EEE57AF1EEF6
:20BA800010FA0CD5DFED724A9FED735AF0EE672AF4EEC52AF1EE10FA77EEA47AF6D4F4EE82
:20BAA000C67AF1EE10FA40F39A8074EE677A27EEA75AB0EE630AA5EE030ADFED684AE5EEBB
:20BAC000004A65EE272AB7EE005AE2EEA47AB0EE458AF0EE454AA1EEA78AE1EE274AC5EEFE
:20BAE000088A84EE880A77EE067ABDEEE75A15EE101A203140296FD8B4EEC67AF1EE10FAE6
:20BB00000CDD9FED535A9FED537AF0EE674AF4EEC74AF1EE10FA77EEC57AF6DCF4EEE57A88
:20BB2000F1EE10FA0CD59FED4A5A9FED4B7AF0EE674AF4EEC74AF1EE10FA77EE857AF6D421
:20BB4000F4EEC67AF1EE10FA3CDD74EE677A27EEA75AF0EE632AE5EE032A9FED407AA5EE24
:20BB6000227A65EE274AB8EE005AE4EE877A67EE857A87EE887A0132A24203F1280343ED61
:20BB8000048A03ED037A03ED017A43ED028A83ED000AC3ED056AC3ED026AC3ED016AC3ED03
:20BBA000046AC3ED036AFFF646AF783085427FF43AAF0EF5707EBEF5346F05F570757FF4AC
:20BBC0002EAF75E69FED267AF4EEC77AF1EE10FA48BF75EEE77ABAE7F0EE667AC9E79FED8F
:20BBE000205AF4EEC57AF1EE10FA48BF75EEE77A5DE7B7EE000AF0EE408AB0EE408A72E79A
:20BC0000403C0020384D002083F9223EBD378635CC510020482B0020555555406E12833A0C
:20BC200048E1FA3EC45100200060EA4827D4D2360AD7233C00004842DB0F4940DB0F49C0A9
:20BC4000DB0FC93F92E741B99730083C00000000DB0FC940E4CB1641E4CB16C115A82ABE50
:20BC6000DB0FC9BF48A700202DE9F04F07EE900A2DED068B9FEDF27AF24EDFEDF36AB6F8A5
:20BC8000D43496F8DA54C6F82C05B8EE679A0AEE103A87EE095AB6F8D634C6F8E85400225C
:20BCA00083B0C6F8EC2408EE103AB6F8D834DFEDE77AB8EE4AAA08EE903AB8EEC88A3AEEE2
:20BCC0000A7AF8EEE88AB4EEC78AF1EE10FA68EEA77AB4EEE65A06F2DC43B8BFB0EE478A56
:20BCE000F1EE10FA83ED028A83ED01AAC3ED007A00F1FE8207EE905AF8EEE77AB7EE007A64
:20BD0000C7EE279AD24B96F8A01E1A46143201929E4603F12C04F6EE005A65EE256AF7EEFE
:20BD2000007A86EE887ADFEDCB3ADFEDCB4A9FEDCB6AD3ED05AAB4EEE77AF1EE10FAB8BFCE
:20BD4000B0EE677ABDEEC77AB0EE004A17EE107AB8EEC77A29EE066AC5EE076AC6F88877B2
:20BD600087EE875A66EEA36AAEEC015A8AEE267AC8EE267A37EE257A77EEA57AB4EEC47A81
:20BD8000F1EE10FAF4EEE47AB8BFB0EE447AF1EE10FA88BFF0EE647ABDEEC77AFDEEE77A83
:20BDA00017EE102A17EE900A02F1FF3B00F10108BBF1230FA8BF4FF0230BB8F1230FC146EA
:20BDC0002BEAEB7BA8BF4FF02309C345C8BFD946012FB8BF0127A9EB0B08CEED006A98FB3A
:20BDE000F7F883ED046AC6F89427C6F8980708F10108002940F0E380DFED990ADFED995AB4
:20BE00009FED992A9FED995ADFEDA42A9FEDA43ADFEDA43A9FED964ADFEDA31A03F5E36274
:20BE200007EE901AB8EEE76A66EE207A37EEA57AFDEEC76A16EE903A2033402B00F211820D
:20BE4000F3EE026AB4EEE66AF1EE10FA0CDDDFED914ADFED8F6AB0EE471AB4EEE61AF1EEE5
:20BE600010FA37EE647AF6DCB4EEC57AF1EE10FA0CD5DFED884ADFED886AB0EE471AB4EE3B
:20BE8000E61AF1EE10FA37EE247AF6D4B4EEE57AF1EE10FA40F3FA81DFED766A36EEC77A83
:20BEA00067EE076AB0EE431AA6EEA21AB0EE630AA1EE260A67EE264AFDEEE76AA4EE807A1A
:20BEC00016EE903A2033402B27EE047A00F2D381DFED696AB4EEE66AF1EE10FA40F3FC81D3
:20BEE0009FED6C0A9FED6A1AF0EE676AF0EE664AF4EEC14AF1EE10FA76EEC06AF6DC9FED31
:20BF00005D1AF4EEC14AF1EE10FA13D59FED611ADFED614AB0EE660AB4EEE40AF1EE10FAE7
:20BF200076EE816AF6D4DFED546AB4EEE66AF1EE10FA0CDD9FED576ADFED556AF0EE674A33
:20BF4000F4EEE64AF1EE10FA77EEC67AF6DCF4EEC57AF1EE10FA0CD59FED4E6ADFED4E6ABC
:20BF6000F0EE674AF4EEE64AF1EE10FA77EE867AF6D4F4EEE57AF1EE10FA40F37F81DFEDDF
:20BF80003D6A76EEE77A67EEA76AF0EE434AE6EEA24AB0EE631AA4EEA61A27EEA66AE6EE3E
:20BFA000017A67EE847A0131242982ED007AC2ED017A02F108027FF433AFDFED30AA4FF0EA
:20BFC000000A44E905AB44E902874FF490720021204644F80C9C61F07AFD4FF49072A0184F
:20BFE000002161F074FD264B04F51574A342E8D1019BDFED247AC3ED00AA012329EE279A71
:020000040800F2
:20C0000086F8A03E002D00F02781DFED1F7A1F4E9FED182ADFED152AC7EEA81AA6F114042E
:20C0200006F5117738EE4A8AB1EE611A69EE889ADFED0C5ADFED0C6A234630463AE000BFC4
:20C0400000247449384D00200000FA440AD7233CC4540020398E633C00000C429C53493781
:20C06000C3B8B23DDB0FC93F00000000DB0F49C072F97F3FDB0F494000001042BC297E3FE1
:20C08000EC5B002027D4D2360000484228520020E4CB1641DB0FC940E4CB16C192E741B920
:20C0A0009730083C15A82ABEDB0FC9BF000010C20000807F0022B7EE005A07EE902AF8EED7
:20C0C000E77AB6EE007A77EE877AB0EE4A7AA7EEA97AF0EE477A29EE077AE0EC017AFDEEF8
:20C0E000C77A17EE901A2031402900F2D780B4EEC27AF1EE10FAF0EE477A0CDD1FED1B4A8D
:20C100005FED1D4AB0EE676AB4EEE46AF1EE10FA77EEC47AF6DCF4EEE27AF1EE10FA0CD5A7
:20C120001FED244A5FED244AB0EE676AB4EEE46AF1EE10FA77EE847AF6D4F4EEE57AF1EE36
:20C1400010FA40F3B58072EE677A67EEA74A5FED2D3A1FED2D4A1FED2D6AA4EEA34A67EE39
:20C16000A43AA4EE246AF0EE454AE3EE867AB0EE456AE1EE274AA1EEA76A84EE864AC5EE61
:20C18000064A77EE257AFDEEE73A13EE901A2031402900F28A80B4EEE57AF1EE10FA0CDD0B
:20C1A0001FED443A5FED463AB0EE677AB4EEE37AF1EE10FA77EEC37AF6DCF4EEE27AF1EE31
:20C1C00010FA0CD51FED4D3A5FED4D3AB0EE677AB4EEE37AF1EE10FA77EE837AF6D4F4EE99
:20C1E000E57AF1EE10FA6DDD72EE677A27EEA73A5FED560A5FED563A1FED567AE3EE203AE7
:20C2000063EE270AA3EE237AF8EE003AE0EE877A67EEA37A87EE867A0132AA4203F128035A
:20C22000C3ED0B4A83ED0C7A83ED0E7AC3ED0D4A83ED0F4A83ED145AC3ED116AC3ED106A08
:20C24000C3ED136AC3ED126A7FF437AFC834A74206F114067FF4ECAE03B0BDEC068BBDE897
:20C26000F08FFDEEE76AB0EE427A16EE903A2033402B7FF62DAEF0EE427A94E6F4EEE17A7C
:20C28000F1EE10FA48BF75EE677A7CE6B4EEE17AF1EE10FA48BF35EE477A01E6B7EE004A61
:20C2A000F0EE444AB0EE446A6BE7F0EE667AB1E71FED836AF4EEC67AF1EE10FA48BF72EEB3
:20C2C000E77A42E71FED887AF4EEC77AF1EE10FA48BF72EEE77A89E75FED8C6AB4EEE66A4E
:20C2E000F1EE10FA48BFF0EE676A3FF50FAE2EE65FED919AC6F8E824154603E508480023A3
:20C3000002461178022902F1060204D00133062BF7D10020704703EB430300EB4300704735
:20C320007C1B002000B50021084B83B00846C3F8C41F33F0C9FC0422054B01930DEB020111
:20C34000062033F0B5FC03B05DF804FB384D00205475C52A70B5461E00F13105344614F849
:20C36000011F601E801BFF29C0B201D033F0ACFCAC42F4D1A02055F08BFA0121022033F0AA
:20C38000A3FC40F2E93401E0013C04D04220FFF71DF90028F8D16220FFF718F9132124205D
:20C3A00033F092FC2520092133F08EFCBDE87040A02055F06DBA00BF10B58CB000234CF20E
:20C3C0000502044601A9CDE90633CDE90833ADF800208DF8023003220B930123CDE9031254
:20C3E0008DF814308DF82830CDF808D046F074F8204602A945F05EFC204646F06DF89DF822
:20C4000006000CB010BD00BF2DE9F043784D794F83B005F596702422002161F058FB97F82B
:20C42000C94F0023C5F85031002C3CD1724ED6F8F83063B39B6A53B370489847836833B30B
:20C4400003886F4F013B9BB2BC46384600210678032E00F106001ED001310629F7D100228A
:20C460003978022907F1060700F0A1800132062AF6D1D5F85011052909D0481C02FB01C247
:20C48000C5F8500102200021938010705180204603B0BDE8F083062303FB0151B1F82E3135
:20C4A000013B9BB2DBE797F8C80F07F57D63C7F8CC3F10B9504E0024B9E744F077FDC7F893
:20C4C000D80F18B183790BB1412BF3D121464D4845F066FD04460028ECD0D7F8CC3F474A97
:20C4E0009868C3F8942008B12023C380092143F013FBD7F8CC3F404E986845F041F84248C3
:20C50000D7F8CC8F45F082FD4FF00109A8F804003220C6F8188186F81C9144F04BF80423DE
:20C52000D7F8CC0F4FF0000C0DEB03029F21CDF804C045F097FE9DF805809DF804309DF87E
:20C5400006104FEA082848EA034848EA0108414606F1F80050F0AEF900287FF468AF40460F
:20C56000FCF7DEF9034600287FF461AF9DF806009DF805209DF80710000240EA0240234A21
:20C580000843904217D0C6E94033A6F8FC30A6F80831FCF7C5F9804600287FF448AF97F83C
:20C5A000C80F44F003FD45F065FB44463FE7062101FB02C266E7164AC6F8FC204FF4003347
:20C5C0004FF00062C6F800314023A6F80831C6F8042186F80A91FBF7ABFD06F1F80086F88E
:20C5E000119150F0B3F80B4BC6F8F8301FE700BF501A0020384D0020482B0020402C00205F
:20C600007C1B0020085D0020404B4C0021AAEF000004000870DB06082DE9F041BC4BBD4E8F
:20C62000BD4DBE4C0822C3F88820336B82B043F00103336307464FF4C052284640F2023345
:20C6400088466946CDE9002308F016FB6B6AC4F8548523F470436B626B6AC4F85C7543F4E1
:20C6600020436B626B6AAE49C4F8581523F470236B626B6AAB4844F8900C43F420236B6237
:20C68000736CA94944F88C1C43F480437364736BA648A74944F8800C43F0800302257363DD
:20C6A000A44F04F8885CA44EA44D44F83C1C4FF0A04344F8843CA24A44F8747C03F534636B
:20C6C000A1F5D07144F8385C44F8706C44F8343C44F86C1C0123DFF898C244F878CC07F55A
:20C6E0001077A5F5E465A6F5A066A1F58C6144F8307C44F87C5CE66304F8853C05F5A0759B
:20C70000536106F5B076216084F8823019468D4B8D4AA560A7F5BC67A03566618B4E2761C6
:20C72000A36107F5D45703F56953E5614FF050250020DFF840E22264ACF5687C02F5A04223
:20C740006764A66407F5A04706F5A046E3642565A3F54853A4F19005C4E916766265E367C8
:20C76000C4F804E0C4F80CC002462B4684F88400402683F81C21A3F822210132042AC3E9CF
:20C78000496083F81D1183F81F01C3F8300103F12803EED1002211462B46402083F8742386
:20C7A000A3F87A230132042AC3E9DF0183F8751383F87713C3F8881303F12803EED14FF0D9
:20C7C000A04363489A6822F001029A60DA6842F04002DA6007F00EFB14F8873C0022212197
:20C7E00061F317420BB142F4801214F88D1C54F8843C01299A6300F0E280DA68E66F54F8EB
:20C80000800CC2F3076121F0600141F0400161F31F620021DA603160026861F3CC220260BC
:20C8200014F8852C012A00F0B7801021494807F033FE484807F016FE54F8800C14F88F3CB5
:20C8400000224FF0FF31026142618161C26153B305F11407404E114607EB83074FEA830CFC
:20C860004FF0FF0E56F8042F1368002BACBF00234FF09043B74213601161C2F808E0F1D163
:20C8800005F15003354963440027FF2651F8042F1568002DACBF00254FF0904599421560C4
:20C8A00017619660F2D1036914F88D1C43F480730129036160D054F8842C294800239361BA
:20C8C00000294FF0FF336FF0804151615360516114BF00231023906143F470139069D4F8EE
:20C8E000581543F4605343F00803034393619368096843F00103936088471A4B1A4ADA6001
:20C9000068461A4B0093FDF723FB02B0BDE8F08100E100E00038024000000240305E00206C
:20C920005C040020080401004000400100080050000B00502009005040090050200B0050A9
:20C94000003C0140C00500500010005000300050AC5D0020A05D0020B45D0020F05D002081
:20C960000008008000ED00E00005FA0543020001000900502005005054F8842C144B036389
:20C980006FF08041134D00234FF0FF30936151615060516195619FE701680F4A0F4E41F0B2
:20C9A00003010160802159629E62C3F80421E022C3F80821C0F24002C3F80C2135E79A68F6
:20C9C00022F03E0141F02A0161F307029A6014E70301810000080080A000400080002000CB
:20C9E00010B5194C94F86505B8B9184B83F85100586594F86835012B05D0022B20D0D4F8A7
:20CA00006C351BB910BD124BC4F86C3511495B68BDE81040A1F10C00184744F0C7FA94F88A
:20CA200067250A49003A18BF012281F8512048650028DED01F22C280202143F06DF8D8E75B
:20CA4000054BC4F86C35E1E7305E0020501A00209C040020A06300207804002099B10A6BEB
:20CA6000824216D9154BD3F8AC25914221D34C3991421ED30B6B9842F9D38B6B9842F6D83D
:20CA80000B46184670470D4BD3F8AC150A6B904212D30B680BB9F4E70A6B90420B4602D3A1
:20CAA0008A6B9042EDD951F84C3F002BF4D1184670470023184670470A46D8E7305E00201B
:20CAC0002DE9F047CC0143D10346224A43F8082B4FF0FF324260022418467E26DFF87880FC
:20CAE000D8F8B0952644013E051D49466FF070474FF0010A08E0A3421CD0631C45F8043CB2
:20CB0000321B1C460435CAB10B6BA34202D88B6BA34204D22046FFF7A1FF014690B10A79C5
:20CB20004B6B002AE7D1A34204D0E6D245F8042C631CE5E745F8047C631CE1E7C8F8B015AB
:20CB4000BDE8F08745F804AC321B631C4946D8E78026C3E7F8FFFF0F305E002070B44479CE
:20CB600041BB03684FF400524FF40076202502213CBB1A8C22F001021204120C1A841A8B6F
:20CB8000188C22F0F30280B2120420F00A00120C014342F0010241F001011A8319841A8BDF
:20CBA00022F00C021204120C1A831A8B92B270BC1A83704700220368164615461146002C54
:20CBC000D7D0042C21D0082C38D0198C21F480510904090C19849C8B1D8C45F6FF7040F657
:20CBE000FF4128402140024342F4805241F4807199831A849A8B22F440621204120C9A83D1
:20CC00009A8B92B270BC9A8370471A8C22F010021204120C1A84188B198C89B240F6FF4215
:20CC200021F0A00102400D4342F4807245F010051A831D841A8B22F44062B3E71A8C22F44D
:20CC400080721204120C1A84998B1A8C21F0F30192B2090422F42062090C324342F48072A6
:20CC600041F0010199831A849A8B22F00C02C4E738B50E4D0446006807F002FFD5F83025C3
:20CC8000204652084FF6FF7140F06EFD20460021FFF764FF064BC5F89C3D05F69C5120466F
:20CCA0000022BDE8384040F06DBC00BF482B0020910E0208036870B55E6A26B13346052212
:20CCC000BDE87040184704460D464E1D00E023689B68204698470028F9D0236815F8011B40
:20CCE0001B6820469847B542F1D170BD0A44914217D010B40139541E11F8013F0822584003
:20CD0000430010F0800F08BF400083F0D50314BFD8B2C0B2013AF3D1A142EDD15DF8044BDC
:20CD2000704770472DE9F047164D0746002095F9BD9505F2C45684B007EB010805F66405E4
:20CD400004464FF0B60A3368ABB193F83830142B11D019F1020F01D04B450CD10022694656
:20CD60003046CDE90244CDE90078ADF808A08DF80D4034F08BFAE036B542E4D104B0BDE830
:20CD8000F08700BF305E00202DE9F0479AB0DDE9226ADDF8909004460D461746984602E017
:20CDA000206844F06DF8206844F072F80028F7D10146642201A860F08AFE264B8DF80450A4
:20CDC000CDF85CA00293002D40D0AB1E012B3FD9042D14BF002203221F4B0396D3F88430E6
:20CDE0008DF805201E440123CDE9059404968DF85B3037B14246394607A860F007FE8DF892
:20CE00005A80164E96F8A69800231893B9F1000F19D196F8A508642202FB006001A900F6D9
:20CE2000A80060F0F3FD012386F8A59886F8A638236843B143463A46294620461AB0BDE803
:20CE4000F04712F01FBC1AB0BDE8F0870522C3E70222C1E794660020482B0020305E0020E0
:20CE60000C480D4BD0F8281910B40C4CC0F818398A1E2231B0F846391B01A4FB03C3DB0852
:20CE8000A3F5B06322F8023F9142F3D15DF8044B704700BF305E002039810208CDCCCCCC38
:20CEA00070B5084C251D2E4614F8010B34F056FC28B1037805F8013BB442F5D170BDFF231D
:20CEC000F8E700BF9C6700202DE9F0471D4F012607F10805B2464FF03C094FF0000817F8DA
:20CEE000010B44F063F8044690B180F80690C671FB7803F07F02012A18D013F0800F2046D5
:20CF00000DD185F8048044F035FB85F805802C600136052E05F10805E1D1BDE8F08785F888
:20CF200004A044F02DFB85F805A0F0E71B0605D40121204642F0F0FDFB78DEE744F020FBD0
:20CF4000F6E700BFA46700202DE9F04FDFF8FC91DFF8FCA183B009F10C06012419F8018BDC
:20CF6000B8F1000F00F0C6804FEA1815013D042D08F00F0200F2C1800AEB4503B3F8840046
:20CF800040FA02F717F0010700F0D28001239340013B184055445EF0A1FA95F89030664FFE
:20CFA000184407EBC00704237761FC71BB71002302E0152B00F09E8003EB43025F49895CB1
:20CFC00041454FEA430B03F10103F2D15C4B1A4492F84512002900F0AD80404640F026FD84
:20CFE0000546284640F042FD0378002B40F08280534B5B44042283F8854283F88422002D3E
:20D0000078D0002F5DD03B68287A03F13F4202F57E020AEB92224FF0010C92F8982002F012
:20D020001F015209032A0CFA01F171D0042A67D0022A75D0B7F804E0BEFA8EF2C2F11F029A
:20D04000C2F3CC0103EB810102F007020F6A92004FF00F0C0CFA02FC27EA0C070F620F6A6C
:20D0600090403843002208624FF0010B11460BFA01FC3CEA0E0001F101011ED11868032774
:20D08000974020EA07001860D3F800800220904040EA08001860986820EA07009860986840
:20D0A0009860586820EA0C00586058685860D86820EA0700D860D868D860102902F1020241
:20D0C000D5D1204B204AB3F89C19B3F89E390091002001340190B2FBF3F330469BB22946B7
:20D0E000E4B232F01BFE0123092C737406F118067FF434AF03B0BDE8F08F0027776156E7A1
:20D10000DFF850C0DCF830200A43CCF8302091E7DFF840C0DCF840201143CCF8401089E748
:20D12000DFF830C0DCF844201143CCF8441081E777613CE70D4654E7F82D00208C2D002075
:20D14000482B0020305E002040420F00D067002070DB0608003802402DE9F041214E224FAC
:20D1600096F86F3A87F8083F06F66C2607F60C7500244FF0050816F8010B20BB2860013484
:20D18000032C05F10405F6D197F8081FD7F80C0FC94301F0010144F0F9F997F8081FD7F850
:20D1A000100F81F00201C1F3400144F0EFF997F8081FD7F8140F81F00401BDE8F041C1F323
:20D1C000800144F0E3B943F0F1FE013401212860E3B210B180F80680C371286842F09CFC1B
:20D1E000CEE700BF305E0020482B00202DE9F0412A4C2B4DB4F8746AA5F8186F82B0EEB9BE
:20D2000094F8700A43F0D2FE94F8712AC5F81C0F003A18BF012285F81A2F48B194F8721AEB
:20D220002B22002914BF11210121C28042F074FC002002B0BDE8F04144F0B0B994F8708AA2
:20D24000002240462B2140F049FC0746404643F0ADFEF8B1F7B12B22C5F8340FC280397A21
:20D26000FCF7B6FE4FF000080E4AB2FBF6F3C3F34F0000909BB23946CDF8048005F572605C
:20D28000A4F8766A32F04AFDD5F8203FC3F8008085F8318F02B0BDE8F08100BF305E0020D0
:20D2A000482B002040420F002DE9F84F254C94F8843A84F8783A04F67B27002604F698248C
:20D2C0005FFA86FB0BF101085FFA88F8012117F8010F42460E448A4640F000FC4FF0000937
:20D2E000054640B3387804F80E9C04F80D9C04F80FBC04F810AC44F8045C43F057FE18B189
:20D3000080F806A080F80780297AFCF761FE0E4A0021284640F028FA0C4B23600C4B221D52
:20D3200021462846C4E9013940F02CF9697928684A4632F06FFC082E04F11C04C0D1BDE8CC
:20D34000F88F00BF305E002040420F004DFC030885DE030870B52C4C2C4B94F8B00BC4F86F
:20D36000A83B00220221C4F8682BC4F86C2BC4F8702BC4F8A42BA4F8AC2B40F0AFFB00288C
:20D3800041D0234B0268054603F1C000597C11B159688A422BD018338342F7D1002394F8FF
:20D3A000B00BC4F8945A84F8883A43F0FFFD08B10223C380297AFCF70BFE2846154A0021ED
:20D3C00040F0D2F9144A1549C4F8981A0026111F2846134BC4F89C3AC4F8A06A40F0D2F8B4
:20D3E000697928683246BDE8704032F013BC138D0C490D4A9BB2D2F830250133B2FBF3F37E
:20D4000081F82833CAE770BD305E002000FFFF00CC2C002040420F00CC680020ADDE03081B
:20D4200049E0030898010020482B00202DE9F04FC14FC24C85B08B460546C02207F5C27098
:20D440000021CDF808B060F042FB94F81C3C002B00F0DA8094F81D3C002B00F0F48097F845
:20D460007031012B67D0022B00F0F980B44BB54E03931D460FCE0FC50FCE0FC597F866C1FF
:20D4800097F8623196E80700AF4EC4F8006CBCF1000618BF0126072B85E8070084F8256C5C
:20D4A00000F22A81042B00F26381DFF8C0A20026AAF1120B029BB3424FF0030139DD1BF8B5
:20D4C000019B07EB090309F1010893F867515FFA88F82846424640F001FB034628461D4657
:20D4E000002B00F0218143F061FDCAF8140020B14FF00303837180F8078097F8632197F85D
:20D500006231F1B2002A00F00D81EA7982F00102009228464A46013658F0DAFC002800F058
:20D5200003814FF00103082E8AF811300AF1180AC0D1039B66E0854E029BC4F8283C0FCE2C
:20D54000834DDFF828920FC50FCE0FC596E8070097F8663197F8626184F8686C00269B1BBC
:20D5600085E8070018BF012305F1980031464FF44C7284F8253C84F8266C60F0A8FAA9F1BF
:20D58000120305F57275B2460393D4F8283C534540F3AA80039A12F8013B03923B4493F860
:20D5A0006761304642F060F98046304643F0FEFC97F863310646002B00F0988098F80730D0
:20D5C00083F0010B0BF0010894F8252C08F1010884F8248C0AB18BF0010B002E00F093804A
:20D5E000B279002A59D0412A57D05A4B5A495B4AC4F8D03B012384F8263CC4F8CC1BC4F806
:20D60000D82B0023C4F8203CD4F8203C63B10022029883F82C00012183F82D101A6383F85B
:20D620002E2005B0BDE8F08F4D4E4E4D0FCE0FC50FCE0FC596E80700A5F1200385E8070079
:20D64000C4F8203CEDE797F864210299003A284618BF0122FBF740FAC4F8200CD4E797F82F
:20D660006631002B3FF402AF97F86231082B7FF462AF344EDFF8D0C00FCE04F6E8350395B6
:20D680000FC50FCE0FC596E80700012385E8070084F8253CC4F800CC31E0304643F0D4FFF6
:20D6A0004FEA48180AF1010A48F009014FF0030369616860EE6085F810B086F807A0B371DE
:20D6C000304642F029FA1BF0010F304611D043F051FFEB68C9F81430BAF1080F05F1200555
:20D6E00009F118097FF451AF194B8BE798F807B068E743F045FFECE7082B7FF4D6AE1A4B57
:20D70000C4F82C3CD1E6304643F09EFF4FEA481848F009010AF1010A69616860EE6085F8AA
:20D7200010B0CDE7EA79F3E60C4B0A4AC4F80C3CC4F8042C002365E7482B0020305E0020EE
:20D74000186A002060DC0608D93706088CDC0608E46900207DE0040881E0040875E00408A5
:20D7600034DC0608646A002015E10408CC2C002097F86531064AC4F82C2C012B05D0022BCC
:20D7800006BFBCFA8CF35B09002384F8303C8CE645E104082DE9F0416E4F97F8400997F811
:20D7A000415943F003FC60B12D23C3802021044642F0B2F90A2042F0DFFD204643F03AFF87
:20D7C00028B9DFF8988158F85C3CDA0001D5BDE8F081013D092DFAD897F83F49D4B9402080
:20D7E0003DF0A0F80028F2D090F9043097F81119092BC8BF143B43440A2913F8584C00F0A1
:20D800009B8013F84C3C97F83E29002A08BF1C46002CDCD0204643F0C9FB0546002800F079
:20D8200083802D23C380012142F076F90121084643F0E6FE2B68AA881A833C2042F0BAFE60
:20D840000021012043F0DCFE97F84139002B4CD0414C00261FE02B68AA885A8342F08CFD1A
:20D8600094F8081FD4F80C0F01F0010143F08EFE94F8081FD4F8140FC1F3800143F086FECE
:20D880002B68AA881A83782042F076FD97F8413901369E4229DA94F8081FD4F80C0FC94320
:20D8A00001F0010143F072FE94F8081FD4F8140F81F00401C1F3800143F068FE7820002D27
:20D8C000C9D1782042F058FD94F8081FD4F80C0F01F0010143F05AFE94F8081FD4F8140FD5
:20D8E000C1F3800143F052FECDE797F83F399BB9D7F8403903F0FF13B3F5803F7FF467AF24
:20D9000058F85C3C13F080537FF461AF87F84139BDE8F0414BF030BB322042F04BFE284696
:20D92000002142F0F9F8E3E7012142F0F5F80121084643F065FE80E758F8343C5B057FF597
:20D9400046AF09F0FBFC00287FF441AF002C7FF461AF3CE7305E0020482B0020286F00208D
:20D96000084B53E90C02904253F8283C02DC114602460846984204DD9A42B8BF1A461046FA
:20D9800070477047286F00200B6810B414681B1B036054684B681B1B43608B6892685DF88C
:20D9A000044B9B1A836070472DE9F047041E0D4612DB092C26DC824A0B468248A0FB04104D
:20D9C000C00800EB8000A4EB40000021125C1A7059702846BDE8F08764422D23092C01F8B5
:20D9E000013B24D8764A774BA3FB0403DB0803EB8303A4EB43030020D35C48700B702846AC
:20DA0000BDE8F0876F4B632CA3FB04264FEAD60621DC6B4A0B466B49A1FB0601C90801EBAD
:20DA20008101A6EB4101515C03F8011BC5E7654A632CA2FB04364FEAD60637D8604A614B92
:20DA4000A3FB0603DB0803EB8303A6EB4303D35C01F8013BC7E7A3FB0627B4F57A7F4FEA39
:20DA6000D7070DD2564A0B465649A1FB0701C90801EB8101A7EB4101515C03F8011BCAE72D
:20DA8000A3FB072842F20F7294424FEAD80836D84B4A0B464B49A1FB0801C90801EB8101A9
:20DAA000A8EB4101515C03F8011BDDE7A2FB0637B4F57A7F4FEAD7070CD2414A414BA3FBE3
:20DAC0000703DB0803EB8303A7EB4303D35C01F8013BB4E7A2FB073842F20F739C424FEA65
:20DAE000D80821D8364A374BA3FB0803DB0803EB8303A8EB4303D35C01F8013BDEE7324ACD
:20DB0000A3FB080994424FEAD90921D82C4A0B462C49A1FB0901C90801EB8101A9EB410175
:20DB2000515C03F8011BB5E7274BA2FB08099C424FEAD90921D8224A224BA3FB0903DB080D
:20DB400003EB8303A9EB4303D35C01F8013BCAE71E4AA3FB090394424FEAD30A21D80B461A
:20DB60001849174AA1FB0A01C90801EB8101AAEB4101515C03F8011BCAE7144BA2FB0902AA
:20DB80009C424FEAD20A13D80E4B0D4AA3FB0A03DB0803EB8303AAEB4303D35C01F8013BB6
:20DBA000CAE70A22BAFBF2F04AF0D6FF0346D7E70A22BAFBF2F04AF0CFFF0146E4E700BF3F
:20DBC0001C5E0708CDCCCCCC9F8601003F420F0070B4334810F8243CA3F13001092956D8A9
:20DBE000A0F124042246153812F8015FA5F13001092904D88242F7D1002070BC7047141BBA
:20DC0000022C4ADD2748002101E010F8013B01EB810103EB4103161A303B022E044603F052
:20DC2000FF01F2DC204B03FB01F1A2424FF000030DD903EB830314F8016B5B00303B334486
:20DC4000A24203F0FF03F4D1184800FB03F32E2D06D01748A0FB032301EB930070BC704722
:20DC6000013204200024157804EB8404303D6400092D00F1FF30A4B202D82C44A4B20132D5
:20DC800010F0FF00EFD1642202FB0433E1E700211D46A0F124020B46D9E7064C0021C4E7D9
:20DCA000286F0020056F00208096980040420F00ABAAAAAA046F002038B504460D460A46C4
:20DCC0000068FF215FF003FF21682944216038BD83B50C46164605463BF0D0F820463BF04A
:20DCE000CDF80021204B0846002E08BF1E4643F087FC0021012043F083FC284643F0C8F821
:20DD0000B0B10121002043F07BFC284643F0B8F80746204643F0B8F80028FAD039462046F8
:20DD200043F0BAF83846B0470021084643F068FC204643F0ADF80028DFD00121002043F0F9
:20DD40005FFC204643F09CF801462846019143F09BF801990028F8D0284643F09DF800214D
:20DD6000084643F04DFCC8E7794C0408F0B50023C1E90033C1E902330B610268DFF888C0E0
:20DD800089B004ADC2F385572E4647FA03F0C007344604D513F80C0004F8010B2646013387
:20DDA000062BF2D1164CDFF864C0C2F303200023205C33708DF81800C2F305370DF119064D
:20DDC00047FA03F0C007344604D513F80C0004F8010B26460133062BF2D100233370C2F3C7
:20DDE000834406ABCDE90134084602F00F0305490095C2F303124DF0F9FA09B0F0BD00BF6C
:20DE00005C5E0708445E0708645E0708545E070870B5094C54F8142C054662B1002654F820
:20DE2000140C2D21013644F0AFFCAE42F7DBBDE8704049F085BB70BD286F00202DE9F04F95
:20DE40005FFA81F9002185B007460846164643F0D7FB0021012043F0D3FB43F047F8022EB8
:20DE60000AD0042E44F6C01818BF4FF49648B9F1070F07D900200CE0B9F1FF0F4FF4164887
:20DE8000F5D10326BE4D15F8103C2BB9002045F80C0C05B0BDE8F08F032EBA4C0DD0A14404
:20DEA000002299F8670103213FF018FE0028EDD0C4F87805C3799A07E8D415F8100C84F882
:20DEC000936D002203213FF009FEC4F87C090028DCD0AD4AAD4BC4F8343502F1480003233C
:20DEE0004FF48061A4F83835C4F84805002302F24C404FF0010A032EC4F83C85C4F8603500
:20DF0000C4F84015C4F85435C4F85035C4F84C05C4F84415C4F85C35C4F8583584F8843D75
:20DF2000A4F880ADC4F88C3DA4F8903D84F8923D91460ED0D4F878B59BF8040043F036F839
:20DF4000C4F87405584614F0D9FB5146484614F0E9FB322042F02EFB012E09D1D4F87C0902
:20DF60004146FAF7ABFFD4F87805FEF781FE0AE0022E3BD1D4F8780514F0AFFBD4F87C0954
:20DF80004146FAF79BFF45F80C9C4FF0060A022E11D055F80C0C42F07BFF60B101210020C6
:20DFA00043F02EFB55F80C0C42F072FF014600287FD143F025FB384642F06AFF80B101217F
:20DFC000084643F01DFB4FF0050B4FF00008384642F05EFF0146002874D1012043F010FBF2
:20DFE000042ED6D0052042F0E5FAD0E7032E58D14FF0000A5146664884F894AD40225FF006
:020000040800F2
:20E0000066FD8DF80FA04FF0010A9DF80F30072B09D95D48012114F085FBD4F87C09414614
:20E02000FAF74CFFAFE79DF80F3003EB430304EBC30393F895316BB39DF80F3003EB4303DA
:20E0400004EBC303D3F8983123B39DF80F30234493F86701F0B1002203213FF03FFD834658
:20E06000C0B114F03AFB9DF80F3094F8942D03EB430304EBC30305EBC201D3F8983141F86C
:20E08000083C9BF807300132DB0748BF01F804AC84F8942D9DF80F300133DBB28DF80F3017
:20E0A000B3E7042E7FF46FAFD4F8780514F015FB54E755F80C0C42F0E3FE0146384642F0FC
:20E0C000EBFE6FE7384642F0DBFE95F8463001468BB9242803D14FF0010385F84630012E65
:20E0E00004D13846019142F0D7FE019955F80C0C42F0D2FE6BE7012B06D14D280CBF022379
:20E10000002385F84630EAE7022B06D13C280CBF0323002385F84630E1E7032B10D10A28A0
:20E1200002D985F84680DAE7042385F8390085F8388085F83B8085F83A0085F84630CEE757
:20E14000042B09D195F83A3085F84700434085F83A3085F846B0C2E7052BC0D195F83830BF
:20E1600095F8399095F83A004B4513D25A1C2B44484085F83A0085F8382083F83C10AEE7B8
:20E18000286F0020482B00207C300020B8DC0608206F00208842C4D195F8473085F846A052
:20E1A000F42B9CD1B9F1000F99D12421384685F8469042F071FE4D21384642F06DFE3E2111
:20E1C000384642F069FE4946384642F065FEF421384642F061FEF421384642F05DFE032E11
:20E1E0001BD0D4F87805437901689D080223AB40DB439BB20B828D892B408B8100792021D2
:20E2000014F05AFAD4F878054A4649463FF0BAF9D4F87835186806F033FC0022D4F87C09CB
:20E2200011463FF0AFF9D4F87C39186806F028FC01202EE630B583B04D1C009303688572EA
:20E24000C2729C690023A04703B030BD03685B6C0BB102211847704770B51C4C0968E56C65
:20E260001B4EA46CD6EDCB7ADFED1A6A491B00EE901A0168F8EEE00A091B60EEA70A00EE87
:20E28000101A20EEA07AB8EEC00A1C46A0EE007AB1EE400AF1EEC77A67EEA67AFCEEE77A89
:20E2A000C2ED007A4DF038FD9FED0B7ADFED0B7AE0EE077AFDEEE77A17EE902A002ABCBF62
:20E2C00002F50C42A032226070BD00BF286F0020980100202C7D8E3FA00CB34500A00C463D
:20E2E00038B50F4C94F8671001F03F018B1C024601F10A0584F8653084F8625004F160001E
:20E3000084F8632008311EF079FD254485F85E0094F862301C44000A84F85F0038BD00BFE6
:20E32000286F002038B50B4C00250122802120463CF0E4FA30B194F904003CF011FB08B126
:20E34000006838BD0135062D04F10C04EDD10020F7E700BFB06F002038B5041F00F108052A
:20E3600054F8043FD81780EA430016F04FF9A542F6D138BDF8B5C94CDFEDC97A94ED357A80
:20E3800094F83C31B4F83E712DED028BB8EE478A28EE278A002B5FD1D4F8483194F859219E
:20E3A000002B40F30E8107EE902A9FEDBE6ADFEDBE6AF8EEE77AB7EE007AA7EE867AF0EE40
:20E3C000477A07EE103AF8EEC78AB7EE087A87EE270AC6EEA87A20EE270A5EF073F80F2834
:20E3E000B8BF0F2094F83D3185B2A4F83E51002B00F04781AF4234D0B4F840319FEDAB6A85
:20E4000094F8D86007EE103A07EE905AB8EE477AF8EE677AC6EE076A86EE277A76EE887A4C
:20E4200037EE087AC8EE276AC8EE077AB6B394F84231B4F84451C4ED3A7AC4ED3E7AC4ED8F
:20E44000427AC4ED466AC4ED4A7AC4ED4E7A002B5BD0BDEC028BF8BD94F83D31002B00F05B
:20E46000858094F8D860002E40F00381B4F84031DFED8E6A07EE907A07EE103AB8EE676A5B
:20E48000B8EE477AC6EE877A86EE867A77EE887A37EE087AC8EE276AC8EE077A94F8426131
:20E4A000B4F844510023C4F8DC30C4F8E030C4F8E430C4F8EC30C4F8F030C4F8F430C4F844
:20E4C000FC30C4F80031C4F80431C4ED3A7AC4ED3E7AC4ED427AC4ED466AC4ED4A7AC4ED70
:20E4E0004E7AC4F80C31C4F81031C4F81431C4F81C31C4F82031C4F82431C4F82C31C4F861
:20E500003031C4F83431002E66D1D4F8483194F85921002B40F38E8007EE902A9FED616A57
:20E52000DFED616AF8EEE77AB7EE007AA7EE867A07EE903AF8EEE77AB7EE086A86EE070AA7
:20E5400086EEA77A20EE070A5DF0BCFF0F28B8BF0F2080B2A4F84401002E3CD0A8423FF4B8
:20E5600078AF00286DD1BDEC028BF8BDD4F8483194F85A21002B40F3878007EE903AF8EECD
:20E58000E78A3D4607EE902A9FED466ADFED466AF8EEE77AB7EE007AA7EE867AF0EE477A86
:20E5A000B7EE087A87EE270AC6EEA87A20EE270A5DF088FF0F28B8BF0F2080B2A4F84001B9
:20E5C00018E794F83D310F25A4F83E51002B7FF411AF2846F2E7054694F8583184F8953499
:20E5E000002D3FF436AF07EE905A9FED306AD4ED576A2F4BF8EE677ABDEC028B86EE277AC3
:20E600001946002241F8042B012084F894040A609A601A615A619A611A625A629A6237EEEE
:20E62000267AC6EE877AC3ED037AC3ED077AC3ED0B7AF8BD0F20A4F8440146B30F2D3FF4C5
:20E6400008AF07EE900A9FED196AD4ED576A194AF8EE677ABDEC028B86EE277A37EE267AA9
:20E66000C6EE877AC2ED007AC2ED087AC2ED047AF8BD94F84231B4F84451002B7FF4E9AE34
:20E6800043E794F85A217DE73D460F2096E794F8583184F895340546A5E700BF286F00200F
:20E6A000BD378635CDCCCC3D002474494E2DA63D8C730020987300201D4911F8242CA2B36C
:20E6C000F0B4002605463346304637461BB911F8244C2D2C23D02E2A19D0CA1800EB800092
:20E6E00012F8244CA4F13002092A4FEA40009CBFA0F13002A0180E2B14D80133CA1812F812
:20E70000242C002AE2D106B14042F0BC70470133002DF8D0CA182A4402F8247CDDE7012335
:20E720001E46EBE70020F0BC70470020704700BF286F00202DE9F0410C4F0124A02318250C
:20E74000E6B2FF2B0BDCC5F11B0103F10108D7F8E804DBB23246C9B2FFF76CFD4346013DE0
:20E76000EFD10134052CEAD1BDE8F081286F00201FB503AC8DF80C30009400238DF80D302E
:20E780000DF0B8FB04B010BDF8B50546262027F093F9154C014610BBD4F8EC0490F8383048
:20E7A0001E3B012B02D894F8F9340BB142F074FB0E4F0026AE420ADBB4F81A350133A4F8C1
:20E7C0001A350B4BD3F88430C4F82C35F8BD17F8011BD4F8EC0442F05FFB0136EAE70023A5
:20E7E00084F82835EDE700BF286F002022740020482B002010B58021044604F0E1FF2046C3
:20E80000002104F0DDFF2046BDE8104005F018BB2DE9F041B14C94F84335C4F8300582B079
:20E8200088465A2B00F2B980DFE813F0CC00B700B700DC00B700B700B700B700B700B70030
:20E84000B700B700B700B700B700B700B700B7000F01B700B700B700B700B700B700B700EF
:20E8600033017400B700B7007400B700B700B700B700B801B7006201B700B7007C00B700BE
:20E880000902B700B700B700B7005B00B700B700B700B700B700B700B700B700B700B70010
:20E8A000B700B700B700B700B700B700B700B700B700B700B700B700B700B700B700B700E8
:20E8C000B700B700B700B700B700B700B700B700B700B700B700B700B700B700B700B700C8
:20E8E000E40194F844359B0700F16982B4F84A35D4F84525D4F884155BBA9BB212BAD018D4
:20E900008842C4F89035C4F88C2503D904F018FF002854DB0020A4F87C050546284602B059
:20E92000BDE8F08194F88835002B40F0FF8094F94035002B31DAD4F8783508469B689847BD
:20E94000002840F01E82B4F84A05D4F84525D4F8843540BA80B212BA15189D42C4F89005B4
:20E96000C4F88C2507D904F0EBFE002827DBD4F88C25D4F89005D4F88035D4F83C6503FB79
:20E9800000F003FB02F20225B042C4F88C25C4F8900584F8885500F0CF8094F854355A1C9B
:20E9A000D2B204EBC30305204FF40051042A84F8542583F85805C3F85C1500F0A0814FF0EE
:20E9C000FF35ABE7D4F83C35002BE6D1D4F8783508469B6898470546002840F0D281A4F817
:20E9E0007C059BE73E4B002203F1120103F8012F8B42FBD13B4994F87E3594F85405702561
:20EA00000D7098424FF00C05CD7110D004EBC300013390F858558D70B0F85C05DBB2042B54
:20EA200040BA888114BF84F87E3584F87E2594F8473512229342A4F87C2598BFA4F87C35C0
:20EA40000025284602B0BDE8F08194F84435DA0700F13E81D4F8783594F84705DA6901EB45
:20EA6000C10102EB81010A79531D834228BF0346A4F87C35002BE3D0013B1A489BB2013333
:20EA80001944034411F8012D03F8012D8342F9D1D6E7154E154F35460823073EC5F10700B7
:20EAA000A4F87C35002202E092F880211D462B46B54203F8012900EB030217FA82F2F3D1B1
:20EAC000D4F878354046DB6898470028B8D0AB7863F07F03AB70002520E700BF286F0020B0
:20EAE00047970020489700204F97002070DB0608D4F87835C74A5B680846111D98470546C7
:20EB0000002840F03E81D4F88435C34AD4F88015013B180E1070180C09BAD37050701B0AFA
:20EB2000082093705160A4F87C05F7E6D4F89065D4F88C25D4F88035D4F87855B2FBF3F215
:20EB40004FF48057BE4228BF3E462D69B249A4F87C754046B6FBF3F39BB2A8470028C0F2DF
:20EB6000BC803346AC4AD4F83005812104F05CFED4F88C25D4F89005D4F89C353244851B68
:20EB80009E1BC4F88C25C4F89055C4F89C65002D7FF456AF032384F88835BFE69E4E002735
:20EBA000334606F10C0203F8017B9A42FBD1D4F8783540465B686A4601A99847054600284A
:20EBC00040F0E980019BBDF80020013B190E52BAF3713171190C1B0A71710820B37102211B
:20EBE00072810C23BDF80220F07031727272A4F87C3593E6894E8A4F30460823073EC0F128
:20EC00000705A4F87C35002202E092F8882118460346864203F8012905EB030217FA82F256
:20EC2000F3D1D4F878354046DB68984700283FF407AFF37863F07F03F37000256EE694F836
:20EC40008835002B61D194F94035002BFFF6A5AED4F8783508469B689847002840F0918013
:20EC6000D4F878354046DB6898470546002840F0BA80B4F84A35D4F84525D4F884155BBABB
:20EC80009BB212BAD0188842C4F89035C4F88C2500F29F80D4F88015D4F83C0503FB01F34A
:20ECA00002FB01F28342C4F88C25C4F890357FF474AEB3F5805F28BF4FF480530121D4F8AA
:20ECC0003005554A84F888159BB204F0D7FE25E607235449A4F87C35CEE694F854355A1CD3
:20ECE000D2B204EBC30304204FF48851824284F8542583F85805C3F85C157FF460AE00233A
:20ED000084F854354FF0FF3508E6D4F89065D4F87805D4F88035D4F88C254569B2FBF3F245
:20ED2000B6F5805F28BF4FF480560846B6FBF3F339499BB2A847002862DBD4F88C25D4F8F8
:20ED40009055D4F89C353244AD1B9B1BC4F88C25C4F89055C4F89C352DB9D4F8300529464C
:20ED600004F0E0FEDAE5B5F5805F28BF4FF48055ABB2D4F83005284A012104F07FFE0025F2
:20ED8000CCE594F854355A1CD2B204EBC30302204FF468510AE694F8543504EBC3020133F3
:20EDA000DBB202204FF46851042B82F85805C2F85C1522D084F854354FF0FF35AEE594F8EE
:20EDC00054355A1CD2B204EBC30305204FF41051ECE504F0B5FC0028FFF6F1ADD4F88C2584
:20EDE000D4F8903556E794F854355A1CD2B204EBC30302204FF41C51D8E584F85475DEE5EA
:20EE000094F854355A1CD2B204EBC30304204FF440716BE7A8740020489700204F97002083
:20EE200070DB0608E8DC060810B51C2042F0BEF81121044640F070FE204642F09BFBC8208E
:20EE400041F0B8FB2046BDE8104042F099BB00BF08B5002042F0AAF8054BC3F8A40508B110
:20EE60002A23C380BDE80840402140F055BE00BF286F00202DE9F04FB34C54F8843C5A69D8
:20EE8000D2078BB002D50BB0BDE8F08F5A699B6912EA030AF7D0CAF307431AF4002F00933A
:20EEA00040F00281009B5D0743D41AF0020F5FFA8AF503D054F8843C02225A61BAF1000F1E
:20EEC000C0F20C821AF4006FCAF3072740F082812E0708D59D4B9E48D3F83C33984754F812
:20EEE000843C08225A61ED0600F1E481F80600F1A481B90600F12E81009BDA0609D5934B7A
:20EF00009348D3F84C33984754F8843C4FF480125A61009B9B06B6D58C4B8D48D3F8503390
:20EF2000984754F8843C4FF400125A610BB0BDE8F08F54F8802C9369D26913401FFA83FBDE
:20EF4000BBF1000FB1D0DFF80882CDF80CA045464FF0000909E05FEA5B0B09F1010908F13B
:20EF6000040805F1280500F0D4811BF0010FF2D054F8801C5FFA89F708694A6B04EB8703E0
:20EF8000FA4053F8783CD2019B68D2B202431A40D007D3B216D54B6BD8F81820012000FA1F
:20EFA00009F023EA00034B63684B6948D3F83433012191603946984714F88D6C012E00F06F
:20EFC000F58101231A0703D5D8F8182008239360DE0603D5D8F8182010239360580603D558
:20EFE000D8F8182040239360990703D5D8F81820022393601A06AED5D5E94C60D5F82431EC
:20F00000D8F818C0311A8B42DCF8182028BF0B46033392B2B2EB930F9DD954F8802C32375C
:20F0200004EB8703CDE9019890469946B04238D2BEB3D5F8241114F88D3CD5F82821371AA8
:20F04000B94228BF394601F1030E4FEA9E0E83B98FB20337BF1059F888AC0AD0013352F804
:20F06000040BCAF800009F42F8D1D5E94C60D5F82821DCF8183008440A44B042C5F82821E7
:20F08000C5F834010AD195F81C11D8F83420012707FA01F122EA0102C8F834209BB29E4557
:20F0A000C4D3DDE9019856E754F8803C9D69DB691D402D0C3FF4F6AEA4F19006DFF88CB020
:20F0C000B046B146002708E06D0807F1010706F1040608F128083FF4E5AEEB07F4D5F9B269
:20F0E00004EB810254F8803C52F83C2C92685B691A40D007D3B218D514F88D0C726D0123DB
:20F100009842936007D11269D8F87C33C2F312029B1AC8F88C33DBF830334846984714F8A4
:20F120008D3C012B00F0508101239A0702D5726D022393601B07C7D5DBF83833484698471D
:20F14000736D08229A60BFE7305E002098010020A05D002054F8803C54F8781C9A68086827
:20F16000C2F34102022A08BF03224FF0000514BF65F30A0062F30A0008605A6842F4807255
:20F180005A6006A805F02AFD54E92120D368BD49079D6FF38D23D3608068C0F34100014422
:20F1A00091F89011032900F0CA80B749B7480126294404F88E6C81424FF0400624F88C6CDA
:20F1C00000F210810E2161F38D234FF40051D360516191E6AE4B94F88220D3F84433AD482B
:20F1E00000218DF817108DF81720984754E9212114F8863C88684FF400615161002B3FF4B6
:20F2000067AEC3077FF564AE94F88530012B7FF45FAE9DF81730032B7FF45AAEE36F9E49DE
:20F220001A6842F001021A601A6842F003021A600B6943F006030B614AE654F8802C954849
:20F2400053684FF0000823F001034146536005F023F914F88F6C414656B1904BFF2203EBCB
:20F26000860653F8045FD86BAA609E428260F8D154F8803C87484FF0FF329A614FF00112E8
:20F28000DA610B2262F3070162F30708C3F8148019611A686FF30A121A6004F0D1FD54F8F4
:20F2A000842C7B4B7B48D3F840334FF48051516198471EE654F8843C9A6922F010029A6100
:20F2C0001A6AC2F34340022802F00F0142D0062822D09A6942F010029A6107E614F8863C17
:20F2E00033B1E26F136823F0030161F30703136054F8802C66495368D1F84813654823F030
:20F3000001035360884754F8843C4FF000425A61D8E5DDF80CA0C8E501EB8101256C04EB46
:20F32000C1012E68D1F8FC02C4F83C65C2F30A1202442868C4F84005C1F8FC22C9E7002101
:20F340004FF4007004F88E1C092124F88C0C61F38D233AE747F6F0701042BAD001EB81006B
:20F36000C2F30A1204EBC00002F1030C5FEAAC0CD0F8F052D4F840E04FEA810818BF00205B
:20F3800006D00130DEF8006045F8046B8445F8D1414404EBC101D1F8F052D1F8FC02154491
:20F3A0000244C1F8F052C1F8FC2292E7B9F1000F7FF407AE94F88130042B7FF402AE3548CF
:20F3C00004F03EFD3346FDE5002F7FF4ADAE94F88120052A7FF4A8AE4846019304F030FD3E
:20F3E000019BA2E62E48A5F57401A1F51051814203D80D2161F38D23E7E62A492A4829447E
:20F40000814203D20C2161F38D23DEE62748A5F18C71A1F54341814203D80B2161F38D2375
:20F42000D3E6234923482944814203D20A2161F38D23CAE6204921482944814203D2092157
:20F4400061F38D23C1E61E48A5F1B771A1F55851814203D2082161F38D23B6E619491A4879
:20F460002944814203D2072161F38D23ADE6174917482944814234BF0621052161F38D2395
:20F48000A3E600BF70DB0608401E1BFF3F420F0098010020A05D002000ED00E0B45D0020EF
:20F4A000DFC810002013FBFE20D61300FF69180000D3CEFE40771B00C05BB3FEC091210031
:20F4C00040AC2700C01D6AFE40E13300803C36FEE09C4100704700BF704700BF704700BF71
:20F4E000704700BF2DE9F0414FF0FF35324A33482C46002304E001330B2B02F1100215D018
:20F50000917A0429F7D103F5B17100EB0111C979CF07F0D4661C116801D0A942EBD21C4622
:20F5200001330B2B0D4602F11002E9D1631C02D10120BDE8F081214D04F5B17705EB07132D
:20F540009988F1B9DFF880802601AB19D8F86C251B4916691B4A41F2186001EB4421185809
:20F560000023B047D0B1022808D141F2CC6205EB0717AB58013B0121AB50B9710020BDE833
:20F58000F081DFF8448005EB0413D8F86C2541F21860D268185826019047D6E741F2CC6286
:20F5A00005EB0717AB580321B97141F2D061013B0124AB506C54BCE714D40020F8BD0020EC
:20F5C00010BE0020E5F50008305E0020044B41F2E472995C09B90121995401225A7070476B
:20F5E000F8BD002038B5174D174B41F2D0640020285504E001300B2803F1100314D053F801
:20F600000E4C8C42F6D11C78032CF3D16AB10F4B03EB40239A4201D0FFF7D8FF00F5B1701E
:20F6200005EB00100123837138BD41F2CC6100F5B1736A5805EB03130420013298716A5062
:20F6400038BD00BFF8BD00201ED4002010BE002038B5134B00209C7B14B11D688D4205D0B1
:20F6600001300B2803F11003F5D138BD72B10D4B03EB40239A4210D0FFF7A8FF0A4B00F5F5
:20F68000B17003EB00100123837138BD064B00F5B17003EB0010827138BD022CECD1EDE732
:20F6A00010D4002010BE0020F8BD00202DE9F84F12F0020E9B4606D028B9FFF787FF0225D9
:20F6C0002846BDE8F88F804C41F638056559002D5BD14FF0FF367D4FB146B046B2460025EF
:20F6E0003B68984200F0B68097F80EC0BCF1000F5BD0BCF1010F15D105F5B17C04EB0C1C42
:20F700009CF807C01CF0010F0CD11CF07E0F09D15FEADC1340F0A880D7F808C0D44501D20F
:20F72000E246A94601350B2D07F11007D8D1751C04D1B8F1FF3F00F09F80464641F2C86841
:20F7400006F5B17754F80850013544F8085004EB061C41F21C694FEA07184CF8095044F81E
:20F76000085041F2186904EB07154FF000084CF80900C5F8048004EB0715AD79042D9CD8C7
:20F78000DFE805F01A330F334D0004F5C25741F63C063F68A65907FB0565A84299D3FFF7E8
:20F7A00015FF00252846BDE8F88F2E4601350B2D07F1100794D1BAE712F0010C70D104EB40
:20F7C0000710D51090F80780BBF1030F65F3C71880F8078062D94FF6FF7083455B4628BFEB
:20F7E00003469BB204EB07108380BEF1000F16D004EB061303F5B0531833987B04280ED05B
:20F8000041F2C8654FF0040C60590130605141F2CC65586083F80EC063590133635150073E
:20F8200005D504EB0710C37943F00103C371D30608D504EB0714E379C3F34502013262F3A0
:20F840004603E371224B012503EB46260E602846BDE8F88F05F5B17704EB07164FEA071C8C
:20F86000B67986B92E4669E7A84601350B2D07F110077FF435AF5AE7B9F1FF3F18BF4E4600
:20F880007FF45CAF8DE741F2C8682E4654F80850013544F8085044F80C506CE76346A1E715
:20F8A0000C4B0B49D3F86C350B4AD3F8088001EB46210023C04700283FF473AF04EB071485
:20F8C0000223A371FCE600BFF8BD002010D4002010BE0020305E002051F60008F0B5124D86
:20F8E0002B7841F63002022B0BBF070AC0F3D417C4B200F07F04A85883B00E4600230122A0
:20F90000384401A9FFF7D2FE01280AD12B78022B019B16BF53F8243033F8143023F07043E2
:20F92000336003B0F0BD00BFF8BD002010B5144602070B4610D50B4941F2C472581C8B58CE
:20F94000834204D305D100232360012010BDFFF73DFE2060012010BD21461846BDE8104048
:20F96000BCE700BFF8BD00202DE9F0414268C2F308030B44B3F5007F82B004460D4657D330
:20F9800090F91A30591C0AD0304A03F5B17302EB0313FF21DA796FF30002DA71817694F906
:20F9A0001B305A1C0FD0294A03F5B17302EB0313FF20DA79C2F34501013921EAE17161F3BD
:20F9C0004602DA71E0762378022B37D01F4A02F5C2531B68B5EB432F4FEA432824DC41F68A
:20F9E00048036768D6583E407342AB421CDCAB19434511D32169207E01AAFFF797FF0128EF
:20FA000012D16768236963614744019B2361A5EB0801BF1B67608D192046F8F7E1FD20B94D
:20FA20003D446560012000E0002002B0BDE8F08115444560012002B0BDE8F08161680120C6
:20FA40002944616002B0BDE8F08100BFF8BD002070B5154604460E46FFF786FF50B994F8EE
:20FA6000280028B9022384F82830C4E90B5670BD022070BD1DB12046A847012070BD012068
:20FA800070BD00BF10B4D0E9011390F91A208B4238BF0B46511C83600AD0144B02F5B1726E
:20FAA00003EB0212FF21D3796FF30003D371817690F91B305A1C0FD00C4A03F5B17302EBB0
:20FAC0000313FF24DA79C2F34501013921EAE17161F34602DA71C4760022436A5DF8044B74
:20FAE0004261426011460361B2E700BFF8BD002038B54422002111485DF0E9FF104B41F645
:20FB000002011A784FF6FF745C52022A41F2E87118BF032203F5C05041F64C055A5441F6C1
:20FB20000C0441F6010203215D5900F8181910211D519954FFF7A6FF012038BDE0D5002066
:20FB4000F8BD00202DE9F041B1F904300F2B82B00C461646054632D02846F8F765FD95F9F7
:20FB60001B80B8F1FF3F074633D02D4B41F2186203EB08118A58904211D1183303EB48234D
:20FB8000A188013109B203EB4113A18028463360F8F74AFD2060012002B0BDE8F081FFF756
:20FBA00015FD2846F8F71CFD28B100230120336002B0BDE8F081002002B0BDE8F0814FF41A
:20FBC0000071FFF7D1FE0028F5D04FF6FF73A380C2E72846F8F704FD0028E2D10FB9FFF788
:20FBE000F5FC38460023112201A9FFF75FFD0128D7D1019B0B4A9A1A48BF02F2FF12B2F51B
:20FC0000B05F4FEA622106D24FFA81F885F81B80002BB5D1C5E7FFF7D9FC019BF6E700BF07
:20FC2000F8BD002010BE002030B50446C06983B010B9012003B030BD0D460023032201A9A7
:20FC4000FFF734FD0128F5D1B4F92030002B03DAFFF7BCFC0220EDE7019A012D4FEA43118F
:20FC600002EB431303D0022D12D1E5255554A268DA612278032A04D100221A775A779A7733
:20FC8000DA77626A5A83C2F30F429A8203B030BDE268DA61EDE700BF10B50378023B012BE7
:20FCA0000446037E02D913F0060F5AD198063AD494F91A30591C0AD02D4A03F5B17302EB09
:20FCC0000313FF21DA796FF30002DA71A17694F91B305A1C0FD0264A03F5B17302EB031319
:20FCE000FF20DA79C2F34501013921EAE17161F34602DA71E076237E1B070BD51C4841F289
:20FD0000C873C35C072B01D0FFF760FC41F2C8730022C254E26A0023237084F82830FAB10D
:20FD2000BDE81040104700231249E0691A018A58904206D001330B2BBAD01A018A58904248
:20FD4000F8D10B4A03F5B17302EB0313DA79C2F34501013921EAE17161F34602DA71A7E70C
:20FD600010BD0121FFF760FF0128F9D1237E9DE7F8BD002010D4002030B1027822B190F898
:20FD800028201AB1002070470120704710B5D0E90142A242C16238BF22460321826080F8FC
:20FDA0002810FFF779FF012010BD00BF2DE9F04FDFF868918A4699F80010DAF8003002292D
:20FDC000174683B0834641F6300240F08B8059F80250DEB2A6EB030805EB1325B8444FF4F0
:20FDE00080729044BB4208F1FF38B8FBF2F875D2A844032906EB0704A4EB03040CBF802215
:20FE00004FF48072944228BF1446A8EB050366B994422CBF0A220B2201A92846FFF746FC72
:20FE2000012809D003B0BDE8F08F0B2201A92846FFF73CFC0128F5D199F80020DAF80010F4
:20FE4000022A01F1010321D0A64210D2019906F18042013A081F00EB840001EB820242F8F7
:20FE6000043F824203F10103F9D1DAF80010A61B7318BBF1010FCAF800301BD09F4205F11B
:20FE800001052BD999F800100026B2E7A642EED2DDF804C006F10042013AACF1020000EBB9
:20FEA00044000CEB420222F8023F904203F10103F9D1DCE7BB42E1D199F80030022B21D083
:20FEC00004F18044019B013C4FF0FF3243F82420DAF800309F4205F10105D3D8012003B043
:20FEE000BDE8F08F59F8022003F07F060329C3F3D415A6EB03081544B84414BF4FF480722F
:20FF000080226EE704F10044019B013C4FF6FF72584623F8142003B0BDE8F08FF8BD002089
:20FF20002DE9F04190F838300446032B51D8DFE803F002323B462D4BC0681978E76A03F500
:20FF4000C252032911680CBF80264FF4807601FB06F141F2C47C00EB412041F2A87841F206
:20FF6000AC7E53F80C20E06053F80E0053F808502261A5EB4125A0EB4121901943F8085002
:20FF800043F80E1043F80C00C4E90C205FBB6262012384F8383016480021FFF745FE012821
:20FFA00011D1022384F83830626B04F130010120FFF7FCFE012806D1032384F83830002127
:20FFC0002046FFF731FE431EDBB2012B02D9BDE8F081022094F82830062B04BF002384F8F2
:20FFE0002830BDE8F081921B2263D1E7F8BD002098D500202DE9F04FDFF8248198F8006086
:020000040801F1
:20000000012887B08CBF00230123032E02930C460B68154639D0022E62D14FF480724FEA2E
:200020001329DFB201920138012823D8012203929D421AD9384E06F1880A06F11C0B3268B2
:200040001AB1DBF8001099424ED0DAF8000000234844092205A9FFF729FB01281FD0022843
:200060000FD020B123689D42E9D82560032007B0BDE8F08F87B1FFF7A9FA022007B0BDE8D3
:20008000F08F022007B0BDE8F08F80220192C3F3D41903F07F07C6E7019A0392C8E7DDE941
:2000A00002C1059ADDF804E098F80030022B14D0032BE6D152F8273023F07043B3FA83F3E5
:2000C0005B0963450F44236823D00B4477452360EAD309F101090027C5E732F81730EDE7DC
:2000E0004FF480720192D2E70C490968013A02EB41224902B2FBF1F203991344B3FBF1F2CF
:2001000001FB12320AB10B449B1A9D42236096D8ABE7AB42ABD3A8E7A0D5002038D60020C1
:20012000F8BD0020F0B5104D2B7841F63002022B0BBF070AC0F3D417C4B200F07F04A8584D
:2001400083B00E4600230322384401A9FFF7AEFA012807D12B78022B019B0CBF23F8146045
:2001600043F8246003B0F0BDF8BD00202DE9F04390F83C30002983B0044614BF0221002191
:20018000042B7BD8DFE803F0030C3C476900FFF74BFD012870D1626B002A75D184F83C008B
:2001A000404EDFF80881404D4FF6F7771DE01FFA80F9B94594BF4FF000094FF0010901A9F6
:2001C000B9F1000F46D1FFF789FB0128494650D1206BFFF7A7FF01284BD1019B2A682363DC
:2001E000013B934228BF13462B603378206B032BDDD1404594BF4FF000094FF00109DEE7E3
:20020000426B04F130010020FFF7D0FD012833D1032384F83C30234BE16A41F2C47003F5D5
:20022000C2521D581268195041F2A87741F2AC76D8596D1A995902FB05F200EB422501EBCF
:20024000422203F5BD500021DD519A51FFF7ECFC012811D1042384F83C3094F82830042BF0
:2002600004BF002384F82830A36B8BB120469847012003B0BDE8F0830228FAD194F8283070
:20028000042B09D00220F4E7022384F83C30B8E7012003B0BDE8F083002384F828300220A8
:2002A000E7E700BFF8BD00203CD60020F7FFFF0F38B590F834300446052B46D8DFE803F07B
:2002C0001F033F101963006B4FF0FF31FFF72AFF01283AD1E06A002839D1032384F8343082
:2002E00000212046FFF7A0FC01282ED1042384F8343094F82830082B2DD0012038BD41F655
:200300003803224DEA5800F1300102320120FFF771FE012824D00238C0B2012815D805230E
:2003200084F8343094F82830082B04BF002384F8283041F2E5730122EA54022038BDC06ADF
:20034000216BFFF7EFFE0128C7D0002038BD022384F83430F4E7002384F82830012038BD6C
:2003600005F5C252E3681168D4E90B2003EB412341F644016850C4E9033002B960620123BC
:2003800084F83430A0E7014DCCE700BFF8BD00202DE9F04F436883B0C3F308081646002AE2
:2003A00000F0E180714B05468946A3F1180B4FF0000AC8F5007495F91A70B44228BF344676
:2003C000791C28462ED0F8F72FF90BEB071341F218629B58984205D0FFF7F8F8504603B077
:2003E000BDE8F08F614B03EB47202246494640445DF00CFB002221462846FFF729FBA24412
:200400000028EBD02B7E1B0706D5594B2A691B689A4201D3FFF7DAF8361BA1444FF00008A4
:20042000C7D1DBE7F8F7DCF8002849D12846F8F7FBF86968C1F308032BBB21F4FF7323F0FD
:20044000010303F50072AB689A422CBF062207222B7E03F00C030C2B1CD0002301A9FFF772
:2004600025F90128BAD10198404BC31A48BF03F2FF13B3F5B05F4FEA63224FD257B2AF76D7
:200480000028B2D1AAE72B7E03F00C030C2B4FF00702E2D19BF800C0364BBCF1030F1B682D
:2004A0000CBF4FF0800C4FF4807C03FB0CF34FEA432C0CF1FF3C0CEA0101A3EB5123CDE7DC
:2004C0002B7E1A072ED59BF800102A4B95F828201B6803290CBF80214FF4807103FB01F321
:2004E000062A4FEA43233FF479AF23490868834230D891F83D30002B7FF470AF002A7FF4D9
:200500006DAF6B6985F83820062185F82810EB622846FFF705FD012888D05FE7FFF756F87C
:200520000198ACE7154B1A78002A7FF457AF95F82820002A7FF452AF082185F8342085F810
:200540002810D3F85F206B692846C5E90B32FFF7AFFEE0E741F2E573012250460BF8032018
:2005600003B0BDE8F08F924638E700BF10BE0020BCD5002038D60020A0D50020DDD50020BA
:200580002DE9F04390F8384083B00546032C00F29F80DFE804F0021A890BFFF789FE012843
:2005A00011D002280BD1032385F838302B6C002085F82800002B00F0878098470224204660
:2005C00003B0BDE8F08385F838002B78022B77D0404A6F6841F64803D3581F40C7F34F27E7
:2005E0002846F8F721F8DFF8F08006463F1A0AE0D8F80030013B99454AD2FFF7B5F908B914
:20060000FEF7E4FF0136022201A900233046FFF74DF8BC1901281FFA84F94FF400724FF0A1
:2006200000010446CBD101985DF051FAEB694FF400712846002BDBD06B68002BD8D1019B13
:200640004FF020324FF02E0C1A605A6083F800C0C3F807204FF0100E6C6A1A625A6283F859
:2006600020C083F821C0C3F8272083F80BE0EA6B5C83C2F30F4CC4F30F4483F82BE09C82E4
:200680005A87A3F834C0D8F80030013B9945B4D3C3EBC35359022846FFF766F908B9FEF7B1
:2006A00095FF022385F838302B6C002285F8282063B1284698470124204603B0BDE8F08367
:2006C0006F68C7F34F278BE7022478E7012476E7002474E7F8BD002038D600202DE9F04FC3
:2006E00090F8303089B00446042B00F2A880DFE813F0A900B20005008A00E800B64D41F670
:200700001003EB5C002B40F09A80B44F04F11C09B84607F1380BBA4601AE32464946404678
:20072000FFF710FA012840F018810198002800F0FA800378E52B01D0002BEED1A84A821AC8
:2007400048BF02F2FF12B2F5B05F4FEA622380F03C811B01A34A13449A7B042A0CD041F23A
:20076000C86104266A5801326A5041F2CC615A609E736B5801336B5041F60202AB565E1CE4
:2007800009D003F5B17305EB0313FF26D979AE546FF30001D97141F603016B565A1C0ED0E8
:2007A00003F5B17305EB0313FF26DA796E54C2F34501013921EAE17161F34602DA71202222
:2007C00000215DF084F92346019A53F8311F58685060116019899B7A93721181019B627EE4
:2007E000DA7205A848F0E2F9BDF81430002B40F02F8144F28172019903200A82CB810A839E
:20080000CB8284F83000237E980600F1A9802046FFF738F92369002B00F0AE80237E03F090
:20082000F70213F00403227640F0B480122A00F0BA80002384F828302046E36A984709B011
:20084000BDE8F08F6548FFF71DF94FF6FF720123228484F83030614F04F11C0801AE04F1F2
:200860003109324641463846FFF76CF901282FD00228E4D1584D41F60202AB56591C09D030
:2008800003F5B17305EB0313FF20D979A8546FF30001D97141F603016B565F1C0ED003F5CF
:2008A000B17305EB0313FF20DA796854C2F34501013921EAE17161F34602DA71042384F8C4
:2008C00030300020E36A2070984709B0BDE8F08F019D0B2249462846002D00F087802B7870
:2008E000002B00F0838095F80BA01AF0080FB8D15DF019F90028B4D1637E8AEA0303DB06B0
:2009000040F1C780344D41F602016B565F1CC1D003F5B17305EB0313FF26DA796E5460F328
:200920000002DA71B6E73B782F49022B4FF009025046C3D00B78002BC0D1C1E905330A7067
:200940008BF800304A6B0B7351F8143CC1E90132FFF716FE01283FF4E0AE0228AED06EE74A
:20096000E0690023112205A9FEF7A0FE01283FF44EAF09B0BDE8F08F237E19077FF559AF24
:20098000154A41F2C873D15C00297FF458AF0721D1544EE70023E26AA16884F82830204686
:2009A000FFF756F84BE7626AE06AA0630421C4E90233C4E90B2284F83C30636384F8281065
:2009C00063622046FFF75EF839E7FEF7FFFD01986FF00F03BEE600BFF8BD0020E0D5002078
:2009E00010BE002010D4002008D60020474D41F60202AB565E1C09D003F5B17305EB0313C2
:200A0000FF20D979A8546FF30001D97141F603016B56581C0ED003F5B17305EB0313FF202D
:200A2000DA796854C2F34501013921EAE17161F34602DA71237EDA067FF540AF3448FFF7D8
:200A400021F84FF6FF720223228484F8303056E6304B05A9B3F9A82502A848F0C5F89DF80E
:200A60000C309DF80D609DF80A509DF80B20BDF808109DF80E00DB0243EA461342EA451233
:200A8000A1F2BC7143EA500342EA41229BB292B2B1E6A98A6B8B204A43EA0143126863621C
:200AA000EB69A3605202B3FBF2F102FB113109B113445B1A154DE36041F6020184F819A021
:200AC0006B565E1C09D003F5B17305EB0313FF20DA7968546FF30002DA7141F603016B5607
:200AE000581C0ED003F5B17305EB0313FF20DA796854C2F34501013921EAE17161F3460226
:200B0000DA71032384F830307DE600BFF8BD0020E0D50020286F002038D600202DE9F0438E
:200B200090F82830013B83B00446082B41D8DFE803F048054D525865406A4300384B46684F
:200B4000056B41F6480103F5C2525F5813683740EA19B2EB432F4FEA432816D258E0216990
:200B6000207EFEF7E3FE012823D1256B666823696361A5EB08053D444644F61B019B66601B
:200B8000A84525634F46236142D82046F7F728FD01AA81460028E2D06668A368E26A9E42E3
:200BA00038BF1E460023A66084F828300AB12046904703B0BDE8F083FFF7E2FC03B0BDE8EE
:200BC000F083FFF78BFD03B0BDE8F083FFF764F803B0BDE8F0830021FFF7C8FA03B0BDE80B
:200BE000F0830121FFF7C2FA0128E2D10023216C84F828302046FFF7BFF8DAE7FFF790F9FB
:200C000003B0BDE8F083FFF753FB03B0BDE8F0832046F7F7E5FC0028BFD12E446660BCE732
:200C2000F8BD00202DE9F04782B0054602AF18461C460E4690465AF0F9FB083020F00700ED
:200C4000ADEB000D0DF1080A013CD14614F8013F5BB989F800304246CDF800A031462846A8
:200C600040F0BEFFBD46BDE8F087184647F06EFEC3B2A3F120023F2A88BF202309F8013B0C
:200C8000E4E700BF2DE9F04704460D469046002144221E46089F5CF01AFF01234FF6FF7239
:200CA0002676628384F828302B782E2B4CD02E4604F1310A307804F1390968B12E280BD0FA
:200CC00047F044FEC0B20AF8010BCA4506F1010607D030780028F1D120200AF8010BCA4548
:200CE000F7D130782E2808BF707804F1380908BF013604F13B0A58B147F028FEC0B209F838
:200D0000010FD14506F1010607D030780028F3D1202009F8010FD145F7D118F0100F14BF1B
:200D20000323012384F819802370E7622B782E2B26D16B7823BB0323204684F83030FFF766
:200D4000CDFC2046BDE8F0876B78002BAFD1114B41F2F47241F60C0041F2F0719A5818588C
:200D60005958E26041F601026062A1609A5C627641F2E8729B5C2370E7622B782E2BD8D0B1
:200D80000023204684F83030FFF7A8FC2046BDE8F08700BFF8BD002010B5104C14F8863C4F
:200DA00023B90F4B4FF480225A6110BD0D4A136823F0060313605AF005FB14F8863C002BEC
:200DC000EFD054F8803C9B68DB07EAD5E26F136823F0030161F307031360E2E7305E00207D
:200DE000003C014010ED00E008B50121032003F053FD72B64BF00AF92DE9F04F8DB0CF4C41
:200E0000DFF84C93CE4D00904FF0000854F80B0C002800F0FE8040F03BF80646002800F06A
:200E2000DB81D9F8843044F8073CE0260023C54F04F8033CA4F10B0B06FB08F654F80B0CCD
:200E400040F026F8002800F0E48054F80B0C40F017F814F8023C5A1E82460B2A0DD8DFE8BB
:200E600012F01F003A004600530083009B00E3001701370142017901910124280CD0009A1C
:200E80003AB995F8D220824240F08281012204F8032C0D2BD2D186E0012304F8023CCDE748
:200EA00000234D28C4F8C53084F8CD3084F8CE3004D0582808D004F8023CBFE7022204F8CA
:200EC000022C84F8C430B9E7032304F8023C022384F8C430B2E704233C2804F8023C0BD0A6
:200EE000BAF13E0F0CD0002304F8023CA6E70A233C2804F8023CF3D1002304F8013C9DE7C5
:200F0000012304F8013C99E7D4F8C500BB190344421CC4F8C52083F8CFA594F8CD00022AD5
:200F20008AEA000184F8CD1088D12378C02BDAD86278FF2A08D1052BD5D9012384F8C43004
:200F4000072304F8023C79E7A4F8C12000229342C4F8C93014BF0523062384F8C320C4F865
:200F6000C52004F8023C69E7D4F8C500BB190344421CC4F8C52083F8CFA594F8CD00D4F843
:200F8000C9308AEA00019A4284F8CD107FF456AF062304F8023C51E794F8CD308342A2D1DA
:200FA0000D2304F8023C14F8017C002F40F0F680654B08940FCB04AE86E80F00D4F8C9304F
:200FC000D4F8D100ADF82A7023440993B4F8C130ADF8283094F8C3308DF82C3001238DF88F
:200FE0002D30324603AB08A9039730F001FC48B1049B059394F8C420544B0493314658461B
:2010000030F044F9039E002304F8023C002E40F0DB8008F10108B8F1030F04F1E0047FF4B3
:20102000F5AE0DB0BDE8F08FD4F8C500BA190244431CC4F8C53082F8CFA594F8CD2094F87F
:20104000CE0001938AEA020284F8CD205146D52247F03AFE019B84F8CE00072B7FF4EEAE29
:20106000B4F80530C02B3FF63EAFB4F80320A4F8C120A27884F8C32000229342C4F8C93011
:2010800014BF08230923C4F8C52004F8023CD5E6D522014694F8CE0047F016FE94F8CD3024
:2010A00084F8CE008AEA0303D4F8C50084F8CD30BB190344421CC4F8C52083F8CFA5D4F88D
:2010C000C9309A427FF4BAAE092304F8023CB5E694F8CD30434084F8CD3094F8CE3083428B
:2010E0007FF401AF54E7D4F8C500BA190244431CC4F8C53082F8CFA594F8CE000193D52205
:20110000514647F0E1FD019B84F8CE00052B7FF495AEB4F80120B4F80330A4F8C120227894
:2011200084F8C32000229342C4F8C93014BF0B230C23C4F8C52004F8023C7FE6FF630020B2
:20114000286F0020305E002004DD060878A00120482B0020D522014694F8CE0047F0B4FDEF
:2011600084F8CE00D4F8C500BB190344421CC4F8C52083F8CFA5D4F8C9309A427FF45EAE6B
:201180000C2398E694F8CE3083427FF4ACAE07E7232804BF022204F8032C7AE6012F4FF06C
:2011A000000602D004F8026C33E7D4F8C93008942344099308A8B4F8C130CDE90A66ADF857
:2011C00028302DF029FEEDE754F80B0C37F056FE54F80B0CB0471CE714F8033C002B3FF4BB
:2011E00018AFD9F8842054F8071C521A632A7FF610AF012B29D0022B7FF40BAF54F80B3C05
:20120000C5F8AC350122C5F8B035C5F8B835402385F8AA2585F8BD050D4A0E4885F8BC35B8
:201220000D4BC5F8B42545F8143CC5F8003646F08BF94FF400503AF035FB084846F078F9A2
:2012400085F8046685F80566E3E6FFF7CDFD00BF19E00408745E0708DC740020AA5E07080A
:20126000202301480B807047F4040020642301480B80704714050020432301480B8070474C
:201280007805002010B5074CD4F8C800FF2807D0054951F8042BF7F7CBF8FF23C4F8C830BA
:2012A000002010BDF404002050D60020EAE700BF08B5D0F8E4355B6A9847002008BD00BF6D
:2012C00008B5D0F8E4351B6A9847002008BD00BFD0F8E43510B504461B689847D4F8E8352D
:2012E0009B689847002010BD08B5D0F8E435DB6903B19847002008BD08B5042290F8121137
:20130000D0F8E83580F8131180F81221DB689847002008BD10B5D0F8E83504461B69984743
:20132000032384F81231002010BD00BF0B0630B41CD401EB810200EBC202002300EB810585
:2013400082F8741382F8753301241A4604FA01F16D6D61F31F4201696FF3CF332B60CB69D9
:2013600023EA0203002030BCCB61704701F07F0101EB810400EBC404012200EB8105002320
:2013800084F81C1184F81D2102FA01F11A46AD6961F30F02DFE700BF10B581210446FFF7F5
:2013A000C5FF20460121FFF7C1FF024B0020187010BD00BFB074002010B581210446FFF7BF
:2013C000B5FF20460121FFF7B1FF82212046FFF7ADFFF7F775F8002010BD00BF38B50D4639
:2013E00004468321FFF7A2FF29462046FFF7E4FF002038BDF0B416460A063AD401EB810515
:2014000000EBC5052824002204FB0104022B85F87413C5F87C6385F8773385F8752304F5A3
:201420005D7448D0154600EB8107012202FA01F17F6D61F31F45D7F800C01CF4004F11D170
:20144000E488204946F0805242F4004242EA834204F00F041C4B42EA845211400CEA030389
:20146000194339600269D3692B430020F0BCD361704701F07F0101EB810500EBC5052824C7
:20148000012204FB0104022B85F81C11C5F8246185F81F31A5F8221185F81D2104F58E74B9
:2014A0000CD0002500EB8107012202FA01F1BF6961F30F05BFE722711546B4E7002525712D
:2014C000F0E700BFFF87CC13007833EC002310B5194604464022FFF78DFF802120460023DB
:2014E0004022FFF787FFD4F8E835A078012284F812215B689847002010BD00BF70B44B7806
:20150000012B26D00B784A6900EB83035C6D25682369D2B18A684A6102F07F0223F4002353
:2015200023F07F0342F4002213432361C378012B04BF0B696361C5F3076363F07B0363F339
:201540001F652560002070BC70478A6802F07F02E4E782694C691568136944B38E68B442D3
:201560008CBF06F07F0404F07F0423F4002323F07F0344F4002443EA040388BF4E61136167
:20158000C378012B1DD0C5F3076464F07B0464F31F651560002BD5D14B69002BD2D00269F4
:2015A0000878516B012383400B435363CAE723F4002323F07F0343F400231361C378012B4F
:2015C000E1D10B780C6900EB8300C5F30763816963F07B0363F31F654C610020156070BCCE
:2015E000704700BF2DE9F0434B78012B30D00B784C6900EB83035E6D356837691CB38B68CA
:201600001C44013CB4FBF3F4C4F3090203FB02F3C3F312034B61144643EAC44363F31C0764
:201620003761C378012B04BF0B697361CB78012B44D0C5F3076363F07B0363F31F653560BB
:201640000020BDE8F0838A680124C2F31203E3E791F800804E6900EB880EDEF818C0DCF8E4
:201660000050DCF8107076B3D1F80890384A06EB0904013CB4FBF9F402EAC444C6F3120222
:201680002243CC7807F060473A43012C174649D0CCF81020C278012A55D00269516B03FA41
:2016A00008F30B435363C5F3076363F07B0363F31F65CCF800500020BDE8F0834B7973B328
:2016C00045F00055B5E707F0604747F40027CC78CCF81070C378012B2FD0012CE3D10269AA
:2016E0009268D20554BF45F0005545F08055C5F3076262F07B0262F31F65CCF80050002B6A
:201700009ED1B0B203308010DEF8D04098D0CA6852F8041B216001339842F9D190E745F047
:20172000805586E764F35E77CCF81070C378012BD5D10A69CCF81420D1E70A69CCF814205C
:20174000012CB0D1CBE70B69CCF81430ABE700BF0000F81F0E4BDA68D20310D4DA68D106D8
:201760000FD4DA68D20510D4DA6812F0E00F0AD1DB6813F0020F14BF082009207047012028
:20178000704706207047072070470220704700BF003C024000207047104AD068A8B1136983
:2017A0009BB188420FD88B4234BF00230123DBB243B193695161994204D0094B91611420CD
:2017C00083F8CC0070470023F1E7A1F59C53083BB3F57A7F2CBF00230123E9E750D600205F
:2017E000F4040020054B5A7F19778A4204D0044A5977142082F8CC00704700BF50D6002024
:20180000F4040020704728B1034B987F012894BF00200120704700BF50D6002008B5FFF78F
:20182000F2FF50B1054AD37F127F5B0003F00203002A18BF43F001030B6008BD50D6002083
:2018400008B5FFF7E0FF10B1014B1B6A0B8008BD50D6002070B5FFF7D6FF50B10A4A958C68
:2018600035B1966A0023B3421C4603DB002000E00D7070BD02EB44040133A48DAC42DBB26B
:20188000F1D10B70F5E700BF50D6002008B5FFF7BAFF10B100230B70137008BD042070473C
:2018A00028B1034B93F9CE00003818BF01207047F404002008B5FFF7F3FF50B1054B93F926
:2018C000CE20012AC3BF93F8D130C3F340030B60002008BDF404002008B5FFF7E1FF18B124
:2018E000024B93F8D0300B7008BD00BFF404002070B5FFF7D5FF38B10E4C94F8D130DB0758
:2019000003D500230B70137070BD0B4D94F9CF3095F83C6093FBF6F301330B7094F9CF40D2
:2019200095F83C1094FBF1F301FB134301331370EAE700BFF404002050D60020032070478A
:2019400070B50A4A92F8403006255E1CB6FBF5F405FB146492F84150AC4205D002EBC303CC
:20196000C3E9110182F8404070BD00BF50D60020002230B504461046914200DC30BDA35C3B
:201980000825584010F0800F4FEA400318BF83F0D503013DD8B2F5D10132EDE710B5D9B171
:2019A0000E4B586F814217DCB2B1DB6B9A4213DC0B4C013A013903FB012184F8DC1004F194
:2019C000D8000521FFF7D4FF062184F8DD0004F1D800BDE81040B3E710BD00BF50D6002092
:2019E000F40400200023038083708380C3800381704700BF074A084992F87830097801336D
:201A0000DBB2994282F8783004BF002382F87830704700BF50D6002078500020F8B5794C1E
:201A2000E36F83B1784B1B6893F82E305BB1774B94F88020A3FB0013012A4FEA931330D03C
:201A4000022A08D002B1F8BD714B9842FBD9012384F88030F8BDD4F8842064329A423ED8B3
:201A600094F8783004EB031393F8F824FF2A06D068490132012083F8F82481F8DE00FFF79E
:201A8000B9FF654B1B780122092B84F88020DAD1B4F87A35614A01339BB2A4F87A35538088
:201AA000F8BD94F878105C48C4F884308C2303FB0143007883F89A20002384F8963004F151
:201AC0008C050A2202230928C4F8885084F8972084F88030B7D1514B01311980F8BD94F8D0
:201AE000962094F897309A42ADD104F18B0004F19405002310F8012F082153405A0013F001
:201B0000800F08BF5B0082F0070214BFD3B2DBB20139F3D18542EDD194F895209A4239D10A
:201B200094F8786094F8935094F89430B4F88F00B4F8912094F88DC004EB061743EA0523B0
:201B400094F88E5087F8F81440BA52BA81B292B245EA0C202F4DC7F8FC141BB294F98C1077
:201B6000C7F80025032E4FF00102A7F8FA04A7F8043587F8F91485F8DE2008D8264A1278B8
:201B80000C2A29D00D2A02D1244B23F81610FFF731FF5CE794F8783004EB031393F8F82413
:201BA000FF2A06D01B490132012083F8F82481F8DE00FFF71FFF184B1B780122092B84F8A3
:201BC00080207FF440AFB4F87835144A01339BB2A4F878359380F8BD1149124A91F8221049
:201BE0000E4803EB830303EB830349089B0093FBF1F382FB0312DB17C3EBA20320F8163014
:201C0000C5E700BF50D60020506A0020D34D62103F4B4C00F4040020404A0020484A00205D
:201C2000A82C0020676666660B4B93F8961093F8972091420ED010B493F89620D3F8884005
:201C4000511CD2B2C0B2C9B283F89610A0545DF8044B7047704700BF50D60020FD2870B530
:201C600022D0F02804D0EF2822D00224204670BD114D0320052641282E444FF0000405F104
:201C8000010580F080030DD0042B0BD9FFF7E6FF2044B542C4B2E9D015F8010B412880F004
:201CA0008003F1D10420F3E7044D0B200426E2E7034D0C200626DEE7EC5E0708F45E07084B
:201CC000E45E07080E4BD3F88025B3F97C05530707D400EB8000400080B200F5C87080B24C
:201CE0007047084B084AD3F8C430323382FB0312D817C0EBA20080B200F5C87080B270474E
:201D000050D60020283C00206766666600B5062983B00A464FF03203014628BF06220DF131
:201D200001008DF800305BF071FE044B6846D3F88435984703B05DF804FB00BF50D60020C7
:201D40005E2810B511D05D2805D00D4BBDE81040D3F8883518470A4CD4F888359847D4F83F
:201D600088353D20BDE810401847054C5D20D4F888359847D4F888353E20BDE81040184784
:201D800050D6002070B5094E0546D6F888355E200C469847D6F8883528469847E0B2FFF79C
:201DA000CFFFC4F30720BDE87040C9E750D6002003682DE9F041002B3D4D3E4F3E4EB8BF35
:201DC0005B42A5FB0321890D07FB0137C7EB0717BF0096F8923585FB0725FA170446C2EB3A
:201DE000A555002B57D101EB810101EB810105EB810109B2DFF8BC801320FFF7C3FF2F4917
:201E000008FB057581FB0531ED17C5EBA11109B21B20FFF7B7FF2368254D002BB4BF53217C
:201E20004E212320FFF7AEFF636896F8922583EAE376A6EBE376A5FB0631890D08FB0168B4
:201E4000C8EB08184FEA880885FB08354FEAE873C3EBA5552ABB01EB810101EB810105EB3C
:201E6000810109B21220FFF78DFF124B134903FB058581FB0531ED17C5EBA11109B21A2023
:201E8000FFF780FF6368002BBDE8F041B4BF57214521222076E7C1EB011105EB810109B226
:201EA000A8E7C1EB011105EB810109B2DAE700BF6BCA5F6B806967FF50D60020D34D621002
:201EC00030B40023022515244FF4167140F2D93205808471018130BC42814380838083811F
:201EE000704707B50DF1060210F022F968B1084BBDF80620B3F8B0159A84914205D0054983
:201F0000A3F8B025142081F8CC0003B05DF804FB50D60020F404002013B50446FFF7C0FCAF
:201F200008B300230DF106022046ADF8063010F0FFF8C0B10D4C9DF8062094F9CE1084F819
:201F4000E320032908BF62F07F024FF00501084808BF84F8E320FFF70BFD062184F8E40058
:201F60000348FFF7EDFC02B010BD00BFF4040020D305002008B5044BD3F8B4053EF088FFA4
:201F8000B0FA80F0400908BD50D600202DE9F04F204B85B04FF0000804461E2093F800A0E4
:201FA00093F801B09D78B3F80490DF881E7ACDF80480ADF80C8023F07FFD18B117B1B946F9
:201FC0000125C246144A92F8B835D9070AD492F8BF253AB9012E1BD0022E03D113F0020FAD
:201FE00008BF01258DF80C608DF804A08DF805B08DF80650ADF80890ADF80A7001AB03CBEF
:020000040801F1
:202000001B88206020466160238105B0BDE8F08F3546E7E71874002050D60020144B30B47B
:20202000D3F8E44514B300220F2583F8EA15090A83F8E90583F8EB15C3F8EC25C3F8F02582
:20204000C3F8F42583F8E85503F5BD60012110F8015F01312A440E29D2B2F8D183F8F6259B
:202060002046044930BC10223EF0E2BE30BC704750D6002038DC0020034B002183F8F815AD
:20208000C3F8FC15CAE700BF50D6002013B504462620019123F010FD019920B9204602B029
:2020A000BDE81040BAE702B010BD2DE9F743B74CD4F8E4350D464BB14FF0020800264FF0D6
:2020C0000109D4F8E4053EF0E3FE58B90027A37F042B00F25781DFE813F08F00E400F700AB
:2020E0003D014601D4F8E4053EF0CAFED4F8FC355A1C2344C4F8FC2583F8000694F8F835BF
:20210000012B0AD0022B11D0002B70D10F280CBF84F8F895C4F8FC35D3E7A0F17203012B5B
:2021200001D9762863D184F8F885CAE7102AC8D197490023012211F8010F013203440E2A85
:20214000DBB2F8D194F80E2684F8F8659A42C4F8FC65B6D194F80F36002BB2D194F801768E
:20216000732F37D0762F0DD0722FAAD194F8032694F8023653EA0223A3D0E360B4F80436A1
:202180002361A4E794F8032694F8023653EA022397D094F8051694F8042694F80906236271
:2021A00042EA012294F80616E17794F8071684F8121694F80816A4F8102641EA0021A4F81F
:2021C0001416616901B96361A38C002B7FF47FAFA2847CE794F8072694F8063643EA022336
:2021E0001AB2002B3FF46DAFA4F816266FE784F8F865C4F8FC6564E7722F44D10123A37736
:202200000022644B1B78402B2FD1634E94F812C6A08CA37FB4F810E6338005024FEA0C33B8
:20222000217F778005F4706503F440532B434FEA0E1543EA8133EDB22B43276A65691BB2CB
:20224000BD4214BF0825002513432B43704514BF042000201843514B614514BF0221002116
:2022600093F8CC30F3800143B180636F1BB1A36A002B40F09D804A494A481F2203B0BDE80E
:20228000F0435BF062BCD4F81836474AEB1A934201DC0022B5E77220FFF7EEFEC4F81856E4
:2022A000F7E7762F03D10223A3770022A9E7D4F818363D4AEB1A9342EBDD7620FFF7DCFE2D
:2022C000C4F8185600229CE7344ED4F8183696F8CC20EB1A82B3344A934230DDE27FD20745
:2022E0001BD46169226A91420ED089B24620FFF7CDFE96F8CC30C4F81856013B86F8CC301C
:202300000423A37701227CE7A18CB4F810268A4203D05020FFF7BAFEEBE7217F94F81226F4
:202320008A4206D0B1FA81F149094920FFF7AEFEDFE7142286F8CC201C4A9342BDDC762FA2
:20234000A7D17320FFF798FE0323A377C4F81856002256E7732F9CD0D4F81816124B691A35
:202360009942A0DC95E7D4F818360F4AEB1A93428FDD7620FFF780FE0223A377C4F818565E
:2023800000223EE70023A3771A463AE750D6002050DC0020404A0020484A0020F404002032
:2023A000AF5E0708D90500203F0D03003F420F00334DD4F81C662A2385F8E5300DF1020275
:2023C00020230DF10101304685F8E6300FF047FF30B19DF801109DF8027051EA070339D18F
:2023E000552385F8E730462385F8E830202301A9304685F8E9300FF02CFF0346214813B13A
:20240000BDF804209ABB204948F0F0FFB4F814761E4D87B30DF1030130460FF01DFF50B38D
:202420009DF803100DF1060230460FF081FE10B3BDF8062016493B46BA420CBF20222A2227
:20244000284648F0D3FFB4F81636A4F8203603B0BDE8F08330460FF0E7FE394685F8E70012
:2024600030460FF0CDFE037885F8E830BEE7094948F0BCFFCAE70849284648F0B7FFE2E7FB
:20248000F4040020DE050020D15E0708E2050020C95E0708E6EA0708D05E070838B50B682A
:2024A0000E4D5A1C0A6005221A700B6895F8CE200C46591C21601A70236895F8D120591CF2
:2024C00021601A70B5F8D410204646F025F8236895F8D620591C21601A7038BDF40400200C
:2024E0002DE9F0472DED028BFFF7DAF9C8B31E4B93F9CE00012834DD93F804411B4F9FEDE1
:202500001C8A15468E1E02EB44084FF03209454504D1BDEC028B2046BDE8F08737F802AB68
:2025200026F802AF07EE90AAF8EEE70AB2EE040A60EE880A5AF0A2F8BCEEC00ABAF10E0F18
:2025400010EE103A9BB209D91933B3FBF9F39BB203EB830303EB83035B009BB225F8023BE7
:20256000D5E70024D5E700BFF404002072DC0020CDCCCC3D38B50D46FFF792F9044638B1E4
:202580000C4890F8D130DB0704D5B0F8D2002880204638BD084A90F9CF3092F83C2093FBD8
:2025A000F2F102FB11320132013100F584700FF0D3FDECE7F404002050D6002038B5134C5E
:2025C00094F8413094F840209A4219D004EBC3030F49D3E911200023984212DC93780D4A06
:2025E000C4F834065B081370FCF7CEF894F8413006210133B3FBF1F201FB123384F841302F
:2026000038BDD55C01F8015B0133E5E750D6002022740020507400202DE9F04FA94B1B7883
:202620008BB08146002B40F0B580A74ED6F81C56002D00F0AF80A54AD2F80C4104F0F0217C
:20264000B1F1E02F6BD1C2F80C31D6F83826944265D004930593ADF818309D4BC6F838461F
:202660009A881F78ADF8142093F801C01A7A93F802A08DF810700DF110088DF811C08DF8C5
:2026800012A08DF8182098E807000DF11C0EAEE803009049AEF80020C4F34252895CC4F3FD
:2026A00003428F4202F101021F4601D1944508D028468DF81C108DF81D200FF04DFDADF857
:2026C000200028460FF099FF032804F0070B33D0042835D000239A4501A9284618BF8DF8FA
:2026E0001E300FF0B3FD48B1019BC4F3001103F001038B4202D028460FF056FE0A2207A94D
:2027000040465BF0BCF950B19DF81E30BDF81C20BB703A80BDF82030BB8046F02DFC96F84C
:202720003CA6DFF8ACB104AF96F83C36032B7BD8DFE803F00A3376A3674B13F80B30CAE796
:20274000664B13F80B30C6E7394628460FF084FD044658B107A8FFF719FC9DF81E109DF803
:2027600010308B4260D028460FF0AAFE96F83C36013303F0030386F83C360CB99A45D3D1A2
:2027800096F8B835DB0700D524B12B6849461B68284698470BB0BDE8F08F01A8FFF7F6FBD1
:2027A00096F8B8859DF8044008F00108ECB1B8F1000F39D13A460DF1030128460FF04FFDDA
:2027C000044688B307A8FFF7E1FB9DF81C109DF803309DF81D208B4203D19DF8103093424D
:2027E00022D028460FF076FEC0E7B8F1000FBDD1394628460FF02DFD0446A8B107A8FFF7BB
:20280000C5FBBDF82010BDF810308B420CD086F83D8686F83E862B6828469B699847A5E782
:2028200096F8B835D80701D500249FE707A928460FF00CFD04460028F6D01E2023F03CF9DA
:2028400096F83F3683428046EED086F83F0660B1BBF80630002BE7D1079BD907E4D4012130
:2028600028460FF0A1FD444680E7079BDA07DBD5014628460FF098FD78E73846FFF786FB8C
:2028800097E8070007AB03C31A809DF810309BB10DF11D0207A928460FF0E1FC0DF11E014B
:2028A00028460FF0D9FC0A2207A938465BF0E7F8041E18BF012459E708A928460FF0C9FC11
:2028C000ECE700BFD274002050D60020F404002018740020145F0708085F0708FC5E070895
:2028E000024B0146D3F840063EF0D6BA50D600202DE9F041FD2984B0044600F0DD80F029DE
:2029000000F0BC80EF2900F02F814AB10346861803AD002003F8010B9E4205F8010BF9D167
:20292000994B0B2003F1090501E013F8010F814200F0C780AB42F8D14B1E832B00F29280BF
:20294000DFE813F03001370184004101AF01B501480153015F0190009000650165016501C9
:202960007B017B017B015F019000900086018E0190009000900090009000900090009000CD
:20298000900090009000900090009000900090009000900090009000900090009000900037
:2029A000900090009000900090009000900090009000900090009000900090009000900017
:2029C00090009000A4019000900090009000900090009000900090009000900090009000E2
:2029E0009000900090009000900090009000900090009000900090009000900090009000D7
:202A00009000900090009000900090009000900090009000900090009000900090009000B6
:202A2000900090009000900090009000900090009000900090009000900090009000900096
:202A400090009000900090001D011D014F4B93F89715002900F0628101922DF0C1FB019A26
:202A6000ADF80C003AB1224403AB13F8011B04F8011BA242F9D104B0BDE8F081444F032138
:202A80004FF00508B844002501370CE0FFF7E6F8064660193246FFF72BFF70194745C5B2E8
:202AA000E9D017F8011B412981F08003084601D0042BEBD80426ECE7364F0B214FF00408CA
:202AC000E0E7324BD3F8800580060CD4002AD2D0224403AB13F8011B04F8011B9442F9D13D
:202AE00004B0BDE8F08193F84406870741D52A4D287D052834BF02260326142916D97C3925
:202B0000C8B20628E2D80629E0D801A050F821F0F52C0108F52C0108DF2C0108CD2A01080A
:202B2000052D0108FF2C01080B2D01080929CDD90A390A29CAD801A757F821F0C52C0108F3
:202B4000112D0108CD2A0108CD2A0108CD2A0108CD2A0108CD2A0108CD2A0108CD2A01082E
:202B6000D72C0108F52C01080C4F0C214FF0060888E7094B0B29187DA8D10126C9E0084B22
:202B8000D3F8C03003936DE7D85E070850D60020EC5E0708F45E0708706F0020E45E0708FB
:202BA000283C00200192FFF78DF8019AADF80C0058E76A4BD3ED037AFDEEE77A17EE903AEB
:202BC000ADF80C304EE701922DF00AFB019AADF80C0047E7624D95F8B835DE0700F1A7808A
:202BE000B5F86C36ADF80C303CE75D4B5D49B3F9E83681FB0301DB17C3EBA103ADF80C30C5
:202C000030E7574BB3F8EA36ADF80C302AE7564BDFED566AD3ED007A0C39C9B203EB8103A5
:202C200093ED127A67EEA67A67EE877AFDEEE77A17EE903AADF80C3014E7494B03EB410102
:202C4000B1F8C63603EB83035B00ADF80C3009E7434B93F8B83503F00103ADF80C3001E769
:202C60003F4BB3F88816CD055ABFCB4303F00103032311F0440F18BF042311F0020F18BF30
:202C8000072311F4806F18BF0923ABE70192FFF719F8374B019AD3F8C83043EAC040039047
:202CA000E0E62F4BD3F87C36ADF80C30DAE62C4BB3F86C16002934D001922DF0A9FA019AF7
:202CC00080B2CDE62B8A03EB830303EB83039B00ADF80C30FAE6EB89ADF80C30F6E6EB8971
:202CE000244903EBC3039B00A1FB03135B09ADF80C30EBE6B3F84636ADF80C30E6E66B68A9
:202D00000393E3E62B680393E0E6AB680393DDE6F6B28DF80C608DF80D00D7E6B3F8480618
:202D20009EE6D3F8840680F3100080B298E605F5CA65019222F026FFD5ED037A019AFCEED0
:202D4000E77A17EE903A9BB200287FF44BAF0A49096811F0100F18BF002343E7A0DC0020BD
:202D600050D6002067666666DCDC002000007A44283C00201F85EB51F46E002070B5214D65
:202D800095F8EC36EA181C4692F8F0268AB11E4E09225C1CA6FB04135B0803EBC303E31A6A
:202DA000E918DCB291F8F01609B1013AF1D185F8EC4602681549561C06600C2616700268CD
:202DC000561C0660002616700268561C066003EB430603EB8603147019440D2245F054FBEB
:202DE00095F8EC16084B4A1CA3FB02035B08294403EBC3030120D31A81F8F00685F8EC3648
:202E000070BD00BF50D60020398EE3384CDD00202DE9F041684ED6F81C7684B004463846FC
:202E20000D460FF0EAFB86F8710757B10DF1090202A938460FF013FA002840F08E8096F82B
:202E400071070023ADF808308DF80A301A46431EDBB20021FF20FD2B8DF80C20ADF80E1011
:202E60008DF80B0003D9002004B0BDE8F0819DF80830042B00F09680052B00F09980032B93
:202E800000F09880022B00F08C80012B08BF042100F088809DF809309DF80A10D6F81C0684
:202EA000013B0DF10E028DF809300FF041F996F87137032B73D0042B0CD1404A9DF80A00F5
:202EC0000121002301E012F8011F81426DD20133082BF8D1D6F87427029B394F9A420DF108
:202EE00008084FD023680D22591C21601A7023680022591C21601A7023689DF80820591C7F
:202F000021601A7023689DF80920591C21601A7023689DF80C20591C21601A7023689DF8F1
:202F20000A20591C21601A70BDF80E10204645F0F3FA23689DF80B20591C216020461A705B
:202F40000721FAF7B9FE98E8030087E803000120C6F87C5704B0BDE8F08101A938460FF009
:202F600075F900283FF46BAF38460DF10A010FF073F900283FF463AF019B96F8710703F07A
:202F8000010264E77A68D8F804309A42AAD1D6F87C370C4AEB1A93427FF665AFA2E70A4A8F
:202FA0008CE703218DF8081074E78DF80A3091E70121F7E70221F5E750D60020FC5E07089D
:202FC000C4DD002080841E00085F07082DE9F0412A4C2B4AD4F87C36B4F88077B4F88466AF
:202FE00082FB0352DB17C3EBA2031FFA83F8474582B00D4603D1B4F88237B34233D002687A
:203000000190511C34230160137002680023511C01601370414645F07FFA0198314645F01F
:203020007BFA019847F6FF7145F076FA019847F6FF7145F071FA019847F6FF7145F06CFA69
:20304000019847F6FF7145F067FA01980221FAF733FE0120A4F88087A4F88267C4F88457D6
:2030600002B0BDE8F081D4F88437064ACB1A9342C5D8002002B0BDE8F08100BF50D600206D
:203080006766666680841E00026810B57F21541C0460117002680024511C01600E21147042
:2030A000FAF70AFE012010BD2DE9F04FC24B1B68804613F0800083B000F07181BF4B93F851
:2030C000440610F0020000F06A81DFF810B39BF81430052B40F26881DBF80030B84D009372
:2030E000002BB8BF5B42A5FB0342B648B649920D00FB0233C3EB03139B0085FB034502EBCC
:203100008202DC1702EB8202C4EBA55400FB043304EB8204A4B281FB0321DB17C3EBA11130
:20312000BCB10025A94F2E46A7FB0432D20802EB8203A4EB4303E8B2A4469BB28000834084
:20314000BCF1090F94B246EA030605F10105EBD8340489B2B9B100259C4F2E46A7FB013236
:20316000D20802EB8203A1EB4303E8B28C469BB280008340BCF1090F91B246EA030605F1FE
:203180000105EBD83443DBF804E08D4D8D4E8E498EEAEE70A0EBEE70A5FB0032920D06FB7B
:2031A0000200C0EB0010830085FB035002EB8202DD1702EB8202C5EBA05506FB053305EB58
:2031C0008205ADB281FB0321DB17C3EBA111C5B10020DFF8F8C10646ACFB0532D20802EB00
:2031E0008203A5EB4303C7B2A9469BB2BF00BB40B9F1090F95B246EA030600F10100EBD80E
:20320000350489B2C1B10020DFF8C0C10646ACFB0132D20802EB8203A1EB4303C7B28946C4
:203220009BB2BF00BB40B9F1090F91B246EA030600F10100EBD83543DBF80830634A0193D0
:20324000002B1846B8BF5842A2FB0030604E6149030AA6FB0363DB0901FB03F1C1EBD0014A
:2032600089B2B9B1002691463746A9FB0132D20802EB8203A1EB4303F0B28C469BB28000F9
:203280008340BCF1090F91B247EA030706F10106EBD8B9B2BBF81070DFB10026DFF82CA16F
:2032A000B446AAFB0732D20802EB8203A7EB43035FFA86F938469BB24FEA890903FA09F3AB
:2032C000092897B24CEA030C06F10106E9D81FFA8CF7BBF812303D4AA2FB0306F608632E23
:2032E00028BF6326092B63D9002093468146ABFB0632D20802EB8203A6EB43035FFA80FA5A
:20330000B4469BB24FEA8A0A03FA0AF3BCF1090F96B249EA030900F10100E8D85FFA89F9C6
:20332000009B019A002BCCBF392338231616BEF1000F26F07F0635DD274A3343964543F05E
:203340000206C8BF43F00606D8F800301622581CC8F800001A70D8F800300022581CC8F853
:2033600000001A70404645F0D7F82146404645F0BBF82946404645F0B7F84046394645F051
:20338000CBF8D8F800305A1CC8F8002083F80090D8F800305A1CC8F8002001201E7003B051
:2033A000BDE8F08F1E43CFE7002003B0BDE8F08F4FF00009B4E700BFF46E002050D6002071
:2033C0006BCA5F6B806967FFD34D6210CDCCCCCCC55A7C0AA0860100FFC99A3B706F002074
:2033E0002DE9F047AB4B1B68064613F0800084B000F09E80A84B93F8440610F0020000F03C
:203400009780A64F397D052940F29780632900F292800024DFF898C289B22546ACFB01320E
:20342000D20802EB8203A1EB4303E0B28E469BB280008340BEF1090F91B245EA030504F142
:203440000104EBD8EDB2BB68954A82FB0312D917C1EB623189B2002900F018814FF0000C0A
:20346000DFF84CE26446AEFB0132D20802EB8203A1EB43035FFA8CF088469BB28000834070
:20348000B8F1090F91B244EA03040CF1010CEAD8E4B2FB8983494FF4F36707FB03F7A1FB0C
:2034A0000737C7F38F1742F20F739F4249D8CFB10020DFF8FCE18446AEFB0732D20802EBEF
:2034C0008203A7EB4303C1B2B8469BB289008B40B8F1090F97B24CEA030C00F10100EBD879
:2034E0001FFA8CF7704BD3E9002313433ED14FF0FF3833681722591C31601A70336800229A
:20350000581C306039461A70304645F005F84146304644F0E9FF33685A1C32601D70336812
:203520005A1C326030461C700621FAF7C5FB012004B0BDE8F087992585E7002004B0BDE815
:20354000F0870021DFF868C10F46ACFB0302D20802EB8200A3EB40039BB28B400431102932
:2035600047EA030793B2F0D1BFB2BBE701A845F01DFB9DF80810002900F08A804FF0000CE6
:20358000DFF82CE1E046AEFB0132D20802EB8203A1EB43035FFA8CF089469BB280008340F3
:2035A000B9F1090F91B248EA03080CF1010CEAD84FEA08289DF80910E1B10020DFF8F0E08D
:2035C0008446AEFB0132D20802EB8203A1EB43035FFA80F98A469BB24FEA890903FA09F374
:2035E000BAF1090F91B24CEA030C00F10100E8D848EA0C089DF80A104FEA0828E1B10020BE
:20360000DFF8ACE08446AEFB0132D20802EB8203A1EB43035FFA80F98A469BB24FEA8909C9
:2036200003FA09F3BAF1090F91B24CEA030C00F10100E8D848EA0C08BDF80C301B49632B6B
:20364000A1FB03214FEA08184FEA51117FF651AF0020DFF85CE08446AEFB0132D20802EBA1
:203660008203A1EB43035FFA80F98A469BB24FEA890903FA09F3BAF1090F91B24CEA030CF5
:2036800000F10100E8D848EA0C0832E70C4600E788468FE7F46E002050D60020706F0020D5
:2036A00089B5F814D34D6210D8DD00201F85EB51CDCCCCCC08B5A0F10103B3FA83F30228A9
:2036C0004FEA531301D0184608BD0F2022F0C4F930B9064B93F8B83503F00103184608BD8D
:2036E000BDE808400F2022F0E7B900BF50D60020014B1B681B6A18479C630020024B186858
:2037000008B18369184770479C630020024B186808B14369184770479C63002010B5074C50
:20372000606D40B13DF086FF94F8513013B180F00100C0B210BD012010BD00BF501A002061
:2037400030B40A490A480A78531CDBB20525042B00EBC20400F8325008BF00234FF404525B
:203760000B7062604FF0FF3030BC70477C74002080740020037870B4FBB10446C0F101068A
:20378000A31914F8015FDBB2002DF9D101335B00DCB2032513800C704D7004785CB10223BE
:2037A00000255A1CD2B2CC548D5410F8014F0233DBB2002CF5D170BC704702242346E8E79C
:2037C0000B0617D401EB810300EBC30310B400EB81000124002283F8764383F8741383F8A4
:2037E0007523426D5DF8044B136843F4001300201360704701F07F0101EB810300EBC3033D
:20380000012200EB810083F81C1183F81E2183F81D2182691368002B01DA43F0804343F465
:20382000001313600020704770B501F07F0505EB850400EBC404282101FB05010126C4F837
:2038400030310023C4E94A2284F81C5184F81D61C4F8343101F58E711DB9FDF74FFE00209B
:2038600070BDFDF7BFFE002070BD00BF2249F8B5D1F890370F2B04D05A1CC1F890270020A2
:20388000F8BD1E4C25780023C1F89037002DF6D11B4E1C4B3268B2F5006F17D01B689A420F
:2038A00027D017D9C2F50063402B15D9403B02F14005C1F8943701232370356092B2402384
:2038C00011490A448121FFF7AFFFD8E71B6835607BB12A469B1AE7E74FF0000502EB0307C9
:2038E000C1F894570CBF02210121376092B22170E6E700232370C2E750D60020C42300202F
:20390000AC230020B0230020C8230020AEE700BFF8B51D4C2378012B03D0022B09D0002090
:20392000F8BD01461948D0F8943753B923700020F8BD00231A468121FFF776FF00232370DD
:20394000F5E7402B11D9124C2268403B02F14005C0F89437256092B240230E4C08462244DE
:203960008121FFF761FF0020F8BD094D2A684FF0000603EB0207C0F8946708BF02202F602B
:2039800092B208BF2070E8E7C423002050D60020AC230020C823002038B5134602250A46B9
:2039A000C0E94E3380F811510021FFF73DFF002038BD00BF10B50C7814F0600413D0202CFC
:2039C0000AD14B78023B092B18D8DFE803F01B21171717171717272E22490122FFF7DCFFB4
:2039E0000024204610BD4B78062B24D00A2BF3D01D4B8A78C3F8A027204610BDFAF7FAFE88
:203A00000224EEE719490122FFF7C6FF0024E8E717490122FFF7C0FF0024E2E74B88124A24
:203A20001B0AC2F89C370024DBE70F4B8A78C3F898270024D5E74B881B0A222B0CD0212BCB
:203A400004D021462246FFF7A7FFCAE7CA880949092A28BF0922F6E7CA880749362A28BFC7
:203A60003622F0E7F0DD002050D60020ECDD0020E8DD00204E0600200406002038B501EB9F
:203A8000810400EBC4040D46002184F87453C4F88C1384F87513C4F88833C4F88023C378C7
:203AA0002821012B01FB050108BFEDB201F55D7108BFC4F884231DB9FDF720FD002038BD3F
:203AC000FDF790FD002038BD144B9A6870B5044662B1134A1B7B92F8A4572B4316D08121FF
:203AE0002046FFF76DFE022D09D070BD0C4B93F8A45781212046FFF763FE022DF5D1204633
:203B0000064ABDE870401F230121B7E70121FFF757FE20468121BDE8704051E65C7400200D
:203B200050D6002070B5094A094D1173094B13600021044629700D238121FFF775FE204681
:203B4000054ABDE870401F23012197E7BC740020B0740020555342535C74002010B5064B08
:203B6000597B0446FAF754FE002800DB10BD20460121BDE81040D5E75C7400202DE9F041A4
:203B8000314D2C7834B1012C01D1FFF7E7FF0020BDE8F0812D4FDFF8D080B0F8B4337A68F9
:203BA000C8F804201F2BBA68C8F80820064606D1274B3A689A4202D1797B01291AD9254A67
:203BC00025491378052401F8334001EBC3000133DBB2042B08BF00234FF4005113701F4B4D
:203BE00041600222304683F8A427FFF76DFF0020BDE8F081BB7B013B0F2BE0D8FAF708FE51
:203C0000002819DB2B78013B022BC0D9144B1988B1B1BB68D8F8082088F80C408B4228BFE6
:203C20000B46D11A0424C8F808100E4A2C7030468121FFF7F9FDAAE73046FFF745FFA6E782
:203C40003046FFF76FFFA2E7B07400205C740020555342437C7400208074002050D6002036
:203C6000A474002048970020BC74002008B5084B1B78022B07D0033B012B02D80021FFF7BB
:203C800051FF002008BDFFF769FF002008BD00BFB074002010B501EB8101084A00EBC10177
:203CA0000446B1F88C131046F4F720FB034A204640230121FFF7E2FE002010BDF8DD002026
:203CC000E8E700BF70B50A7812F060050C46064611D0202D16D1CD88D5B113062AD52A4632
:203CE0001F496078F4F7A4FBE2881D493046FFF753FE00250AE04B780A2B16D00B2B0ED06C
:203D0000062B03D13046FAF775FD0225284670BD022260781144F4F78BFB284670BD8B78A3
:203D2000D3B9104BC3F8E857F0E70F490122FFF733FEEBE70D4964780A4AC1F8C8400321EC
:203D4000C0E9E45542F8045B2B4680F811110021FFF794FE0025D9E7FAF74CFDD6E700BF99
:203D600054D6002050D6002038DE0020F40400200B7803F00303012B03D0022B04D00020C9
:203D800070478B881BB915E68B88832BFBD099E710B50223044640228121FDF72BFB2046C6
:203DA000022340220121FDF725FB8221204603230822FDF71FFB064B02229A80F4F788FBE2
:203DC000044A204640230121FFF758FE002010BDB0010020F8DD002038B509220D460446F6
:203DE00003238321FDF706FB29462046FFF7D0FF002038BD82B00023016801930B690193FB
:203E00000E4B03E00A690192013B13D0019A002AF8DA019A094B42F001020192019A0A61ED
:203E20000A69019203E00A690192013B02D0019AD207F8D4002002B0704700BF400D0300AD
:203E4000436D064A1A61C278012A06D100F2CC5058614FF0802219681A60704718000860D1
:203E600010B5002304220446194680F811211A46FFF7DAFC2046FFF7E3FF002010BD00BFCB
:203E800010B5044629B990F81131032B0DD0002010BDD0F8E4359B69002BF8D090F81221DC
:203EA000032AF4D19847002010BDD0F89013D0F87C33994214D9C078D4F880230128A1EB3E
:203EC000030104BFD218C4F880238B4228BF0B46C4F890139BB220460021FFF7CFFDD6E71B
:203EE000D0F8E4351B691BB190F81221032A03D02046FFF7B5FFCAE79847F9E7F0B501218F
:203F000090F8D17590F8D36590F8CFC590F8CE5590F8D03590F8D22580F8111190F8CC153D
:203F200085B005EB0C2503EB072302EB062201F01F06AFB292B290F8CD558DF808109BB2AF
:203F4000012E0446ADF80A70ADF80C30ADF80E20C0F840218DF8095017D0022E1FD036B131
:203F600001F08001FFF72CFC002005B0F0BD092D0FD8DFE815F0BF00AC000E00D5000E00EA
:203F8000EA0085000E007700540090F81221032A2FD02046FAF72EFC002005B0F0BD01F0FE
:203FA00060012029DAB234D0012D00F02081032D00F00681002DD7D190F81211022900F0C6
:203FC000DF800329E5D11B0600F14B8102EB820200EBC20393F87633002B00F04D81BF4B7A
:203FE0000122C3F8FC27BE4920460222FFF7D4FCBAE7DAB2012ACCD8D0F8E43502A99B68DE
:020000040801F1
:204000009847BDF80E30002BAED12046FFF728FFAAE7D0F8E43502A99B689847A4E7F9B26C
:20402000AE4D012985F8EC17B3D890F81231022B00F02781032BACD1002900F0868190F86D
:2040400010110129E1D0D0F8E4355B68984795F8EC1784F810112046FDF73AF92046FFF7CB
:20406000FFFE81E7012A94D190F81231022B00F01781032B8DD100F58871FFF78DFC73E778
:204080003D0A022DADF8062000F05081032D00F00B81012D7FF47DAFD0F8EC3580781B6841
:2040A0000DF106019847BDF80620002A3FF45CAFBDF80E30002B3FF457AF9A4228BF1A465F
:2040C00001462046ADF80620FFF766FC4CE790F81231023B012B3FF65CAF012F7FF444AFD3
:2040E000D0F8E43500229B68C0F8182102A9204698478AE790F81231023B012B3FF649AF07
:20410000764BD0F818210021C3F8F41712B10222C3F8F427734920460222FFF73DFC23E7BA
:20412000012F00F09880022F7FF41EAF13F0FF0F7FF41AAF02691B0A023B5268032B00F2E2
:204140001D81DFE803F0393531241A437FF421AF90F81231032B3FF41CAF036907F07F05C6
:2041600080F81451196867F30A120A431A60FFF777FE002D00F0E580022384F81231F3E6FA
:2041800051063FF4F1AE1146FFF71AFBECE6052363F30612514B012184F816112046C3F8AA
:2041A000F827FFF75DFEDFE6042363F30612F1E7032363F30612EDE7022363F30612E9E792
:2041C00090F81231022BDBD0032B7FF4E2AE27B9550602D01146FFF7F3FAD4F8E43502A934
:2041E0009B68204698472046FFF73AFEBCE690F812110229C4D003297FF4CBAE002F7FF41D
:20420000B3AE12F07F013FF400AF180600F1A78002EB820304EBC30304EB810083F87673A8
:2042200083F8741383F87573282303FB0243416D03F55D73DA780B68023A6FF35553012ADF
:20424000D4F8E42598BF43F080530B602046936802A99847D9E6D0F8E435C0F818719B68F2
:2042600044E702F07F0202EB820200EBC20393F81E31002B7FF4B3AE184B0022C3F8FC2743
:20428000B1E600293FF4C1AE0121032380F8101180F81231FDF71CF82046FFF7E1FD63E695
:2042A0001149FFF779FB5FE6FDB2052D3FF671AEDFE805F0342C241C0B03D0F8EC35807875
:2042C0009B690DF106019847EDE6D0F8EC3580785B690DF106019847E5E600BF50D60020CA
:2042E0004CDE002044DE002040DE0020D0F8EC3580781B690DF106019847D4E6D0F8EC3508
:204300008078DB680DF106019847CCE6D0F8EC3580789B680DF106019847C4E6D0F8EC3571
:2043200080785B680DF106019847BCE6D0F8E43580789B6A0DF1060198474570C4F8F00514
:20434000B1E6012384F812310EE60222D0F8E43580F8101180F812215B68984755E628227F
:2043600002FB014304EB810083F81E7183F81C1183F81D51816903F58E735BE7012363F352
:20438000061207E770B5044649B990F81131022B1BD094F81631012B0DD0002070BDD0F8D3
:2043A000E4355B69002BF8D090F81221032AF4D19847002070BD2A4A2369D2F8F8275A60B1
:2043C000002384F81631002070BDD0F83831D0F82451AB4217D9C278012AD0F82821A3EB5B
:2043E000050308BF5219C0F8383108BFC0F828219BB20021FFF718FA00231A4619462046DC
:20440000FFF73CFBC5E7D0F83C31B3FBF5F605FB163666B99D420AD8D0F84021934206D2F3
:2044200033463246FFF700FAC4F84061E4E7D4F8E435DB681BB194F81221032A0CD0002394
:20444000052284F8112119461A462046FFF716FB2046FFF7F5FC9CE720469847EFE700BFB1
:2044600050D6002082B000230193019A094B42F010020192C168019A0A610A69019203E02F
:204480000A690192013B02D0019AD206F8D4002002B07047400D030082B000230193019A6C
:2044A0000B4B42F020020192019A61F38A120192C168019A0A610A69019203E00A69019283
:2044C000013B02D0019A9206F8D4002002B07047400D0300F8B50B7813F060050C460646C0
:2044E0001CD0202D17D14A78FE2A44D0FF2A3DD14A88002A56D1CD88002D53D11B0651D457
:204500003749384B0D70012183F8A417364A1F23FFF7B4FA00E000252846F8BD4B780A2B3D
:204520004BD00B2B44D0012BF6D191F904308988002B47DBFFF796FF21792A4F3046FCF700
:20454000F5FE0223217940223046FCF753FF97F8A437022B3BD094F90420002ADCDA012B2D
:20456000DAD030460121FFF7DDFAD5E70225FAF741F92846F8BD4D88A5B9CC88012C11D165
:204580001A060FD5194B1B689B6998471549C0B281F8000830B1224601F500613046FFF7F0
:2045A000FBF9B9E730460225FAF724F92846F8BD0C4B4A8883F80128AEE70D490122FFF7C8
:2045C000EBF9A9E701F07F01FFF766FFB4E730468121FFF7F5F8002387F8A4379CE700BF46
:2045E000B074002050D600205C740020A074002051DE002038B50446FCF7CEFE204602233D
:2046000040228121FCF7F6FE2046022340220121FCF7F0FE0C4B0D491B680D4A00250D7096
:204620001B6882F8A457284698472046FFF71AFF20460121FFF730FF064A20461F230121F9
:20464000FFF71CFA284638BDA0740020B074002050D600205C740020012905D008B503215D
:20466000FFF71AFF002008BDFFF752B90B88F0B433BB028C4C880E898B88C98822F00102AE
:204680001204120C0284058B028CADB225F0F30592B22B4322F00A0243EA061322439BB20E
:2046A00042F0010203830284038B23F00C031B041B0C0383038B9BB21943F0BC018370471F
:2046C000042B048C2CD0082B4E888A880D89C98851D024F480542404240C0484838B078C8F
:2046E0002C0344EA022440F6FF421A4045F6FF733B4043EA063322439BB292B243F48053D8
:2047000082830384828B22F440621204120C8283838B9BB243EA01239BB2F0BC83837047AD
:2047200024F010042404240C4D880F898A88C9880484068B038C12029BB242EA073423F0A6
:20474000A00340F6FF42324043EA051322439BB292B243F0100302830384028B22F44062FB
:204760001204120C0283038B9BB243EA01239BB2F0BC0383704724F480742404240C048432
:20478000848B038CA4B29BB224F0F30423F42063224343EA062342EA05129BB243F48073BE
:2047A00092B282830384838B23F00C031B041B0C8383838B9BB21943F0BC8183704700BFD0
:2047C000214A038890429BB212D002F5806290420ED0B0F1804F0BD0A2F58032904207D01C
:2047E00002F58062904203D002F58062904203D14A8823F070031343144A904218D002F5FF
:204800008062904214D030B423F440730C894D6802F56C429BB2234390420C880380C562A0
:2048200004850DD18B7A0386012330BC8382704703800B884A68C262038501238382704763
:20484000034B9842EED0EFE700000140001000400004014000B583B009238DF80730FCF703
:2048600079FF8DF807009DF80730012BF7D09DF8070003B05DF804FB82B0064B002201929A
:204880000193019B03EB80000190019B186802B0704700BF5028004082B0064B00220192B5
:2048A0000193019B03EB80000190019B196002B0704700BF502800400023C0E90033C0E92C
:2048C0000233C0E90433C0E90633C0E90833C0E90A33C0E90C338363704700BF0B6870B43C
:2048E000D1E90524CD682B431343D1E9072523431343D1E909422B43D1E90D6523431343DF
:2049000004680B4A334322402B4313430360D1E90B3442690D6922F0070223431343D1E92C
:20492000014243614560846070BCC260704700BF3F801CF002683649002310B422F0010293
:20494000212488420260036043608360C3600361446138D02F4B98422ED02F4B98423CD017
:204960002E4B984240D02E4B984232D02D4B984241D02D4B984246D02C4B984217D02C4B05
:2049800098423CD02B4B984216D02B4B984224D02A4B984228D02A4B98421AD0294B9842E9
:2049A00029D0294B98422ED0284B984208D14FF03D5243F8AC2C03E04FF4746243F8202C28
:2049C0005DF8044B7047224B5DF8044B3D229A607047204A43F8642CF2E74FF474125DF82F
:2049E000044B43F8382C70474FF074625DF8044B43F8502C7047184A43F87C2CE0E73D2280
:204A000043F8082CDCE7154A43F8942CD8E700BF1060024028600240406002405860024034
:204A20007060024088600240A0600240B86002401064024028640240406402405864024036
:204A40007064024088640240A0640240B8640240006002403D000020400F002000003D20A3
:204A6000024A536A23EA00005062704700380240024A136A23EA00001062704700380240C4
:204A8000484B98422ED0B0F1804F32D0464B984236D0464B98421ED0454B984237D0454B6E
:204AA00098423BD0444B98423FD0444B98424BD0434B984240D0434B98424CD0424B9842B2
:204AC00051D0424B984256D0414B98425AD0414B98425ED07047404A136A43F00403136297
:204AE0000420C5E73C4A536A43F0010353620120B6E7394A136A43F0010313620120B7E78E
:204B0000354A136A43F0020313620220B0E7324A136A43F0080313620820A9E72E4A136ADA
:204B200043F0100313621020A2E72B4A136A43F02003136220209BE7274A536A43F480336A
:204B400053624FF480308BE7234A536A43F002035362022084E7204A536A43F40033536251
:204B60004FF400307CE71C4A536A43F4802353624FF4802074E7184A136A43F040031362A5
:204B8000402075E7144A136A43F08003136280206EE7114A136A43F4807313624FF48070B4
:204BA00066E700BF000001400004004000080040000C0040001000400014004000040140E7
:204BC00000400140004401400048014000180040001C00400020004000380240224A936851
:204BE00003F00C03042B10B421D0082B22D01F4B03601D4C1E4AA168C1F30311114491F85D
:204C00006C11CB404360A168C1F38221114491F86C1123FA01F18160A1685DF8044BC1F35D
:204C200042310A4492F86C21D340C3607047114B0360DEE75468516852686302C2F3881248
:204C40004CBF0C4B094B01F03F01B3FBF1F303FB02F3054A5268C2F3014201325200B3FBB4
:204C6000F2F30360C5E700BF003802400024F400F404002000127A002DE9F04700230F6864
:204C800001264FF0030C02E00133102B41D006FA03F232EA0704F7D1D0F800E05C000CFA4F
:204CA00004F52EEA050EC0F800E091F80490D0F800A009FA04FE09F1FF394EEA0A0EB9F182
:204CC000010FA846C0F800E06FEA050515D8D0F808E005EA0E0585604D79D0F808E0A540FC
:204CE00045EA0E058560456825EA020242608A7945689A4092B22A434260C26822EA08020E
:204D0000C260CA79C568A24001332A43102BC260BDD1BDE8F0870B4B93F8B825D20703D508
:204D2000012283F80228704793F802284AB9D3F81C3633B1044B1A7810445A781870114457
:204D40005970704750D600201874002010B50E4C40F0080284F8802194F9CE20022A06DDE1
:204D6000420704D583071CBF012384F8D63005210648FCF7FDFD062184F88101BDE810408B
:204D80000248FCF7DDBD00BFF40400207006002010B5FCF785FDA8B31B4C94F9CE30012B1C
:204DA00030DD59B3022B2DD094F8D6309BB971B180230521154884F88631FCF7D9FD06215F
:204DC00084F88701BDE810401048FCF7B9BDBDE810400420BAE7002914BF0020042094F893
:204DE000D1301A0748BF40F002005B0701D411B108B940F00100BDE81040A7E7022BD3D119
:204E00000420ECE710BD00BFF404002076060020F8B5224C04F5C477030A84F88D010546AA
:204E20000621384684F88C31FCF7A2FD94F8D13084F88E01DB072AD4B4F8D220AA4226D109
:204E4000174DD4F88831C5F80338C3B285F8093841F26F714FF6FF738A4218BF0123134456
:204E600005F60306C3F307220621304685F8072885F80838FCF77CFD072185F809083046B1
:204E8000FCF75EFD052104F28F10FCF759FDBDE8F84004480721FCF753BD00BFF404002095
:204EA00050D600207C06002008B5FCF7F9FC48B1A1F59C53083BB3F57A7F03D2BDE8084041
:204EC0000846A5E708BD2DE9F0476B4E3368002B3AD06A4D6A4C05F1CE0730683BF0D8FF8B
:204EE000002833D1674B198809291D4609D95F8864227A43B2FBF1F2452A40F3A1811880A6
:204F0000588094F84138012B00F0C581022B00F0E08133B95C480521FCF712FD012384F87C
:204F200041385A4B1D685A4B1B78002B00F0DB81584B1B68EB1A782B40F2D581D4F83406C3
:204F4000F9F722FCC4F84458BDE8F08730683BF097FF94F80A388046052BBED8DFE803F062
:204F60000309171D3745AA28B7D1012384F80A38B3E7552803D1022384F80A38ADE7414A4C
:204F8000938801339380002384F80A38A5E7032384F80B0884F80A389FE7132884F80C087E
:204FA000C4F8240807DD374AD3880133D380002384F80A3891E718B9052384F80A388CE73F
:204FC0000023C4F82838042384F80A3885E7D4F82838E218013382F80D08D4F82428C4F884
:204FE000283893427FF479AFE6E7D4F824382A4803F1020A4FFA8AF1FCF7BAFC804594F8BC
:205000000B9840F01481262020F056FD204B48B100221A701B4A538801335380002384F889
:205020000A385AE71A784A4519D100221A7009F1FF33102B00F2F680DFE813F030008E00DF
:205040008E00DE008E00F400F400F4003000F400F400F400F400F400F400F4003000B9F1C4
:20506000090F02D0B9F1110F01D1012ADDD0054A538901335381DAE714740020F40400201E
:2050800050D600204274002083060020CC2B002050740020547400205BDE0020BAF1060F4F
:2050A0005ADDB9F1010F06D0B9F1090F0CBF4FF002094FF0030994F8100894F8111894F822
:2050C0000F2894F90DE894F90FC894F80E3885F8CE9041EA002109B2900785F8CFE085F8BF
:2050E000D1C0A5F8D21006D512F00C0F14BF0122002285F8D620B9F1030F13D1BAF1090FBA
:205100002ADD94F91328082AA8BF082222EAE27285F80421002043B29A4200F1010059DCE3
:2051200094F81238D4F828A0002002469BB25245904657DB7C4B85F8D0001B78232B0BD1E0
:2051400009EB8903794A03EB83030CEB83031380A2F802E09180D080754976480A2258F0BB
:205160008EFC10B1002384F83638714B3A681A607A685A603A891A8194F836382BBB95F898
:20518000D6306D4A002B14BF0223012384F8363895F8D130117884F8381813F001031CBF5C
:2051A000B1FA81F35B09517884F83918D8B29188927884F83708A4F83A1884F83C2813B1DC
:2051C00009B1A4F83E1884F840080DF089FE0DF087FE1FE704EB4308234493F81538A8F83A
:2051E000223698E704EB48080132B8F82C8052B2984508BF10469AE7BAF1040FACDD94F8B8
:205200000D2894F80E3843EA022359041AB204D5C3F30D03A5F8D4309EE7002AF8DBA5F8AD
:20522000D23099E7454A938901339381F2E619F0010F7FF4F3AE414A138901331381EDE632
:205240003F4BD3F89421B3F89811012A1AD141F25632914203D14FF0FF32C3F89421D3F8CD
:205260009421306802EB820202EB820201EB420189B2A3F8981103681B69984700232B80B5
:205280006B803EE60132EAD1B1F5965F04BF0122C3F89421E3E72A4D95F9CE60002E3FF4C2
:2052A00040AE022E11D14FF48040FFF7B1FD84F8416895F9CE30012B7FF733AE95F8D13085
:2052C000C3F3400385F8D6302BE6032384F84138EFE71B4BB3F8D430002B3FF422AE0323E7
:2052E00084F841381DE694F8402094F841309A4204D0FDF763F9C4F8445825E6D4F8443822
:20530000EB1AB3F57A7FBFF41FAE0E4B1B68ED1A952D7FF619AE0C480521FCF711FBBDE868
:20532000F047FDF74BB900BF404A0020484A00207CDE0020C2050020187400204274002040
:20534000F40400205474002083060020104BD3F81C0610B5D8B10F4C217841B162780CF052
:20536000FBFEA38883421ABFA08001210021E2885AB141F288339342B8BF13469A4204D050
:20538000E380BDE8104043F0F7BD0029F9D110BD50D600201874002010B4014404460020A9
:2053A00014F8013B08225840430010F0800F08BF400083F0070314BFD8B2C0B2013AF3D1BF
:2053C0008C42EDD15DF8044B704700BF30B54FF4806085B035F0A6FA40B3154C90F9040044
:2053E00094F84838134A002B18BF08234FF4E1310125CDE90153009100234FF4806135F095
:20540000F2FAFF23E067003818BF012084F8F83484F8083584F8183584F8283584F838351B
:2054200084F8483584F8583584F8683505B030BD50D60020291C0108374B1B6813F00063B0
:205440005CD02DE9F04F354B1F78B84251D3FF2856D1334B93F8DE30002B47D0DFF8D4A0A4
:205460000022CAF84C28CAF85028CAF85428AAF85828002F4CD00AF59F63104614461146E7
:205480001546164603EB071BB946B3F802C09F8993F8008093F901E061443A444645D3E9CF
:2054A00001C738BF464610337545B8BF75469B4509B212B264443844E7D191FBF9F192FB34
:2054C000F9F28AF84C688AF84D58CAF85048CAF85408144BAAF84E181B781149AAF8582896
:2054E000092B4FF0000281F8DE200CD00E48BDE8F08F0E4A02EB0010BDE8F08F18467047DC
:205500000020BDE8F08F0A4B9AF84C28DA80EDE73A463946DDE700BFF46E002078500020D2
:20552000F4040020404A00209CDE002048DB0020484A002050D600200268F8B53A4E3B4CAE
:20554000B6F95C38511C01607E2111700168054603EBC30384FB0302481CDC17002328602C
:205560000B70FF20C4EB6204FFF766FF2034304BA4B200284DD01B78B0F90C1023BB2D4B09
:20558000A1F57A729A4246D82B48B0FBF1F189B2284642F09BFF96F897357BB12AF020FE5C
:2055A0000146284642F092FF2146284642F08EFF28460821F8F780FB0120F8BDB6F84816FC
:2055C000284642F083FFEFE71C4B1F78002FD6D01B48002300EB830201339289BB42114469
:2055E000F8DB184B9FED186A93F8223007EE103A07EE901AB8EEC77AF8EE676AC6EE077AD9
:2056000067EEA67AFCEEE77A17EE901AB1FBF7F1B5E71B7813B94EF69C21B9E7074B1F7802
:20562000002FF8D00146D3E750D6002067666666556A00201783930300879303785000207F
:20564000B0DE0020A82C0020000048432DE9F8434A4C427894F8E43802F00F05C3B9EDB9AC
:205660002B46002184F8E818EB1AD9B20E290BD8234493F8981539B102F0F002802A4AD041
:20568000902A5FD0A02A0DD000273846BDE8F8830021AB4284F8E818F6D8E5E784F8E458D9
:2056A0002B46DEE7412966D081F08003042B62D90846FCF7D3FA031D0246DBB2304884F8BF
:2056C000E83865F05F0584F8E958FDF711F994F8E878002FD8D0BE1E16F0FF0024D1FF2579
:2056E000A946022756B1DFF89C80464418F8011BD4F80C093BF0D0FB4645F7D1D4F80C09D7
:2057000049463BF0C9FBD4F80C0929463BF0C4FB3846BDE8F88365F07F050427022684F88B
:20572000E95884F8E8783046164A4FF6FF71104412F8015B491B904289B2F9D15FFA81F9F9
:205740000D0ACFE7412914D081F08003042B10D90846FCF783FA65F06F050627042684F8C8
:20576000EB0884F8E95884F8EA1884F8E8783046DAE70420EFE7082304229FE750D60020D1
:205780003ADF002038DF00202DE9F04FC31D85B0544C03F4FC7300AFADEB030DD4F81039BD
:2057A00004F5126B0DEB00025B4506468A46FA60E9462FD094F8601A94F861CAD4F814593F
:2057C00001F00F0040EA4C1001310DF101088DF8000084F8601AC7F8088007F10800ED1A41
:2057E000A2EB0808A845194644DD2A4642F04CFED4F81029B968C4F810B92A44A1EB090104
:205800004846C4F81429C9B2D04700201437BD46BDE8F08F94F860CA94F8610AB4F91A5910
:205820000CF00F0141EA401141F01001002DC9B2D4F81459B8BF41F080010CF1010C012861
:2058400084F860CA89F80010A5EB0B0822D1B8F1FE0F3ADDFF2394F8182989F8013007F115
:20586000080009F103031FFA88F1786089F80220BB6020E0424642F007FED4F810294244AE
:2058800048463146C4F81029D04701201437BD46BDE8F08F94F81C39B4F8181989F80130F4
:2058A00007F1080009F102037860BB6042F034FE78681FFA88F142F02FFED7E90282D4F8B1
:2058C0001459D4F81039786889E794F8181989F8018009F1030889F80210C7F8088007F160
:2058E00008007CE750D6002001297FD9F0B50378654CC3F34115032D83B084F8615A03F00B
:205900000F0700F0848013F01003164606D0012D6ED0052912D8002003B0F0BD94F8342B46
:20592000002AF8D094F8352B013202F00F02BA4255D0184684F8343B03B0F0BD437884F852
:20594000303B4388A4F82C3B85884318811DC02D7ED84E4AC4F8242B15444FF0000C01205D
:20596000C4F8285BA4F82ECB84F8340BAA1A5B1A934284F8357B66DB454D002A5CD1B4F987
:205980002C3BFA2B53D0414A4249D4F8243BD1F89C01C4F8242B2946151FA2F5A276C4F898
:2059A0001459C4F8283B0025A2F5AA7201ABC4F8106984F8345BC4F8185901952BF018FFA2
:2059C000013058D0019B0BB100209847D4F81039C4F814390120C4F8106903B0F0BD4318E8
:2059E000D4F8285BD4F8242B411CBFE700207047022990D045788378A4F82C3BFF2D1FD101
:205A0000042988D94318B0F80350411D9FE70023214984F8203904F5126204F62113C4F805
:205A20001819C4F81029C4F81439012074E7002EA9D005233370A6E7284642F025FD9EE775
:205A40004318C11C83E712481A4642F01DFD62E7124BB4F82C0BC4F81039032101334FF673
:205A6000F672A4F81809C4F8143984F82019A4F81A29012050E7D4F810390222591CC4F8A2
:205A800010191A709EE700BF50D60020B4E0002074E10020F40400200000F6FF70DF002024
:205AA0000B4B93F86A2612B1B3F8A8254AB9B3F9E836084AD81782FB0323C0EBA30000B289
:205AC0007047D3F8840690FBF2F000B2704700BF50D6002067666666F8B5184CC6B2054672
:205AE0003146D4F8380B3BF0D7F994F83C1BD4F8380BC5F307274E40394684F83C6B3BF0F2
:205B0000CBF994F83C1BD4F8380BC5F307464F40314684F83C7B3BF0BFF994F83C1BD4F8FF
:205B2000380B2D0E4E40294684F83C6B3BF0B4F994F83C1B4D4084F83C5BF8BD50D6002071
:205B400070B50C4DC6B231460446D5F8380B3BF0A3F995F83C1BD5F8380B240A4E402146A0
:205B600085F83C6B3BF098F995F83C1B4C4085F83C4B70BD50D6002038B50B4C00230546AC
:205B80002421D4F8380B84F83C3B3BF085F9D4F8380B54213BF080F9D4F8380B2946BDE8CA
:205BA00038403BF079B900BF50D600202DE9F043DFF894932DED028B99F83D4B83B00E467D
:205BC0001546002C00F03982013C89F83D4B9FEDD88AD84FDFF874833378002B62D099F8D1
:205BE0003D4B002C5ED135B13AF066FC2B68C01A002880F2028499F83E4B002C40F0A68324
:205C000099F83F0B062840F2D781CB4A92F8A53192F8A411994200F00082D2F8A01199F8E4
:205C200040CB31F8134064440130013302F5D072A4B2C0B2DBB2B4F5E06F89F83F0B5371BB
:205C400000F0D18100F2AA80B4F5806F00F0F88264D9B4F5A06F00F0CC823CD9B4F5A16FE3
:205C600025D8601EC0B2FFF7E7FBC8B1B0F90C30B24AADF8014092F82210D9F8842503EBFB
:205C8000830303EB830349089B0093FBF1F31021CDF803308DF800106846904700233370A3
:205CA000002D99D103B0BDEC028BBDE8F083B4F5C06FF5D1B9F86C36002B00F054832AF04F
:205CC000A7FA10220024CDF8030006238DF800208DF801401FE2B4F5826F00F05082B4F56B
:205CE000846F40F0358199F844369A07D8D5B9F84636CDF803301021202204238DF800101E
:205D00008DF801208DF80230D9F884356846002498473470002D7FF45FAFC3E7B4F5067FC1
:205D2000BED8B4F5007FC0F02C81A4F50073182BB6D801A252F823F0B5600108A360010841
:205D4000A3600108A3600108A3600108A3600108A3600108A3600108A3600108A15C0108E9
:205D6000A15C0108A15C0108A15C0108A15C0108A15C0108A15C01087F6001086960010845
:205D800069600108696001086960010869600108696001086960010869600108B4F5116F1C
:205DA00000F0E0815BD8B4F5026F00F0BF8121D9B4F5036F00F07282B4F5046F7FF470AF6E
:205DC000B9F9E836D9F8842503EB83035B001020CDF80330402108238DF800008DF80110DB
:205DE0008DF802306846002490473470002D7FF4F3AE57E7B4F5E46F00F07881B4F5006F23
:205E000076D199F8442691077FF54AAF13F0010F4B4B00F005835A6882EAE273A3EBE273B4
:205E200003EB5303A7FB0313DB08002AACBF43F0004343F04043102100240822CDF803304B
:205E40008DF800108DF80140D9F884358DF80220684698473470002D7FF4BEAE22E745F239
:205E600030239C4200F0B1811DD945F240239C4200F0298245F250239C427FF411AFD9F83A
:205E80008436CDF803301021502252238DF802308DF80010D9F884358DF8012068460024EA
:205EA0009847347036E7B4F5376F00F031826FF437616318072B3FF6F3AEA4F17100C0B25A
:205EC000FFF7BAFA00283FF4EBAE90F90130CDF8033010238DF80030ADF80140D9F884351A
:205EE0006846984700233370002D7FF475AED9E6B4F5E26F7FF4D4AE124B93ED130AD3ED24
:205F0000007A20EE270A002420EE080A56F0DAFA10230722CDF803008DF800308DF80130DB
:205F20008DF80220D9F8843568469847347092E70000C8421F85EB51F4040020A82C002090
:205F4000706F0020DCDC002050D60020C5B3A29140F201439C427FF4A3AEB9F95C38CDF856
:205F600003301021012204238DF802308DF80010D9F884358DF801206846002498473470A2
:205F8000C8E6B4F5807F00F01481B4F5887F7FF487AEB9F9EA36CDF80330012210238DF829
:205FA00000308DF801308DF80220D9F884356846002498473470ADE60130CD4AC0B292F89E
:205FC000AD1192F8AC318B4222D04B1CDBB24900D2F8A841C74A645A89F83F0BB4F5E06F5B
:205FE00053717FF42FAEC44B93ED120AD3ED007A20EE270A002420EE080A56F063FA102250
:020000040801F1
:206000000723CDF803008DF800208DF8014082E0002182F8AD110123DAE7B84999F8403B76
:20602000097882F8A5410133DBB201318B4289F8403B00F087810120C1E700283FF4C7AD33
:206040000378303B012B3FF6C2AD013009F63D320621FFF749FC99F83D3B89F83E0B002B8B
:206060003FF4B5AD3470B2E5A4F11100C0B2FFF7E3F900283FF414AEB0F9023027E799F8CF
:206080009735002B40F0B081B9F84806CDF80300102302228DF800308DF801308DF8022078
:2060A00083E7601EC0B2FFF7C7F900283FF4F8AD43680CE7D9F87C369149D9F8842581FBDF
:2060C0000301DB17C3EBA10300241021CDF8033002238DF800108DF801408DF80230684646
:2060E00090473470002D7FF477ADDBE5824B93ED140AD3ED007A20EE270A002420EE080A79
:2061000056F0E0F9102320228DF80030CDF8030007238DF801208DF802306846D9F88435AF
:2061200098473470002D7FF457ADBBE599F844369B077FF5B5AD734AD9F884359268CDF80F
:206140000320102220218DF8002008228DF801108DF802206846002498473470002D7FF4A8
:206160003BAD9FE52AF03CF810230922CDF803008DF800308DF801308DF8022015E7D9F860
:20618000803513F0200440F0F1805F4B1B681B0640F13981102304228DF803408DF804405F
:2061A0008DF805408DF806408DF800308DF801304AE6D9F8443BCDF80330102200240123ED
:2061C0008DF800208DF80140A5E7B9F9E636CDF803301021302252238DF802308DF80010BE
:2061E000D9F884358DF80120684600249847347090E5FF20FFF720F900283FF451ADB0F975
:206200000C304249D9F8842591F8221003EB830303EB83031020490800249B0093FBF1F3E8
:2062200005218DF80000CDF803308DF801408DF80210684690473470002D7FF4CDAC31E506
:2062400099F8483B0133DAB2042A00F0D08042F2107389F8482B03FB02F3D9F84C2B002AEC
:2062600000F0C080023399F8B825D207B9F8882648BF0433D40748BF0A33900748BF1433D1
:20628000D10548BF2833540748BF6433500648BF03F57A63102100240422CFE599F8443661
:2062A00098077FF5FDAC174BD9F88425D9894FF4F36303FB01F3A7FB03135B091020CDF848
:2062C0000330302187E5B9F9E436CDF803301021402252238DF802308DF80010D9F884352C
:2062E0008DF80120684600249847347012E500BFF40400209C060020DCDC00207850002053
:2063000067666666706F0020F46E0020A82C0020FF20FFF791F800283FF4C2AC90F901304E
:20632000CDF80330102170220B238DF802308DF80010D9F884358DF8012068460024984747
:206340003470E7E489F8404B012038E65C490620FFF71AFA002389F83E0B337003B0BDECC2
:20636000028BBDE8F083D9F88406AAE4554A99F84416538A643BC3EB4370C3EBC00388FB34
:2063800003401844DB17C3EB20230933092BA8BF092323EAE37303EB830311F0020F03EBA1
:2063A000830314BF4FF47A7000209B00C90748BF00F5FA60117DD9F884259BB203440B448B
:2063C000042010218DF80200CDF803308DF800108DF801106846002490473470002D7FF4D1
:2063E000FBAB5FE401333EE729F0FAFE4EE6012389F8483B42F210732FE7347003B0BDEC21
:20640000028BBDE8F08399F89635002B3FF448AC99F8503B032B4ED8DFE803F043392A1148
:206420001A6882EAE273A3EBE27303EB5303A7FB0313DB08002AB8BF43F08043FBE4D9F810
:20644000582B537A907AD17A03F1407303EB0023002203EB014389F8502B10220421CDF873
:2064600003308DF800208DF801208DF802104BE4D9F8541B8A7D087C897A120402EB0022E5
:206480000A44591C89F8501B02EB0363E5E7D9F8541B4A7DC87B497A120402EB00220A44AE
:2064A000EFE7D9F8541B0A7D887B097A120402EB00220A44E5E75A1C89F8502B1B06CCE734
:2064C0000D1D0108706F002030B5A0F17D03012B044683B00D46104608D921463AF0DCFCF8
:2064E00015B1288804442C8003B030BD7D2101923AF0D2FC019884F020013AF0CDFCEFE772
:2065000030B50F4B85B0D3F8B42500230446C51DADF80E3014F8010B01920DF10E01FFF783
:20652000D3FFA542019AF5D10DF10E0016F02CFC019A9DF80E000021FFF7C6FF05B030BD4B
:2065400050D600207E28F8B50F4652D0324E96F8B04164B9314D95F8641B51B11B2885F8C3
:20656000644B3DD00D2837D0012386F8B0310020F8BD7D284AD095F8682B1AB180F0200091
:2065800085F8681B95F8632B062A14D8B5F8664B511C2A440444C9B2A5F8664B85F8631B7F
:2065A00082F85C0B002BE2D10729E0D101231C4886F8B031F8BDB5F8663B1844C0F3072318
:2065C00053FA80F0FF284FF00103A5F8660B86F8B031CCD11248F8BDA5F8664B2046F8BD12
:2065E00090470028C0D0012320463B7086F8B031F8BD0A4B084A0024012183F8634B83F832
:20660000641B3C7082F8B0412046F8BD0123084685F8683BF8BD00BFF404002050D6002065
:20662000ACE10020044AD2F86C3B43F4DF2343F48063C2F86C3B704750D60020013070B5E7
:20664000094EC4B203E045F059FB013448B9E5B2152D21463046F6D9162D04BF034B93F867
:20666000705B284670BD00BFBCE1002050D6002000B1D7E7044AD2F86C3B23F4DF2323F494
:206680008063C2F86C3B704750D6002070B5114C84B00546D4F8740B0E4634F001F994F86F
:2066A000902594F89135003A18BF01220BB142F00802CDE9016200234FF4964195F90000C3
:2066C00000911A46082134F08EF9C4F8740B04B070BD00BF50D6002010B5064C03E0D4F80E
:2066E000740B3AF0CDFBD4F8740B3AF0D1FB0028F5D110BD50D6002010B50D4CD4F8783B4A
:206700001B791E3B012B0DD9D4F8740B01213830FFF7BCFF0023C4F87C3B84F8803BBDE882
:206720001040D9E7D4F8740B01213AF0A1FBF1E750D600200B2814D810B401EB4103094C90
:2067400001EB83032344184490F8FC36934205D02144002380F8FC2681F8F0365DF8044B3B
:206760007047704750D60020F0B5444C94F8813B012B83B005464FD994F8821B4048DFF88E
:2067800010C194F8837B4A1CA0FB026000F4FE7606EB90001944121A5CF8216084F8822BCB
:2067A0002FB1D4F8841B04F6883291420DD06EB9344A0133A2FB031222F0010101EB52024B
:2067C0009B1A84F8813B03B0F0BD2F4E94F89C3B93B92E4B019348F2A501123B15226F461A
:2067E000A4F8A01B009384F8A22B29463846B04758B994F8813BDBE76F46384615F092F9A4
:2068000029463846B0470028F3D094F89C1B49B1384615F001F9ECE71D4A52F82360002EBA
:20682000C6D0D3E7009E1B4A964214D9013A013E41F2210512F8013F81EA0321082311F464
:20684000004F85EA41000ABF490081B289B2013BF5D19642EED1384641F05EFE0E49009D21
:206860006D1A152DA8BF15252A4601F1180057F0CDF894F8813B84F8CD5B99E750D6002076
:20688000CDCCCCCCABAAAAAA7D2D010805E200202CDD0608F3E10020F0E1002070B50C4EE9
:2068A000054606F6D231D52242F0ECF92C686C6006F53D61641A182CA8BF18242960224631
:2068C00006F6E83057F0A2F886F8004C70BD00BF50D60020026810B40421541C046011701F
:2068E00002680B24511C016014705DF8044BC82141F0ECBD70B50C4E054606F60641D52242
:2069000042F0C0F92C686C6006F60441641A402CA8BF40242960224606F6444057F076F810
:2069200086F8844C70BD00BF50D6002010B5104B0A4682B001467B24101D83F8050C83F81B
:20694000064C93F8850C83F8070C03F6444403F609400194C824009083F8044C684683F873
:20696000084C41F091FD6846FFF7C4FF02B010BD50D60020F0B5454C94F8883CD90785B03D
:2069800005463BD594F8893C0F2B5AD9002217463F4E94F8883C84F80C2CA6F13702CDE948
:2069A0000226C3F3820340F6C822DFF8F8C084F80B3CA6F13E01712302A8A4F8082CBA2242
:2069C00084F80A3CC4F804CC42F05CF9029A3F3E961B84F8056C15F0C7F802A8FFF78AFF3E
:2069E00015F0C2F894F8883CC4F88C5C23F0030343EA470384F8883C05B0F0BD9A0728D514
:206A0000D4F88C0C2D1AB5F57A6FF5DB94F8893CD4F8900C0F2B97BF1E4A1F4902EB8303DC
:206A2000D969036801911B69984701990620FDF733FF94F8883C6FF3410384F8883C05B0E3
:206A4000F0BD164B93F834301F1E18BF01273A469EE7134B1B685B05CED4104B93F83430CB
:206A6000002BC9D004F6444104F60542C82302A8CDE9022184F8043CFFF72CFF15F074F8D6
:206A800002A8FFF737FF15F06FF8B5E750D6002094E200202CDD0608A0680600646700202C
:206AA000F46E0020C80032EC044BD3F8AC3530EA030314BF01200020704700BF50D6002083
:206AC000AB4A38B50820002382F8AD31FFF7ECFF002800F08C80D2F8A8314FF48061022043
:206AE0004FF48264198082F8AD0101465C804FF40020FFF7D9FF50B14B1CD2F8A801DBB2F0
:206B000040F2014482F8AD3120F811401946994C94F86936002B6CD194F86A36002B40F0DF
:206B200088804FF40070FFF7BFFF50B14B1CD2F8A801DBB24FF4046582F8AD3120F8115001
:206B40001946D4F88045A50700F11881600700F1EB80894B1B681B0600F1A38000234FF45A
:206B6000803082F8AC1182F8AD3182F8A531FFF79BFFD0B3D2F8A03101214FF4047082F885
:206B8000A51118804FF40040FFF78EFF50B14B1CD2F8A001DBB24FF4007482F8A53120F822
:206BA000114019464FF40030FFF77EFF50B14B1CD2F8A001DBB24FF4A06482F8A53120F830
:206BC000114019464FF48020FFF76EFF38B1D2F8A0014FF437644B1C20F81140D9B200230F
:206BE00082F8A41182F8A53138BD0146CAE701467DE70120FFF758FF00288DD04FF4803098
:206C0000FFF752FFD2F8A85128B94FF4047325F811300131C9B20BB2481CC1B24FF411607C
:206C200082F8AD1125F8130094F86A36002B3FF478AF0220FFF738FF00283FF472AF4FF42D
:206C40000040FFF731FF50B94B1CD2F8A801DBB24FF4007582F8AD3120F811501946042052
:206C6000FFF722FF50B14B1CD2F8A801DBB24FF4C06582F8AD3120F8115019464FF480102A
:206C8000FFF712FF00283FF44CAF4B1CD2F8A801DBB245F2502582F8AD3120F81150194654
:206CA0003FE74FF40050FFF7FFFE50B14B1CD2F8A801DBB24FF4036482F8AD3120F8114055
:206CC00019464FF48050FFF7EFFE68B1D2F8A8014B1C4FF40064DBB28D1C20F81140E9B28B
:206CE00082F8AD1120F813404FF48040FFF7DCFE50B14B1CD2F8A801DBB24FF4846482F811
:206D0000AD3120F8114019464FF48060FFF7CCFE00283FF423AFD2F8A8014FF402644B1C3A
:206D200020F81140D9B219E74FF48060FFF7BCFE50B14B1CD2F8A801DBB24FF4807482F873
:206D4000AD3120F8114019464FF40060FFF7ACFE00283FF4FEAE4B1CD2F8A801DBB24FF499
:206D6000887482F8AD3120F811401946F1E600BFF404002050D60020F46E00208020FFF7EB
:206D800093FE50B14B1CD2F8A801DBB245F2302582F8AD3120F8115019464FF48070FFF715
:206DA00083FE50B14B1CD2F8A801DBB245F2402582F8AD3120F8115019461020FFF774FE86
:206DC00050B14B1CD2F8A801DBB24FF4E06582F8AD3120F8115019462020FFF765FE50B1F9
:206DE0004B1CD2F8A801DBB24FF4E26582F8AD3120F8115019464020FFF756FE00283FF46D
:206E0000A5AE4B1CD2F8A801DBB24FF4E46582F8AD3120F81150194698E600BFF0B5CA4C04
:206E200094F8983CD4F88015C4F8940C0133880785B084F8983C12D411F0340F35D10907AD
:206E400094F8982C42D412F007055BD0282A00F0DB80D4F888355E20984705B0F0BD70201E
:206E6000FFF722FE0028E7D004F2D466242504F28C67F6EC017A97ED007A67EE877A28469C
:206E8000FDEEE77A013517EE901AC1EB411301EB8301C90009B2EDB2FAF774FF272DE8D1BD
:206EA000D4F8801511F0340FC9D04FF40060FFF7FBFD002840F0278194F8982C12F00301AD
:206EC00000F0FD80D4F880150907BCD54FF40070FFF7EAFD0028B6D012F00305B3D19B4A92
:206EE000B4F9E836D91782FB0323C1EBA30109B21420FAF747FF29461C20FAF743FF94F854
:206F0000982CA0E7FF20FEF797FA002800F001810378FF2B00F09A8090F901100220FAF78B
:206F200031FFFF20FEF788FA002800F091800378FF2B00F08D80B0F90C20854B834893F8C5
:206F4000221002EB820202EB82029300490893FBF1F3D91780FB0320C1EBA00001B2032017
:206F6000FAF710FF94F86936002B79D1D4F880359A0640F198804FF40050FFF795FD0028C4
:206F800040F0CB80734D4FF48060FFF78DFD002840F04C816B8A94F8982C297DB3F5967F46
:206FA00002D9100740F1118194F89335002B40F0B280A1F1200307EE903A9FED677AF8EE74
:206FC000E77AF6EE006A67EE877ABEEE007AF5EEC07AF1EE10FA58BFB0EE667A77EE877A85
:206FE000FDEEE77A17EE903A19B20520FAF7CAFE4FF48050FFF758FD002840F0BD8094F84E
:20700000982C282A7FF425AF544A554B15685549A3FB0535AD09A1FB05367609A1FB063103
:207020004909C1EB0111A6EB81010902C6EB0616002309B21720A5EB860684F8983CFAF7E3
:20704000A1FE31B21820FAF79DFE02E7294665E700210320FAF796FE94F86936002B85D0D2
:207060000120FFF721FD002840F0F28094F86A36002B3FF47BAF0220FFF716FD002840F0DA
:2070800040810420FFF710FD00283FF46FAFB4F86C36002B00F0428129F0BAF801B20420C1
:2070A000FAF770FE62E71B07A9D52F4B93E8030002AB83E803001846FAF77AFE9FE74FF4E5
:2070C0008060FFF7F1FC00283FF4FCAE274BD4F8942CD4F8445B9A4240F2F080244BE91792
:2070E00083FB0523C1EB6313642101FB13510DB219B21020FAF746FE29462120FAF742FE13
:2071000094F8982CDEE6B4F9EA163020FAF73AFED2E6014602E709B267E794F844369F0798
:2071200059D44FF48060FFF7BFFC0A4D00283FF431AF002631460120FAF724FE314609204B
:20714000FAF720FE26E700BF50D6002067666666A82C0020706F0020E4380E3FCC2B002002
:20716000D34D62108988888888DD06083F4B4C001F85EB510050C34794F844260023920727
:20718000CDE9003347D494F89C3C012B43D0B4F98C355FED086A07EE103AB4F98E3507EE78
:2071A000903AB8EEC77AF8EEE77A27EE267A67EEA67ABDEEC77AFDEEE77A02A88DED027AD5
:2071C000CDED037AFAF7F4FD19E742F20F719942A8BF1946E8E6544D544BE9894FF4F36625
:2071E00006FB01F14909A3FB0131C9091120FAF7C9FDE9894E4B06FB01F1A3FB01214909B0
:20720000A3FB01235B09642202FB131109B21920FAF7B8FDB7E6D5E9002301216846CDE903
:20722000002384F89C1CFAF7C3FDE8E694F844369E077FF57EAFAB683D4AD91782FB030220
:20724000C1EB6211642606FB113636B209B272E794F8991C00293DD10B460620A4F89A3CE0
:20726000FAF790FDB4F89A3C0133A4F89A3C28F0C3FF94F8943594F8992C012B94F8973564
:207280001ED000EB800086B213B10AB1B6FBF2F6274BA3FB062343F34F113A205D09FAF7C5
:2072A00071FD642101FB1561224B89B20531A3FB0131C9083B20FAF765FDD7E60D4618E72D
:2072C0001BB112B1B0FBF2F080B201B23920FAF759FDCBE6B4F89A0CB4F84826B0FBF1F361
:2072E00001FB1303642000FB02129BB24900B2FBF1F2110241EA0311C2F30322114309B288
:20730000ABE7D4F87C360C49DA1781FB0313C2EBA30319B22820FAF735FDB2E6D4F88436DE
:2073200083F3100319B2BAE6706F0020C55A7C0A1F85EB51CDCCCCCC6766666603685A0640
:2073400007D513F4057F04D007298CBF00200120704703F48253B3F5825F03BFC81FB0FAD7
:2073600080F040090020704770B5BC4C94F89D3C012B84B000F04D8194F8A90CFCF79AF906
:2073800094F8AA3C834205461FD0002800F0D680D4F8783BCBB194F8912593F90400002A17
:2073A00018BF08224FF4964100230325CDE9015200911A46082133F016FBC4F8740B20B104
:2073C000FFF79AF9012384F8AA3C94F8AB3C012B00F0C180D4F8B46C3EB1A14B30465978C0
:2073E000FFF7ACFF002840F0F28094F8B90CFCF761F994F8B83C8342054621D0002800F0EB
:20740000F680EEB1337A002B00F01881954A02EB8303DB6994F8902596F904000093003ABF
:2074200018BF012202210023CDE901121A46102133F0D9FAC4F8380B10B1012384F8B83C68
:20744000D4F8BC6C3EB1864B30465978FFF776FF002840F0AC8094F8C80CFCF72BF994F83F
:20746000C03C8342054622D0002800F0C980F6B1337A002B00F0E5807A4A02EB8303DB695E
:2074800094F8902596F904000093003A18BF012202210023CDE901121A464FF4007133F00B
:2074A000A2FAC4F8C40C10B1012384F8C03C94F8C90CFCF7FFF894F8CA3C8342054631D059
:2074C00090B3694BD4F8CC6CD3F880344FF47A721A613EB34FF480524021304633F00EFA80
:2074E0000546F8B994F8903596F90400002B14BF0921082103224FF4E133CDE90121009374
:207500002A462B464FF4805133F06DFAC4F8D00C40B10123C4F80C0984F8E45884F8D45C0A
:2075200084F8CA3C04B070BDD4F8D00C33F0B8F9C4F8D05C84F8CA5C04B070BDD4F8740BB6
:2075400033F0AEF994F8AB3CC4F8745B012B84F8AA5C7FF43FAF94F8AC0CFCF7ABF805462F
:20756000002871D0D4F8B435002B7FF433AFD4F8B02C002A3FF42EAF94F8915594F89015E8
:2075800092F90400002D14BF08220022002908BF42F0010203254FF46141CDE90152009144
:2075A0001A46202133F01FFAC4F8B40512E794F8C03C002B7FF47BAFD4F8A43C002B3FF426
:2075C00076AF0122C4F8C43C84F8C02C6FE794F8B83C002B7FF434AFD4F8A43C002B3FF4DE
:2075E0002FAF0122C4F8383B84F8B82C28E7D4F8380B33F055F9C4F8385B84F8B85C1FE787
:20760000D4F8C40C33F04CF9C4F8C45C84F8C05C4DE7D4F8A05C124B28465978FFF78EFED8
:2076200020B3D4F84036002B7FF4A6AED4F8A43C002B3FF4A1AEC4F840369DE64FF4964319
:20764000E8E64FF461431BE7D4F8B40500283FF4C1AE33F025F9C4F8B455BBE650D6002037
:20766000406700202CDD0608F43D002094F8A80CFCF720F80646D8B1D4F84036002B7FF4DB
:207680007BAE002D3FF478AE94F8902595F90400B2FA82F252094FF416510225CDE9015213
:2076A00000911A46042133F09EF9C4F8400663E6D4F8400600283FF45FAE33F0F1F8C4F86D
:2076C000406659E670B5C94C94F89D3C002B00F0BF81082033F026F9C4F8780B00283CD0EE
:2076E000082133F015F900260346C149C14884F8A93C0522C4F8DC6C3AF040FA41F2085330
:207700000122BC48A4F8E03C84F8E42C0CF08AFC31462B22B84856F0DAF948F67C607D25E3
:20772000E02331462B22A4F8EC0CB44884F8EF3C84F8175D56F0CBF948F67C21A0224EF274
:207740007B0384F8435D84F8466D84F8EF5DA4F8181D84F81B2DA4F8443D94F8AB3C002B48
:2077600000F06081102033F0DDF81021C4F8B40C33F0CEF8A24B84F8B90C3A2140F23B1074
:2077800094F8692618809F254AF21E40197100219D7198601973002A40F00E8194F86A3686
:2077A000002B72D1D4F88035580700F1FE80990700F1F2801A0700F1E880924D2868C0F36D
:2077C000C010FEF755FF0020FEF738FF03464FF4007084F8703B33F0A5F84FF40071C4F8F1
:2077E000BC0C33F095F8D4F8F03D84F8C80C002B14BF0123002384F8F43D40F09280D4F8C8
:20780000903C002B14BF0123002384F8FD3D43D1D4F8A42F0023C4F8A03F002A00F0DC80BA
:20782000012284F89C3B84F8A82F002376487749C4F88C3B06223AF0A1F940F60943724833
:20784000A4F8903B0CF0EEFB4FF4805033F06AF84FF48051C4F8CC0C33F05AF8D4F8B03F6C
:207860006B4A6C4D84F8C90CC4F8102902F5A070591C0022C4F81409C5F89C31C4F8B01FC8
:2078800084F8CA2CBDE870406EE5D4F86C3B43F00403C4F86C3B85E7D4F88005002310F0DE
:2078A000020084F8FE3D84F8FF3D40F0EA80024694F869362BB10120FFF7F6F8002840F011
:2078C000F28094F86A36002B40F0E7800820FFF7EBF820B1A318042183F8001E01322B6837
:2078E0001B0600F101814C4B10219818053300F8011B8342FBD10521092042F2090384F894
:20790000051E84F8290F45494548A4F8343F2025042284F82A5F3AF031F941480CF082FBA0
:2079200076E794F869362BB10120FFF7BDF8002840F0BF8094F86A26002A40F0E2802B6815
:207940001B0600F1BA80D4F880154E070CD54FF48060FFF7A9F838B1A318082183F8F81D2D
:20796000013284F8FC2D4AE7080705D54FF40070FFF79AF80028EFD10905F2D54FF400607A
:20798000FFF792F80028ECD0E6E7D4F86C3B43F48073C4F86C3B10E7D4F86C2B42F46012B4
:2079A00042F0C002C4F86C2B04E7D4F86C2B42F40272C4F86C2BFAE6D4F86C3B94F86A26C6
:2079C00043F00201C4F86C1B002A3FF4EBAE43F03603C4F86C3BE5E6D4F8AC3F002B4BD0A1
:2079E000012384F8A83F84F89C3B1EE750D6002090DD060828E300203CE3002068E3002012
:207A0000886F0020F46E0020D8E1002038DE060870DF0020F404002050E40020E4DD060826
:207A20007CE50020202032F07DFFC4F8B00C00283FF498AE202132F06BFF354BC4F884350C
:207A400084F8AC0CFFF73CF8012384F8AB3C89E6042032F067FFC4F8A00C00283FF439AE7C
:207A6000042132F055FF2B4A84F8A80C0123C4F8882584F89D3C2CE684F8A83F84F89C3B1C
:207A8000E2E64FF46070FFF70FF800283FF40FAF012084F8000E02460AE70620FFF704F8F9
:207AA00000283FF413AFA318022183F8001E01320CE7012284F8F82D41E74FF4A050FEF7F8
:207AC000F3FF20B1A318022183F8F81D01324FF40850FEF7E9FF00283FF435AFA3180421AB
:207AE00083F8F81D01322EE74FF45850FEF7DCFF00283FF4F8AEA318082183F8001E013242
:207B0000F1E60620FEF7D0FF0028D2D1024616E701650108E1280108084B5A881B88801AA1
:207B20009B1AC00090FBF3F00628A8BF062020EAE070C0F19600C0B2704700BFB0DC002072
:207B4000074B084A33F81010127802EAD122520705D0DA6F511CD967134483F880007047A0
:207B6000ACE60020A806002010B5164B42681B7803F00303032B21D1134B1B88DBB1134B1E
:207B80001349B3F9BE30B1F904100A2491FBF4F15B1A1B0103F5B95314334FF4B471B3FBA0
:207BA000F1F3C3F1080303F00F0360331370436800225A7010BD05231370F8E72D23137046
:207BC000F5E700BF94DC002096DC0020ACE6002034DD0020436872221A70436873225A7032
:207BE000436874229A7043680022DA7070470F4B4268B3F904300A2193FBF1F31B0110B50A
:207C000003F5B9530A4C4FF4B4711433B3FBF1F303F00F031919E35813604B6853600B7AF9
:207C20001372436800225A7210BD00BF34DD002048660708044B93F8C53013F0FD0F14BFFB
:207C40009E209D20704700BFACE60020094B93F8C53013F0FD0F06D142F210735843064B24
:207C600090FBF3F07047242358434FF47A7390FBF3F07047ACE6002040D20600064B07EE98
:207C8000900A93F8C530B8EEE70A1BB9DFED037A20EE270A704700BFACE6002048F95140DD
:207CA00010B5104B93F82C21012A10D1D3F83021811A00290BDD0221B3F8264183F82C110B
:207CC0000949B1FBF4F142B10A44C3F8302193F82C01013818BF012010BD0844C3F8300186
:207CE000F5E700BFACE6002040420F00831E00F17A02EA2123F8021F9342FBD14E2243F607
:207D00004913C280CE2243850281CD2323228380A0F87220A0F87830704700BF08BB1F4848
:207D2000B0F8343103F001036BBB30B490F83841ACB11B4A02F1F00502E00133A3420ED0B1
:207D400052F8041B4904F8D590F8241200EB8101D1F8BC1145F823100133A342F0D130BCA9
:207D600070470E48B0F83421032A4FEA52030BD90A68A0F8343102F5C332A03203F0010336
:207D80000A60002BD1D070470B6803F5C333A03348F205020B60A0F834217047ACE60020C0
:207DA000E8E700202DE9F04100283AD12D4A92F8380180B32C4A2D4B92F804E092F905C041
:207DC00092F90680CEF1FF07AEF17F06FFB2F6B203EB800003F1F002002403E0834202F13D
:207DE000040218D053F8041B8904F7D5E1B2A1EB0C0181EAE175A5EBE175012D0DDC71B1C6
:207E0000414514BF394631468342D17004F1010402F10402E6D1BDE8F0810821F4E7714692
:207E2000F2E7114B1A79F02A09D802F10F000D4A18710B6803F582431A330B60B7E7094AC4
:207E400093F9054092F83A017F2584421D71987905DB4042C0B2987120445871E9E7002C7D
:207E6000FADAF6E7ACE60020A8060020E8E70020F0B5384E78B196F8AC32002B46D0364A61
:207E8000013BDBB286F8AC321378DC0741D4334B0A681A440A6096F838414CB3304B2E4F84
:207EA00003EB840403F1F001002503E09C4201F104011DD053F8042BC2F303200628F5D157
:207EC0003878C00715D596F8AC0296F83BE100EB050CBCFBFEF00EFB10C00128CCBF00200D
:207EE000012058B99C4205F1010501F10401E1D1F0BDE84300F001000028F3D0C2F383429F
:207F000006EB8202D2F8BC210A60EBE796F83B31B5E7D6EDAF7A134B134CFDEEE77A6420FA
:207F200017EE902AA2F57A7200FB02F283FB0230D317C3EBA01303EB4303C3EB031384FB9E
:207F40000302DB17C3EB62130533084A92FBF3F39EE700BFACE6002008DC0020400D0300C0
:207F6000E8E70020D34D62101F85EB5140420F00F0B4524C002868D194F8F802002856D098
:207F80004F4BD3ED007AB3EE097AF4EEC77AF1EE10FA4EDCBBEE097AF4EEC77AF1EE10FA7B
:207FA0004CBF08270027D3ED017AB3EE097AF4EEC77AF1EE10FA3EDD47F0010794F8385186
:207FC000ADB3404ADFF808C102EB850502F1F00014E094F9FB62B142ACBF0221002194F9B0
:207FE000FC62B3421CDB41F004010F421CBFDCF80C300360954200F1040018D052F8043B25
:020000040801F1
:20800000D903F7D594F9FA6203F00F01B142C3F30313DEDC94F9FC62B3424FF00101E2DA76
:2080200094F9FD62B342D8BF41F00801DDE7F0BC70470427B7E7BBEE097AF4EEC77AF1EE70
:2080400010FA48BF47F00207B8E794F8F93263B31B4B1D4DD3ED007A93ED017A0A6894F860
:20806000F802F0EEE77AB0EEC77AF4EEC77AF1EE10FAB8BFF0EE477AFDEEE77A80F0010009
:2080800017EE903A193B03EB4303C3EB031385FB0365DB17C3EBE51305330C4DB5FBF3F31E
:2080A0001A440A6084F8F80268E70B6894F8F80203F5433303F5A0730B605FE7ACE600205E
:2080C000A0DC0020E8E70020353AFC4440420F00C0DE0608F0B40B4F97F8386186B107F5D0
:2080E0009E72054607F50B77002352F8044B35EA040004BF086847F823000133B342F4D145
:20810000F0BC7047ACE6002030B42A4B60B92A48027DCAB993F825322849203301EB83014E
:2081200030BC4FF4A060D5E793F8FE22F2B1013A214883F8FE220A6802F5C32202F52072F0
:208140000A60027D002AE5D01D4A12689106E1D51C4A93F8FE12127892071AD511BB93F8BF
:2081600027321649203301EB8301D9E7124893F8FF42057DA54205D8042483F8FF2283F819
:20818000FE42D8E70134012283F8FF4283F8FE22D1E70029BED193F826320849203301EB4E
:2081A0008301BDE793F823320449203301EB8301B6E700BFACE60020706F0020E8E70020AB
:2081C000D0DB002094DC002010B41E4A48B91E4C92F800030B6823440B6098B15DF8044BEE
:2081E000704792F8013303B3012B16D092F800030B68164C80F00100234482F800030B6020
:208200000028EBD192F8233211495DF8044B203301EB83014FF440705CE792F800030D4CBE
:2082200080F0010082F80003D4E70B685DF8044B03F5742303F5107301200B6082F800036B
:20824000704700BFACE6002040420F0048E80100E8E7002020A107003C4AA0B992F80233DF
:208260006BB192F803138A081341DB070AD501F00101032A06D8DFE802F05048403892F84A
:20828000053353BB704792F80333013303F00F0382F803333BB192F80233086800F5C33035
:2082A000A0300860DCE72A4882F80233437A002B44D12848C07818B143F0040382F802334B
:2082C00025480078C00730D592F804030028E4D043F0080382F80233DFE792F812331F4996
:2082E00001EB83014FF40030F4E61C4B03F13002002914BF19461146F4E7194B03F1180235
:2083000000290CBF19461146ECE7144B03F10802002914BF19461146E4E7104B03F118029D
:20832000002914BF19461146DCE70E4800680028CAD043F0010382F80233C5E792F80133F8
:20834000002BB6D0022382F80233B2E7ACE60020B0DC00200CDC002008DC0020C0DE0608E9
:20836000D0DE06089CE1002030B4022340F203154FF4FA74322146F20142C3700023858077
:20838000C480018130BC42810380704770B40B4C0B490C4B22680E680D6883F82C030021C8
:2083A00022F0200283F83013C3F81C63C3F828532260C3F8241370BC704700BFD0DB00207A
:2083C000CC2B0020ACE6002090F8603043B942690121072082F84430A2F8460082F848102C
:2083E000704700BF034A0123E021C37351701846704700BF94E300204FF0FF30704700BF4F
:208400004FF0FF30704700BF704700BF002070470020704770B4067AAEB1427A0B48002121
:208420002025002352B1142B05DC072903DCC45C202C18BFC55401339342F4D101318E4276
:2084400000F11500EDD1002070BC704797E3002010B50024C4730121FFF7DCFF024B012238
:208460005A70204610BD00BF94E3002070B403980378ABB10C4C02EB4205C5EBC5052544A4
:20848000142901F1010406D8072A294403D8CE789E4218BFCB7010F8013FE1B2002BEFD153
:2084A000002070BC704700BF94E3002014299DF800000CD8072A0AD8064B02EB4202C2EB6B
:2084C000C2021A441144CB78834218BFC8700020704700BF94E30020027A407A02FB00F0BE
:2084E000704700BF027A407A02FB00F0704700BF002070474FF0FF30704700BF034B93F8D9
:208500002121027293F822314372704758E4002000207047002070470120704700207047A2
:20852000027A407A02FB00F0704700BF002070470123C373184670470123C37318467047ED
:208540004FF0FF30704700BF704700BF002070470120704700207047027A407A02FB00F018
:20856000704700BF002070470120704700207047914201D0012A01D9002070470129FBD882
:2085800008B5074BC1EB0110C2EB021203EB421103EB40104FF4F07255F038FA012008BDCD
:2085A0003845002001299DBF024B012083F8341300207047ACE6002001298CBF0020012029
:2085C000704700BF4FF0FF30704700BF034B1B68186A003818BF0120704700BFFC480020E4
:2085E00030B41D299DF808000DD80F2A0BD8074B074D93F834431E23C4EB041413FB0212E1
:2086000002EB44125055002030BC7047ACE6002038450020014B1889704700BFA80600202F
:208620000020704700207047074BB3F88A14B3F88C24034610B4054C1C6001205DF8044BF7
:2086400019815A81704700BFACE60020F8DE0608064AB2F880340BB91846704792F88834CC
:20866000037292F88934437201207047ACE6002000207047034B93F8890493F8883400FB80
:2086800003F07047ACE6002000207047034B0449B3F90A304068012242F0A8BEA8060020F5
:2086A000CA5E0708064B07491A88074B40681B68534342F2107293FBF2F242F097BE00BFBF
:2086C00098DC00201A5F0708CCDC0020054A064992F8A53492F8A42440680133013242F022
:2086E00085BE00BFACE600201F5F07080B4B4068B3F904300A2293FBF2F31A0102F5B9529F
:208700004FF4B4711432B2FBF1F2C2F1080202F00F020349603242F069BE00BF34DD002034
:20872000255F0708034A044992684068072342F05DBE00BFCCDC00202C5F070807B5144AB8
:20874000406892F8B414B2F8B634012909D1009392F8B8340F497B2242F048FE03B05DF809
:2087600004FB022906D10C497B2203B05DF804EB42F03CBE0A22534340F2FF32B3FBF2F32B
:208780009BB2092B054928BF09237B22EDE700BFACE60020325F07086A6007083C5F0708F2
:2087A00013B54468FFF746FA0F4B1B789B07024612D50E4B93F8C3140D4B59B19889FFF71D
:2087C00045FA0C49009203467022204642F00EFE02B010BDD889F2E7009007492D23702279
:2087E000204642F003FEF3E794DC0020ACE60020706F002044600708425F07082DE9F0411B
:208800003F4F90F800C03C78416890F803E0BCF1170F0CBF4FF098084FF0890814F0040461
:2088200086B0064605D0374BBCF1170F0CBF5C681C68354D84EAE473A3EBE473BEF1010F8E
:20884000B3FBF5F201F1010005FB123343D0BEF1020F44D181F800803C214B43B3FBF5FEDE
:2088600005FB1E334B43BCF1170FB3FBF5F105FB1135264BB5FBF3F528D1002CB4BF572351
:20888000452305932223CDE903532723CDE900E3029108231E4942F0A9FD33781D495A0933
:2088A00001EB820103F01F03012202FA03F33A78D1F8C80402F00602042A0CBF034320EA95
:2088C0000303C1F8C83406B0BDE8F081002CB4BF53234E23D5E74FF47A75B3FBF5F3002CDB
:2088E00081F8008002DA2D24881C4C700A4C0B49BEF1000F08BF214642F078FDCDE700BF42
:2089000094DC0020706F00208096980040420F00595F0708ACE60020495F0708515F07089A
:20892000034B0449D3F8D024406842F05FBD00BFACE600206F5F0708044B1B78DB0703D4FE
